:020000040800F2
:100000000000022089350108CF350108D1350108EB
:10001000D3350108D5350108D735010800000000A7
:10002000000000000000000000000000D9350108B9
:10003000DB35010800000000DD3501089DC800081F
:10004000E3350108E5350108E7350108E935010820
:10005000EB350108ED350108EF350108F1350108F0
:10006000F3350108F5350108F735010891E400087A
:10007000FB350108FD350108FF350108013601088F
:1000800003360108E9E400080736010809360108CB
:100090000B3601080D3601080F3601083D1901081D
:1000A00013360108153601081736010819360108FC
:1000B0005DF100081D3601081F3601081DE5000826
:1000C000233601082536010827360108293601089C
:1000D0002B3601082D360108B1C800083136010859
:1000E000333601083536010837360108393601083C
:1000F0003B3601083D3601083F360108413601080C
:1001000043360108A5E000084736010849360108D2
:100110004B3601084D3601084F36010851360108AB
:1001200053360108553601085736010885E00008A6
:100130005B3601085D3601085F360108613601084B
:1001400063360108653601086736010885E4000852
:100150006B3601086D3601086F36010871360108EB
:1001600073360108753601087736010879360108BB
:100170007B3601087D3601087F360108813601088B
:10018000833601088536010810B5054C237833B94C
:10019000044B13B10448AFF300800123237010BD5A
:1001A0003801002000000000207F0108084B10B536
:1001B0001BB108490848AFF300800848036803B939
:1001C00010BD074B002BFBD0BDE81040184700BF07
:1001D000000000003C010020207F010834010020C5
:1001E00000000000154B002B08BF134B9D46A3F5E4
:1001F000803A00218B460F461348144A121A13F016
:10020000F2FE0F4B002B00D098470E4B002B00D076
:1002100098470020002104000D000D48002802D05E
:100220000C48AFF3008013F0FBFD2000290000F024
:1002300013F813F037FA00BF000008000000022096
:1002400000000000000000003801002040C4012030
:1002500000000000000000002DE98048D3B00DF040
:1002600085FEBD4B9A6802F00C02042A08F00E8647
:10027000082A08F0F085B94BB94A1A60B64EB94F52
:10028000B168B94CB94ADFF818C3B948B94DC1F3E0
:1002900003114FF0C808795C1F68CCF8008027FA7A
:1002A00001F18F09A4FB0774A409196004F1FF3E52
:1002B0000721F02400270523C2F804E085F8234035
:1002C0009760116003608DF85270336C4FF080447A
:1002D00043F001033364238823F45C731B044FF061
:1002E00001081B0CD1222380E1622285A4F814802E
:1002F000A3899BB243EA0803A3811C220F2310A801
:100300008DF840208DF841308DF842308DF84380D3
:100310000CF044FC2288984B92B242EA08022280F8
:100320001A68B2F5E13F08F0B6854FF4E1321A6081
:10033000336B924D43EA08033363336B43EA08039C
:100340003363336C04F5003443F400333364236ABD
:1003500023F470632362236A43F4E0632362236A15
:1003600023F470432362236A022143F4E0432362AF
:100370000322204604238DF8441010A98DF845204F
:1003800010938DF846708DF847800CF0B3FB204633
:10039000082310A910930CF0ADFBAB896FEA43431F
:1003A0006FEA53439BB2AB812B8A23F440531B0467
:1003B0001B0C2B82AB899BB223F4B05323F00C03AC
:1003C00043F00C03AB81AB8A23F440731B041B0C7A
:1003D000AB8212A80CF042FBAA89149B674812F466
:1003E000004F03EB8303664A03EB8303A2FB032363
:1003F00014BF5A0C9A0C634BA3FB02418489480931
:10040000642100FB11210201200408F11A85090171
:100410003231A3FB0113C3F3431343EA0201574BE9
:10042000594A89B21981998989B241F40051998157
:10043000136843F02003136000242623012512A82B
:100440008DF848308DF849408DF84A408DF84B5072
:100450000CF0A4FB474B4D4ADA6031238DF84B502A
:100460008DF849408DF84A408DF8483012A80CF0BC
:1004700095FB9DF84B303B2101228DF848108DF8FB
:100480004920002B48F0D884414B4FF00062C3F85C
:100490008420314D3F4C2B6B3F4F43F00C032B63BB
:1004A000636A23F00F036362636A43F00C036362C1
:1004B000636A23F0F0036362636A43F0C00363621C
:1004C000636A23F470636362636A43F44063636244
:1004D000636A23F470436362636A43F44043636274
:1004E000636A23F470236362636A43F440236362A4
:1004F0003B6A23F470633B623B6A43F440633B62B4
:100500004FF4706202232046002612A94FF0010822
:1005100012928DF84D308DF84C308DF84E608DF87C
:100520004F800CF0E7FA3846042312A912930CF01E
:10053000E1FA20464FF4805312A912938DF84F60D0
:100540000CF0D8FA6B6C154843F400636B642B6BAA
:1005500043F480032B6325E0003802407000002044
:100560000024F40060000020632D3E0510E000E050
:100570001400002000ED00E0381E00200044004080
:10058000C5B3A2911F85EB510C4400400006FA054B
:1005900000E100E000080240000C0240245E010877
:1005A000740000200CF038FA434B444918689F88C7
:1005B0000C901A4653F8080F0E9052F8100F9C88B2
:1005C0009388ADF844300A683D4BADF834709A42D8
:1005D000ADF83C40109048F0A1835523F022022151
:1005E00012A88DF849308DF8482012F067FD0346B7
:1005F000002808F02C83334B07931B68002B08F06E
:100600002083314E0BAD3368022B0CBF2F4830488E
:100610000CF002FA2F4F3B68002B40F00483DFF808
:10062000C490DFF8C4B0DFF8C4801C469A4612A814
:10063000C5F80090CDF830B0CDF848900BF0E6FB4F
:10064000031E4FF000020CA9284651DB58F8236026
:100650000EB186F800A00C9E0EB186F800A00C9E8C
:1006600048F823600CF0C2FA0328064607F01D8004
:10067000002808F04C84184B05931B68174AD8686B
:10068000174914F0B1FD731E122B08F24A84DFE8FB
:1006900013F0234419441B3802383C0333032A0364
:1006A0002103F402EB023700E20218030F030603F2
:1006B000FD02D902D0020F440C5E0108A41D0020E7
:1006C000801A060020B8012030B801205C5E0108C5
:1006D000745E0108A81D002024010020E45E0108CA
:1006E000EC5E0108A45E01086C030020441E00209B
:1006F000BD4B05931B68BD4ABD49D86814F074FD15
:10070000059BBC481B682022DB68012114F0CCFD4E
:10071000DFF8FCA2B84CDAF83030DFF8F882B74DD9
:10072000B74EB84F43F001034FF00009CAF830301C
:100730004FF0010B2046C02312A912938DF84CB044
:100740008DF84D908DF84E908DF84F900CF0D2F9B9
:10075000402323834FF080032383DAF8303043F0C3
:100760000403CAF830304FF40054404612A98DF803
:100770004CB012948DF84D908DF84E908DF84F90AE
:100780000CF0B8F9A04BA8F81A40C3F80090DAF8BA
:10079000303043F01803CAF830304FF2B3732846B4
:1007A00012A912934FF003038DF84D304FF6807865
:1007B0008DF84C908DF84F900CF09CF9304612A9B2
:1007C000CDF848800CF096F9DAF8303043F0780331
:1007D000CAF830304CF233734FF0030228461293BC
:1007E00012A94FF002038DF84D208DF84C308DF892
:1007F0004E908DF84F900CF07DF92B6A23F00F038B
:100800002B622B6A43F00C032B622B6A23F0F0035C
:100810002B622B6A43F0C0032B622B6A23F47023F4
:100820002B622B6A43F440232B622B6A23F4700360
:100830002B622B6A43F440032B626B6A23F00F0395
:100840006B626B6A43F00C036B626B6A23F0F0031C
:100850006B626B6A43F0C0036B626B6A23F4706374
:100860006B626B6A43F440636B626B6A23F0706384
:100870006B626B6A43F040636B626B6A23F0704398
:100880006B626B6A43F040436B62304612A9CDF84D
:1008900048800CF02FF9336A23F070433362336AD7
:1008A00043F040433362736A23F00F037362736A49
:1008B00043F00C037362736A23F0F0037362736A8C
:1008C00043F0C0037362736A23F470637362736AE4
:1008D00043F440637362736A23F470437362736A10
:1008E00043F440437362736A23F470237362736A40
:1008F00043F440237362736A23F470037362736A70
:1009000043F440037362736A23F070637362736A23
:1009100043F040637362736A23F070437362736AD7
:1009200043F040437362284612A912940CF0E2F897
:100930006B6A364E23F470036B626B6A43F44003B8
:100940006B622846802312A912930CF0D3F82B6A0D
:1009500023F070432B622B6A43F040432B62DAF89A
:1009600038304FF0204143EA0B040F200D2241F2B2
:100970001003CAF8384012901492CDF84C90CDF87C
:100980005490CDF85890CDF85C90CDF860900B6005
:10099000129B0393039A189B139D149C1698134360
:1009A00043EA0513159A43EA042343EA0243179ADC
:1009B00043EA005343EA02626FF070434A603360D7
:1009C0000B684FF0C04443EA0B030B6014200BF09C
:1009D00045FFA4F800B00A200BF040FFCB23238092
:1009E00039224FF02C0317E024010020E45E0108B7
:1009F000EC5E01085460010800000240000C024057
:100A00000010024000000860EC360020040100A045
:100A100000380240000802403A804FF0C10B3B8092
:100A20003421CF2030254FF0E80E85264FF0780C8A
:100A3000EA234FF00202A7F800904FF0ED0A398048
:100A40004FF0F7083A80122120808122A7F8009009
:100A50006420A7F800B03D80A4F800E03E80A7F82D
:100A60000090A7F800C023804FF0200C4FF0030344
:100A7000A7F800904FF0230EA7F800901026A4F8D6
:100A800000A0C52538803B803E20398086233A80EF
:100A90002821A4F80080C722A7F800C04FF0C00C9E
:100AA000A4F800C04FF0B60AA7F800E04FF008081D
:100AB000A4F800B03E804FF0180B2580F226388055
:100AC000B125398022803B800EF0B2FE55224FF0D6
:100AD000820C4FF0270E3A23112123800A203A80FE
:100AE0002580A7F80090A7F800B0A4F800A0A7F808
:100AF0000080A7F800C0A7F800E02680A7F80090C3
:100B000021800BF0ABFE292323804846EF210EF015
:100B1000C5FE484640F23F110EF0ACFE4FF02C03EC
:100B2000238038464C464FF4A072F02101390480EE
:100B30004FF00003FAD1013AF7D17849784C784D5B
:100B400003C92064080CA4F8441085F84600012469
:100B5000744975482B7085F88120C5F8C42085F844
:100B6000C93085F8C83085F8804013F027F805466D
:100B7000002800F008816D4F2A464FF4807112A8BA
:100B800012F024FF002800F0F980232112A814F0AD
:100B900055FF0446002807F041800023037012A887
:100BA00014F06CFF0028E7D0431E12A90B44C01AB2
:100BB0001A78093AD2B227FA02F1172A01F0010293
:100BC00004D882F00101002A47F032803D2112A8AA
:100BD00014F034FF03460028CED00022027054499E
:100BE00012A85C1C14F00CFF0646002807F00C80CD
:100BF000504912A814F004FF0646002806F0FA87B0
:100C00004D4912A814F0FCFE002846F082874B499B
:100C1000204614F0F5FE002846F06F87404A012375
:100C200082F88030A8E7464B4648059314F0AEFEA4
:100C30006EE5059B44481B682222DB68012114F005
:100C400033FB65E5059B41481B682A22DB680121CF
:100C500014F02AFB5CE5059B3D481B681822DB6805
:100C6000012114F021FB53E5059B3A481B68222221
:100C7000DB68012114F018FB4AE5059B36481B6828
:100C80002122DB68012114F00FFB41E5059B33486D
:100C90001B683B22DB68012114F006FB38E5059B4D
:100CA0002F481B684122DB68012114F0FDFA2FE573
:100CB000059B2C481B682422DB68012114F0F4FA00
:100CC00026E5059B28481B681D22DB68012114F0DE
:100CD000EBFA1DE5059B25481B682722DB680121EF
:100CE00014F0E2FA14E5059B21481B683922DB6801
:100CF000012114F0D9FA0BE5059B1E481B681C2244
:100D0000DB68012114F0D0FA02E5059B1A481B6844
:100D10001A22DB68012114F0C7FAF9E4D86101084E
:100D200038B70120E0610108E46101081300800088
:100D3000F0610108F8610108FC610108086201081E
:100D400024010020A85E0108886101085C61010897
:100D500078600108306001080C600108206101081A
:100D6000DC600108B460010894600108E45F0108D8
:100D7000A85F0108885F01086C5F01080FF016FA90
:100D8000284612F0F5FCB04BD3F8C42012B901226A
:100D9000C3F8C4208022AD49AD4814F077FE11F0AD
:100DA00075FF12F017F8A84BD3F8C430DD0752D501
:100DB000A84CA948236B43F002032363002580233A
:100DC00012A912938DF84C508DF84F500BF092FEF3
:100DD000616CA24AA24B41F480416164D16821F464
:100DE0007041D160D16841F48051D160196821F01F
:100DF00080011960596821F080015960196841F03B
:100E000080011960996821F080019960D96821F00A
:100E10008001D960D2F80C3443F08003C2F80C345E
:100E200010A8012317228DF841308DF842308DF83B
:100E300043308DF840200BF0B1FE236B864843F021
:100E40000203236312A940238DF84C508DF84F50B4
:100E500012930BF04FFE7C4BD3F8C4309C0706F185
:100E60006184794BD3F8C4305C0724D50024794BD6
:100E7000139412941A6B7B4F7B4842F01402FF26A6
:100E80001A6301253E833F2312A98DF84C408DF84B
:100E90004D4012938DF84F500BF02CFE384612A99E
:100EA00012968DF84C508DF84E508DF84F408DF8BD
:100EB0004D400BF01FFE6D4B0393DFF808B26C4BF7
:100EC00004936C4B6B491B68002B40F0D1826A4B3A
:100ED000694A1B68002B40F0DC83684B1B78002BB1
:100EE00040F08A80664B1878002840F08580654A7B
:100EF000654B11881B78654A624D1180624A002B50
:100F000062D0634B624C1B78002B5DD010708B0B52
:100F1000604A207052F82320C1F30D03D35C594A74
:100F2000762B04BF4B1C2B805B4B10881B88013B2E
:100F30009AB2594BB2F5804F1A800DD3B2F5B64F25
:100F400002D2564901230B70930BC2F30D01514A93
:100F500052F82320030A53544F4B1B88013B9AB28B
:100F60004D4BB2F5804F1A800CD3B2F5B64F02D27A
:100F70004A4901230B70930B4649C2F30D0251F805
:100F800023309854464B1B78012B40F2C281022B30
:100F90001AD1444B444A1B7816683E4C1902481C2F
:100FA00082138B0B54F8225054F82340C0F30D02E7
:100FB0003D4806F11303C1F30D010360AA5C635CB5
:100FC00003EB02232F4A13802E4B1A8840F2625300
:100FD0009A4207F0228040F2C2439A4206F0E68726
:100FE000324B1B7803F0FF02002B06F01987304BC1
:100FF0001B68002B46F02386224B264C19882D4B6C
:1010000018688B0BC1F30D0254F823309C5C002848
:101010007AD043F6FE43994206F0D78243F6FF4367
:10102000994271D1244B1B68002B06F0C682234BDA
:10103000234A1B682149D25C0133802B0B6008BF17
:101040000023D2B240E000BF38B7012078B70120BA
:1010500040BD012000380240000402400038014039
:10106000003C014000080240001002400040001017
:10107000F07601205C220020341E0020C1BD01203A
:10108000C2BD01203CBD012071BC01202CBD01204E
:10109000580200200CB701207CBC012091000020E8
:1010A00070BC0120501E0020C4BD0120780000202B
:1010B0005821002030BD0120481E0020A00500203E
:1010C000AC1D0020E0BC012008BF0B6072B60C4BC9
:1010D0000B491B68013B0B6062B69BF806308BF82E
:1010E000072043F001030D2A8BF806300CD1054B85
:1010F0005B6803F5E1521C322023137004E000BF4B
:10110000481E00200CB70120FF2C06F24982DFE8C0
:1011100014F03B321032EC31C6317B311431F530F2
:101120008E30733035300D30E72F9C2F442F252F14
:10113000F72EC72E9C2E782E332E8D2DDB2D612D74
:10114000172DFF2CC12CA62C802C352CD02BB12B8D
:101150005E2B402BD62A762AC14577451A45FC449A
:1011600087445C44AB436943E6429C423F42214290
:10117000F141D341AC417241EC485B48A54743473C
:10118000CE46B04674464546DC499149284909494E
:10119000234AFA49FA49FA49FA49FA49FA49454AC1
:1011A000FA49F43FF43FF43FF43FF43FF43F7D51FC
:1011B000F43FF750F750F750F750F750F750A04C66
:1011C000F750764C764C764C764C764C764CA64E58
:1011D000764C8A4E8A4E8A4E8A4E8A4E8A4E194BD9
:1011E0008A4EFD4AFD4AFD4AFD4AFD4AFD4A2B5002
:1011F000FD4AC24FC24FC24FC24FC24FC24FE64B11
:10120000C24FBD4BBD4BBD4BBD4BBD4BBD4B9D50B0
:10121000BD4B1B4D1B4D1B4D1B4D1B4D1B4DC14055
:101220001B4D1F401F401F401F401F401F405B546D
:101230001F402C522C522C522C522C522C52AC535C
:101240002C52F34BF34BF34BF34BF34BF34BF0526A
:10125000F34BA54DA54DA54DA54DA54DA54DF34D64
:10126000A54D924A924A924A924A924A924A0C5503
:10127000924AE74EE74EE74EE74EE74EE74E334FD2
:10128000E74E4B4B4B4B4B4B4B4B4B4B4B4B5B55F5
:101290004B4BF44C9F524C2A2F28C12778271A27F2
:1012A000D3269C267A265026A7213821DD207820B7
:1012B00031200020D31FA91F8A1F281FDF1E711E87
:1012C0002A1E041ED11DA71D8A1D181D071DA21C44
:1012D000091CD41BA21B781B091BA71A261AED197F
:1012E0008B1953193F191519F91897180708BF07D3
:1012F000780752072507FB06D90677062706F1056A
:1013000097055F0546051D050F05AF049F044304BF
:101310000F01054B04491B6803F10D020A60034AE3
:10132000382313805CE600BFC4BD01203CBD012012
:10133000A74BA8491B880888A74A013B99B2431CC0
:10134000A34812680180A4480B32B1F5804F0260B7
:1013500098B20DD3B1F5B64F02D2A04A0123137053
:101360008B0B9F4AC1F30D0152F82320030A5354FB
:10137000974B1B88013B9AB2954BB2F5804F1A8070
:101380000CD3B2F5B64F02D2944901230B70930BE4
:101390009349C2F30D0251F8233098548D4A3823F3
:1013A0001380904B1B7813B98F4B1B785BB18F4B1D
:1013B0008E4A1B78002B00F048828A4900230B706C
:1013C000894913700B708A4B834A1B6812688249E3
:1013D00013F0030F40F29F2318BF4FF428739A4273
:1013E000FFF46FAD834804688348D0F8C400D31A73
:1013F00042070B6004F10A0500F138827E4BD3F8F6
:10140000C4309B0702D500200CF09AFB079B1B6899
:1014100073B17A4B1968002940F02482784B784ADE
:101420001B680133642B136002D111600DF01EFFA5
:10143000714BD3F8CC30002B00F00A82714B1D6049
:101440006B4B6C491A686F4B1B680B60531C684AE6
:10145000642B136011467FF434AD00220A606A4A9F
:101460006A4901231370694B1B68002B3FF42FADB1
:10147000674B67481B780133DBB20022102B0370E7
:101480000A6007D1634B02701B78624AB3FA83F398
:101490005B091370604B1B682BB1604B1A78604B73
:1014A0001B789A4228D05E4B5E4A1B78002132F8A6
:1014B000134000940846182340F23F120CF090FBB2
:1014C000D8231F221921002000940CF089FBD82377
:1014D00040F23F1219214FF4907000940CF080FB01
:1014E000F12340F23F120094D92100200CF078FB48
:1014F0004B4B4A4A1B781370454B1B7823B1374B33
:101500001B78002B3FF4E3AC4FF480430693069B1B
:10151000BDF818809B1003F03801069BC3F302222C
:101520005B1103F0C0030A431A43D3085B0103F5C0
:10153000B04902F1190A20273B4B1B68002B06F02B
:101540005E80049AC8F30D03D65C384B04931A46A8
:101550003149C9F30D030968D25C39B1344B4344B6
:10156000A3F580431B78B34206F05280304B4344CE
:10157000A3F5804311061E7006F15A80C2F3C2051E
:1015800002F00704530605D505F1080204F108032B
:10159000D5B2DCB2514650460EF080F9F91D3846FE
:1015A0000EF068F94FF0C0422C23138080210822EE
:1015B0001C4B20480E4214BF33F8143033F815305A
:1015C0000380531E9AB24908002AF1D134E000BFCB
:1015D0007CBC01203CBD0120C4BD01209100002045
:1015E0000CB70120C1BD0120C2BD0120DCBC01201F
:1015F0006C2200207022002038B701202CB8012076
:101600007422002054010020580200205C22002097
:1016100068030020542100201CB701201000002086
:101620007EBC012070630108F0B60120F076012035
:10163000A405002000000860083708F1010209F144
:101640000103B7F5907F1FFA82F81FFA83F97FF440
:1016500073AF069B2033B3F5B04F06937FF457AFBB
:101660009B4B9C4A19689C4B9C48002914BF11460F
:1016700019464FF4407212F0ABFC994901220A60FE
:10168000984A00231370984B974A1B68002B3FF42D
:1016900024AC002495499648146012F08FFA07464E
:1016A000002807F079818DF825408DF826408DF8C7
:1016B000274011F08FFB8F49384611F069FA8E49A7
:1016C000384611F065FA8D49384611F061FA8C49B7
:1016D000384611F05DFA8B49384611F059FA8A49BB
:1016E000384611F055FA8949384611F06BFA8849A5
:1016F000384611F067FA8749384611F049FA0DF17A
:101700002701384611F044FA0DF12501384611F051
:101710003FFA9DF82530FF2B07F0388103F02003B6
:1017200003F0FF02002B47F0258115469DF8253078
:10173000794A7A49C3F342033846137011F028FA04
:101740007749384611F024FA7649384611F020FAE4
:101750007549384611F01CFA7449384611F018FAE8
:101760007349384611F014FA7249384611F010FAEC
:101770007149384611F00CFA7049384611F008FAF0
:101780006F49384611F004FA6E49384611F000FAF4
:101790006D49384611F0FCF96C49384611F0F8F9FA
:1017A0006B49384611F0F4F90DF12601384611F075
:1017B000EFF99DF82630002B07F0D880654A012309
:1017C00013706549384611F0E3F90DF126013846EA
:1017D00011F0DEF94D4A9DF8263014885F4A03F077
:1017E00003031370002C07F0DC80D5B94FF480445C
:1017F00001250DF12601384611F0CAF9B4F5B64FAE
:1018000038BF38489DF8262038BF0570A30B5448D0
:10181000C4F30D0150F823300134B4F5803F5A541D
:10182000E7D13A4B4F4A1B8813804F4B00241C7062
:101830004E4B1C704E4B1C704E4B38461C6011F0CA
:1018400097FF4D4B1C70FFF748BB01231370BAE59F
:101850004A4B1B689D427FF6F3AD484B1B689D4287
:10186000F6D8EDE501200DF05BFDE1E5444B444C7D
:101870001B68FBB1012B7FF4C1AD424B1B69DBB28E
:1018800003F0200203F03F0102F0FF030AB93E4AD1
:1018900013703E4B1A68184661F01F033C498B5485
:1018A000531C082B0360364A04BF00230360002347
:1018B0001360A3E5354B37481B68012101FA03F398
:1018C000DB43DAB2FF2343830283216096E500BF46
:1018D000F0B60120F08E012000580010541E0020A8
:1018E0001CB7012091000020341E00204462010832
:1018F0005C210020E7BC0120E6BC0120E1BC012006
:10190000E0BC0120E5BC0120E4BC01203CBD01207D
:101910007CBC0120501E00207EBC0120E3BC0120C5
:10192000E2BC012061BC012060BC012063BC01203D
:1019300062BC012065BC012064BC012067BC0120A1
:1019400066BC0120EBBC0120EABC0120E9BC0120FF
:10195000E8BC012071BC01205521002070BC012091
:101960000CB701202CBD0120DCBC0120C1BD012031
:10197000C2BD0120C4BD0120580200205401002036
:101980007822002000100240780000206003002030
:10199000E436002000080240A04BA14F1E88A14B56
:1019A0009BF807401D68A048731C9BB29A0BC3F3B9
:1019B0000D0157F82220994F3B80EB1D994D2B606C
:1019C000515C04F00F0201F00F03D31A13F0100F53
:1019D000837914BF43F0100323F01003837181EA6D
:1019E0000403621A1F0695B23BD584EA02031C0663
:1019F00037D59BF8063043F004038BF806309BF88C
:101A00000630E8054CBF43F0010323F001038BF8D7
:101A100006309BF8063015F0FF0F14BF23F040038B
:101A200043F040038BF806309BF8063029064CBF84
:101A300063F07F0303F07F038BF806309BF80630DA
:101A40007649B21C43F002030A808BF80630A8E402
:101A5000724B72491B885A1C0A80744A0123137006
:101A6000A5E49BF8063023F004038BF80630C6E7A4
:101A70006A4B6B481C889BF80650631C9BB29A0B00
:101A8000A11C50F82200654A1380C3F30D0289B2ED
:101A90008B0B805C624A52F82320604B1980C1F3A3
:101AA0000D035E49D35C00EB03239EB22B0637D5B2
:101AB0005F4B5C4A1B881068013BE11C9AB200F145
:101AC000110388B25A490A805649B2F5804F0B601B
:101AD0000DD3B2F5B64F02D2564901230B70930BCA
:101AE000C2F30D014E4A52F82320030A5354504BBF
:101AF0001B88013B9AB24E4BB2F5804F1A800CD333
:101B0000B2F5B64F02D24B4901230B70930B4449F7
:101B1000C2F30D0251F823309854404B1E8040E42C
:101B2000404BE21C1B680A803E4A0A33136038E4CB
:101B30003C4B3A4A1B683B49128804330B603749D7
:101B400001320A803C4A012313702AE4334B9BF88C
:101B500006501C88334B1E68631C9AB2A31C98B2B3
:101B6000910B2F4B53F821102C4B1A8006F10A03CE
:101B70002C4EC2F30D023360895C294A830B52F864
:101B80002320264B1880C0F30D03D35C234A01EBBE
:101B9000032329069BB258BFE31C138001E4274BA3
:101BA0001B78002B00F087801E4B9BF808101A68EA
:101BB0009BF809300A3243EA01231A490A601C4A99
:101BC0001380164B154A1B8801331380FFF7E9BBBE
:101BD0009BF80630180679D5154B1C88114B1D68EB
:101BE000631C98B2820B05F10B03A10B0C4D55F849
:101BF000211055F822500B4A1360C4F30D03C0F3B3
:101C00000D02C95C0A4B1880AB5C41EA032303490F
:101C10000B80074BA21C1A80FFF7C3BB3CBD012001
:101C20000CB70120C4BD0120E0BC0120C2BD0120D1
:101C30007CBC01209100002071BC0120C1BD0120AD
:101C4000A84BA9491B880888A84A013B99B2431CA4
:101C5000A44812680180A5480B32B1F5804F02609C
:101C600098B20DD3B1F5B64F02D2A14A0123137039
:101C70008B0BA04AC1F30D0152F82320030A5354E1
:101C8000984B1B88013B9AB2964BB2F5804F1A8055
:101C90000CD3B2F5B64F02D2954901230B70930BCA
:101CA0009449C2F30D0251F8233098548E4A3023E0
:101CB0001380FFF776BB904B1B789BB18B4B9BF847
:101CC0000A101A689BF80B300A3274E7874B874971
:101CD0001A68854B05321B880A60834A01331380DA
:101CE000FFF75FBB814B9BF804101A689BF8053027
:101CF000063260E77C4B7F4D1C887C4B9BF80700CD
:101D00001968631C9BB29A0B073155F82220764D57
:101D10002B80764DC3F30D032960D35C774A1843BB
:101D20008BF807009379002860D003F0BF03050605
:101D300093715ED563F07F039371714B9BF806102E
:101D40001A5C6E4801F0EC038BF80630002A49D08B
:101D500043F004038371644AA31C1380FFF721BB83
:101D6000604B9BF807101B889BF806205F4842EAEF
:101D70000122013B5B49006814B29AB20A805B49B8
:101D800000F10B03B2F5804FA0B20B600DD3B2F59A
:101D9000B64F02D2564901230B70930BC2F30D01CB
:101DA000544A52F82320030A53544E4B1B88013BDC
:101DB0009AB24C4BB2F5804F1A800CD3B2F5B64FA5
:101DC00002D24B4901230B70930B4A49C2F30D0217
:101DD00051F823309C54444B434A1B8801331380F1
:101DE000FFF7DFBA21F017038371B4E743F0400334
:101DF00093719BF8063003F07F038BF806309CE765
:101E0000394B3C481C889BF80650631C9BB29A0BCC
:101E1000A11C50F82200344A1380C3F30D0289B28A
:101E20008B0B805C334A52F823202F4B1980C1F36F
:101E30000D032F06D35C2C4900EB03239EB238D44C
:101E4000284B2A4A1B881068013BE11C9AB200F11A
:101E5000110388B223490A802449B2F5804F0B60F0
:101E60000DD3B2F5B64F02D2214901230B70930B6B
:101E7000C2F30D011F4A52F82320030A5354194B91
:101E80001B88013B9AB2174BB2F5804F1A800CD3D6
:101E9000B2F5B64F02D2164901230B70930B1549C8
:101EA000C2F30D0251F8233098540F4B1E80FFF7F8
:101EB00078BA0E4BE21C1B680A800C4A0A33136086
:101EC000FFF76FBA094B084A1B68084912880433A8
:101ED0000B60054901320A800A4A00231370FFF79C
:101EE00060BA00BF7CBC01203CBD0120C4BD012004
:101EF000910000200CB70120C2BD0120E0BC0120F0
:101F00009063010871BC01207E4B9BF806501C8831
:101F10007D4B1E68631C9AB2A31C98B2910B7B4B3D
:101F200053F82110774B1A8006F10A03764EC2F35C
:101F30000D023360895C754A830B52F82320714B84
:101F40001880C0F30D03D35C6E4A01EB032329060E
:101F50009BB248BFE31C1380FFF723BA6C4B1D886C
:101F6000694B1C68674B1F886B1C98B2A90B04F166
:101F70000A03664C820B54F82140644951F82260F0
:101F8000614A1360C5F30D03C0F30D01E25C604BC1
:101F90001880735C42EA03231BB2C3F307208BF85B
:101FA00006305B4B8BF80700A91C1980554B7A1C37
:101FB0001A80FFF7F6B99BF8063018065CD4544B2C
:101FC0001C88514B1D68631C98B2820B05F10B03F2
:101FD000A10B4E4D55F8211055F822504A4A136076
:101FE000C4F30D03C0F30D02C95C494B1880AB5C10
:101FF00041EA032343490B80454BA21C1A80FFF79B
:10200000D0B9434B3F491B8808883F4A013B99B2EE
:10201000431C3F48126801803B480B32B1F5804FAA
:10202000026098B20DD3B1F5B64F02D2394A0123FE
:1020300013708B0B354AC1F30D0152F82320030AAC
:102040005354334B1B88013B9AB2314BB2F5804F4E
:102050001A800CD3B2F5B64F02D22E4901230B7071
:10206000930B2A49C2F30D0251F823309854254AA4
:1020700028231380FFF795B9234B23491A68214B76
:1020800005321B880A601F4A01331380FFF789B9A4
:102090001C4B1E4D1C881C4B9BF807001968631CC9
:1020A0009BB29A0B073155F82220164D2B80164D06
:1020B000C3F30D032960D35C174A58408BF807001F
:1020C0009379002802F0B18003F0BF0305069371F5
:1020D00042F1AE8063F07F039371104B9BF80610C2
:1020E0001A5C0D4801F0EC038BF80630002A00F072
:1020F000A78043F004038371024AA31C1380FFF7F7
:1021000050B900BF3CBD0120C4BD01200CB7012067
:102110007CBC012091000020E0BC012090630108FC
:10212000854B86481F887B1C9BB29A0BC3F30D011D
:1021300050F8222080480380525CA2F140037B2BA0
:1021400002F25A80DFE813F02E10FD0F9D0F380FBA
:10215000ED0ECB0EBE0E910E660E430EE30DA90DD5
:10216000ED0E870D7A0D700D2A0D090DA60C530C7E
:10217000ED0ECB0E240B070BDB0AC70A640A2A0AF2
:10218000ED0ECB0E0F0A050AFC0BE80BA20B3F0B62
:10219000ED0ECB0E79062C06FE05EA054E080E085C
:1021A000ED0ECB0EF607A1075C073807D9068A06A5
:1021B000ED0ECB0E9D09581073095109F508C5099C
:1021C000ED0ECB0EB8095810581058105810581072
:1021D00058105810581058105810581058105810BF
:1021E00058105810581058105810581058105810AF
:1021F000581058105810581058105810581058109F
:10220000581058105810581082052305D10497040F
:10221000581058105810581069030A030104C703D6
:102220005810581058105810AA025D02C801A40195
:10223000581058105810581045010201A400800091
:1022400021F01703837157E79BF804209BF80530B2
:1022500043EA0224A30B39499BF8000051F82330CC
:102260009BF80110364DC4F30D029A5C10F026FC69
:102270009BF80030013B621EDBB294B28BF8003059
:10228000002B33D02F4B2F4A1B6815331360E1E727
:102290009BF804209BF80530012743EA0225B5F599
:1022A000804F4FEA9533C5F30D060FD3B5F5B64F02
:1022B00038BF254A9BF8011038BF17701F4A9BF89A
:1022C000000052F823400DF0F9FFA0559BF80030B4
:1022D0001B4C013B6A1EDBB295B28BF80030C3B1D8
:1022E000184B184A1B6815331360D8E7154BAA79A9
:1022F0001968114B6C711B88200A42F04202287148
:10230000AA7110480C4A1031013301601380FFF7A5
:1023100048B80C4BA2791968074B65711B88280ACD
:1023200042F042022071A2710648034A1031013383
:1023300001601380FFF735B83CBD01200CB70120C8
:10234000E0BC0120C4BD0120910000209BF80630B4
:102350009BF807209BF800509BF801409BF8040075
:102360009BF8051023F040038BF8063044EA05255E
:1023700041EA002197B202F00F068B0BC248C1F36D
:102380000D0250F823309A5C02F00F03F41ABB1AC6
:10239000681E9AB29BF8063085B2E0064CBF43F047
:1023A000100323F0100301398BF80630140689B2AC
:1023B000B6489BF8063040F1E38063F07F038BF86A
:1023C0000630B34B002D43D01B68B14A1533136060
:1023D000D3E79BF801409BF803309BF800509BF833
:1023E00002209BF804009BF8051044EA052C43EA00
:1023F0000222CCEB020341EA002E9EB274464FF05B
:102400000108A30BA049C4F30D0051F82310B2F545
:10241000804F04F1FF33085C02F1FF374FEA923539
:102420009CB2C2F30D0109D3B2F5B64F3CBF994B34
:1024300083F80080944B53F825305854BAB2964232
:1024400000F0BB80924B92491B6815330B60D8E7B4
:102450001A688BF805100B0A8BF804308C4B8BF83C
:10246000005010328BF801501A609BF8063023F0B0
:1024700004038BF806309BF80620874B42F00202DB
:102480001B888BF80620844A01331380FEF789BF2E
:102490009BF804209BF8053043EA0224A30B7A49F9
:1024A0009BF8000051F823309BF80110774DC4F3DE
:1024B0000D029A5C10F002FB9BF80030013B621C9D
:1024C000DBB294B28BF80030002B33D0704B704AE3
:1024D0001B6815331360E1E79BF804209BF8053077
:1024E000012743EA0225B5F5804F4FEA9533C5F33E
:1024F0000D060FD3B5F5B64F38BF664A9BF80110ED
:1025000038BF1770604A9BF8000052F823400DF066
:10251000D5FEA0559BF800305C4C013B6A1CDBB239
:1025200095B28BF80030C3B1594B594A1B6815332B
:102530001360D8E7564BAA791968574B6C711B8802
:10254000200A42F042022871AA715148524A1031C1
:10255000013301601380FEF724BF4D4BA279196847
:102560004D4B65711B88280A42F042022071A2710E
:102570004748494A1031013301601380FEF711BF0B
:1025800003F07F048BF80640002A7FF41AAF404B1B
:1025900041711A6845700B0A03713D4B02F110013D
:1025A000196044F040022B0A82710370002D3FF441
:1025B0005CAF44F0440383715DE7354A9BF8061035
:1025C0001468354A8BF80360CCEB0E0312889BB27B
:1025D000300A21F016018BF805308BF802001B0A37
:1025E0002B488BF806102C498BF80430103400234C
:1025F000013204600A808BF800308BF80130FEF75E
:10260000D0BE9BF806309BF807209BF800509BF843
:1026100001409BF804009BF8051023F040038BF861
:10262000063044EA052541EA002197B202F00F0680
:102630008B0B1548C1F30D0250F823309A5C02F061
:102640000F03F41ABB1A681E9AB29BF8063085B2C3
:10265000E0064CBF43F0100323F0100301318BF868
:102660000630140689B209489BF8063040F1C28151
:1026700063F07F038BF80630054B002D4ED01B68AE
:10268000034A15331360D3E70CB70120E0BC0120E7
:10269000C4BD0120910000203CBD01209BF80140F9
:1026A0009BF803309BF800509BF802209BF8040035
:1026B0009BF8051044EA052E43EA02220EEB0203C2
:1026C00041EA00271FFA83F83C464FF0010CA30BA8
:1026D000C349C4F30D0051F82310B2F5804F04F143
:1026E0000103085C02F101064FEA92359CB2C2F385
:1026F0000D0109D3B2F5B64F3CBFBA4B83F800C009
:10270000B74B53F825305854B2B2424500F08F8190
:10271000B54BB5491B6815330B60D8E71A688BF8C1
:1027200005100B0A8BF80430AF4B8BF800501032B9
:102730008BF801501A609BF8063023F004038BF8E5
:1027400006309BF80620A94B42F002021B888BF84A
:102750000620A64A01331380FEF723BE9BF804200F
:102760009BF80530A0499BF8074008689BF800607B
:1027700043EA0225AB0B9A4A52F8232000F11003DA
:102780009948C5F30D010360535C9BF80100E21A00
:1027900003F00F0104F00F0394B2954A5B1A13F093
:1027A000100F937914BF43F0100323F010039371BB
:1027B0009BF8063040EA062126064CBF63F07F03F3
:1027C00003F07F038BF806306B1E9BB24A1E91B25A
:1027D0001A0A8BF80420864A8BF805300B0A8BF80E
:1027E00000308BF801109379002940F0C88123F064
:1027F000040393719BF80630002C67D143F040032B
:102800008BF806309BF806307849BA1C43F0020377
:102810000A808BF80630FEF7C4BD9BF804209BF8B5
:10282000053071499BF802600F689BF8031043EA7A
:102830000225AB0B6A4A52F823009BF8002007F1EF
:102840001003694FC5F30D043B6041EA06219BF874
:102850000130005DB1F5804F43EA02240CD3B1F59D
:10286000B64F02D25F4A012313708B0B5C4EC1F34B
:102870000D0256F8233098546A1E631E013994B233
:1028800089B2220A98B28BF804200B0A584A8BF8B6
:102890000230030A8BF800308BF801008BF803102C
:1028A0008BF805409379002840F06D8123F00403F4
:1028B00093719BF806204D4B22F012021B888BF877
:1028C00006204A4A01331380FEF76BBD23F0400314
:1028D0008BF8063096E79BF804209BF805304249B8
:1028E00043EA02250C683E4A9BF80110AB0BC5F386
:1028F0000D0052F8232004F110033B4C2360125CBE
:102900009BF800003A4C10F0D9F89BF80030013BDE
:10291000DBB28BF80030002B58D1A37943F0400391
:10292000A3716B1E314A9BF8061012889BB28BF87C
:1029300005301B0A8BF804302C4B41F002010132A8
:102940008BF806101A80FEF72CBD274B9BF805204C
:102950009BF804101B6842EA0125234A1033B5F5A1
:10296000804F136012D3B5F5B64F02D21D4A012332
:102970001370AB0B1A4A9BF801109BF8000052F839
:1029800023400DF09BFCC5F30D03E0549BF80010B1
:1029900017486B1E9AB24B1ED9B2130A8BF804303B
:1029A0008BF805208BF800108379A1B943F0400320
:1029B00083719BF806200D4B42F002021B888BF8B6
:1029C00006200A4A01331380FEF7EBBCA37923F0FB
:1029D0004003A371A5E723F040038371E9E700BF3B
:1029E0000CB7012091000020C4BD01203CBD012096
:1029F000E0BC012003F07F048BF80640002A7FF43E
:102A00003BAEC14B41711A6845700B0A0371BE4B56
:102A100002F11001196044F040022B0A8271037028
:102A2000002D3FF488AE44F04403837189E6B64933
:102A30008BF803200C68B5499BF806000988120A38
:102A40000EEB07038BF80220AF4A9BB210341460E0
:102A50008BF80530AD4A1B0A20F0160001318BF8C7
:102A6000043000238BF8060011808BF800308BF8BF
:102A70000130FEF796BC9BF804209BF80530A24974
:102A800043EA02250C68A24A9BF80110AB0BC5F380
:102A90000D0052F8232004F110039B4C2360125CBC
:102AA0009BF800009B4C10F009F89BF80030013BAC
:102AB000DBB28BF80030002B58D1A37943F04003F0
:102AC000A3716B1C914A9BF8061012889BB28BF87D
:102AD00005301B0A8BF804308C4B41F002010132A7
:102AE0008BF806101A80FEF75CBC874B9BF805201C
:102AF0009BF804101B6842EA0125834A1033B5F5A0
:102B0000804F136012D3B5F5B64F02D2824A01232B
:102B10001370AB0B7E4A9BF801109BF8000052F833
:102B200023400DF0CBFBC5F30D03E0549BF80010E0
:102B300078486B1C9AB24B1ED9B2130A8BF804303A
:102B40008BF805208BF800108379A1B943F040037E
:102B500083719BF806206D4B42F002021B888BF8B4
:102B600006206A4A01331380FEF71BBCA37923F0C9
:102B70004003A371A5E723F040038371E9E743F025
:102B80000403937136E643F00403937191E69BF8D6
:102B900004209BF805305C499BF8074008689BF8C7
:102BA000006043EA0225AB0B594A52F8232000F19A
:102BB00010035548C5F30D010360535C9BF80100F9
:102BC000E21A03F00F0104F00F0394B2514A5B1AAA
:102BD00013F0100F937914BF43F0100323F0100388
:102BE00093719BF8063022064CBF63F07F0303F01D
:102BF0007F0340EA06218BF806306B1C9BB24A1E0D
:102C000091B21A0A8BF80420424A8BF805300B0A5D
:102C10008BF800308BF801109379002940F08F84F5
:102C200023F0040393719BF80630002C67D143F026
:102C300040038BF806309BF806303449BA1C43F049
:102C400002030A808BF80630FEF7ABBB9BF804202A
:102C50009BF805302C499BF802600F689BF8031025
:102C600043EA0225AB0B2A4A52F823009BF80020C6
:102C700007F11003244FC5F30D043B6041EA062120
:102C80009BF80130005DB1F5804F43EA02240CD37C
:102C9000B1F5B64F02D2204A012313708B0B1C4EA4
:102CA000C1F30D0256F8233098546A1C631E01319B
:102CB00094B289B2220A98B28BF804200B0A154A02
:102CC0008BF80230030A8BF800308BF801008BF888
:102CD00003108BF805409379002840F0358423F0E9
:102CE000040393719BF80620084B22F012021B8804
:102CF0008BF80620054A01331380FEF752BB23F000
:102D000040038BF8063096E7C4BD01203CBD01208E
:102D10000CB70120E0BC012091000020B04BB04C6A
:102D20001B689BF805209BF801109BF800000C33F2
:102D300023600FF0C3FEAB4BAA4A1B8801331380FC
:102D4000FEF72FBBA64BA64A1B689BF801109BF809
:102D500000000C3313600DF0B1FAA34A8BF80500A4
:102D60009379002800F02B8603F0BF0301069371CE
:102D700040F1288663F07F0393719C4B9BF806100B
:102D80001A5C994801F0FD038BF80630002A61D0E7
:102D900043F004038371934ABB1C1380FEF701BB0D
:102DA0009BF804209BF805308D489BF807100768B6
:102DB00043EA0220830B8E4AC0F30D0552F82340EC
:102DC000665D01F00F01320942EA0112844907F100
:102DD0001203B0F5804F0B6006D3B0F5B64F02D2A8
:102DE000844901230B7062559BF807307E4923F01C
:102DF0000F0306F00F021A438BF807208B79002A85
:102E000040F0F08543F040038B71784B9B5C002BC6
:102E100000F0E0859BF8063043F004038BF80630A1
:102E20009BF806206F4B22F012021B888BF80620BD
:102E30006C4A01331380FEF7B4BA694B69491A68CA
:102E4000BB1C0B80664908320A606B4A0023137072
:102E5000FEF7A7BA21F0060383719CE7BB1C9AB268
:102E6000FB1C99B26248930B8C0B50F823005D4B0E
:102E70001A80C2F30D035E4A52F82440C25C594BDB
:102E80001980C1F30D035649E35C086802EB032384
:102E900099B2534A00F11403B1F5804F136027D360
:102EA000B1F5B64F02D2534A0123137050488B0B31
:102EB000C1F30D0250F8233050480088985445F66D
:102EC000FE23994202DC4B4A012313704A1C4B49F2
:102ED000931308884649C2F30D0251F82310030AE0
:102EE0008B54404B3F4A1B8801331380FEF759BA7D
:102EF00043F6FF739942F4D1E5E740499BF804207B
:102F00009BF805300E8836499BF806000968069143
:102F100043EA0225C5F30B02C6F30B03D31A00F0F4
:102F200001015C1AAA1B069B511A2D4A0F3313602C
:102F3000E3042D4A4CBF40F0100320F010039371BE
:102F400086EA05031E0440F18B8085EA01031D0417
:102F500040F186809BF8063043F004038BF806307E
:102F6000214A8BF805100B0A8BF804309379CC03B7
:102F70004CBF43F0010323F0010393718BB2002B8C
:102F800067D09BF8063023F040038BF806309BF89F
:102F9000063008044CBF63F07F0303F07F038BF817
:102FA00006309BF806300F49BA1C43F002030A8032
:102FB0008BF80630FEF7F5B9094B094C1B689BF8F6
:102FC00001109BF800000C33002223600FF076FD07
:102FD000044B044A1B8801331380FEF7E2B900BF9B
:102FE000C4BD01203CBD0120E0BC0120906301086C
:102FF0000CB701209100002070BC01207CBC012096
:10300000B54BB54A1B689BF801109BF80000B34C08
:103010000C3313600DF052F9A379024658B303F054
:10302000BF030106A37129D563F07F03A371AC4BE5
:103030009BF806109A5CA94801F0FD038BF8063056
:10304000AAB143F004038371A64ABB1C1380FEF7A8
:10305000A8B99BF8063043F040038BF8063096E79A
:103060009BF8063023F004038BF8063078E721F054
:1030700006038371E8E743F04003A3719BF8063031
:1030800003F07F038BF80630D1E79BF804209BF810
:10309000053091499BF807000F6843EA02218B0B2A
:1030A000914AC1F30D0552F82340665D00F00F030D
:1030B000894843EA0612B1F5804F07F11203D2B2F4
:1030C000036006D3B1F5B64F02D2884901230B70D5
:1030D00062559BF80730814A23F00F0343EA161329
:1030E00058B2C1B28BF807109379002936D143F05A
:1030F000400393719BF806300028B4BF63F07F0350
:1031000003F07F038BF80630754B5B5CFBB19BF8DB
:10311000063043F004038BF806309BF80620714B11
:1031200022F012021B888BF806206E4A01331380AE
:10313000FEF737B9684B6B491A68BB1C0B806649B0
:1031400008320A606A4A00231370FEF72AB99BF816
:10315000063023F004038BF80630DEE723F040034B
:103160009371C7E7BB1C9AB2FB1C99B25E485E4DD7
:10317000930B8C0B50F823005A4B1A80C2F30D03AB
:10318000594AC05C574B52F824401980C1F30D03D3
:10319000584AE35C127800EB032398B2002A74D0FB
:1031A0004D4A411C1768820B8B13C1F30D0455F86F
:1031B0002210494A55F8236007F114031360C0F345
:1031C0000D03325DCB5C03EB02239BB21A0A8BF832
:1031D00009308BF80820434B424A1B880133138087
:1031E000FEF7DFB83C4B9BF804001A689BF80530EB
:1031F0009BF80610384D394C43EA0020060501F0D3
:10320000010302F10F022A6003EB40054CBF41F0BD
:10321000100321F01003A37180EA050313F4004F9B
:103220009BF806302D4A8BF8055014BF43F0040379
:1032300023F004038BF806302B0A8BF804309379C3
:10324000EC034CBF43F0010323F001039371ABB2D5
:10325000002B39D09BF8063023F040038BF8063062
:103260009BF806301F4928044CBF63F07F0303F02E
:103270007F038BF806309BF80630BA1C23F002035C
:103280000A808BF80630FEF78CB81B4B1B78411C6C
:10329000A3B3114A1768820B8B13C1F30D0455F8C1
:1032A00022100D4A55F8236007F114031360C0F390
:1032B0000D03325DCB5C03EB02239BB21A0A8BF841
:1032C0000B308BF80A2086E79BF8063043F040036A
:1032D0008BF80630C4E700BFC4BD0120E0BC01206C
:1032E000906301083CBD01200CB701209100002033
:1032F00070BC0120C1BD0120C2BD0120A04A1768D9
:10330000820B8B13C1F30D0455F822109C4A55F81B
:10331000236007F110031360C0F30D03325DCB5C33
:1033200003EB02239BB21A0A8BF805308BF80420BA
:1033300051E794499BF806000E8891499BF80420B8
:103340009BF805300968069143EA022500F0010167
:10335000C6F30B030B44C5F30B029C18AA19069B7A
:103360001144874A0F331360E304874A4CBF40F08F
:10337000100320F01003937185EA0603DB0B4FD195
:1033800085EA01031C044BD59BF8063043F0040387
:103390008BF806307C4A8BF805100B0A8BF804304A
:1033A0009379C8034CBF43F0010323F001039371E9
:1033B0008BB273B39BF8063023F040038BF80630D2
:1033C0009BF8063009044CBF63F07F0303F07F03D2
:1033D0008BF806309BF806306C49BA1C23F00203C8
:1033E0000A808BF80630FDF7DCBF654B644C1B6828
:1033F0009BF807209BF801109BF800000C3323601A
:103400000FF05CFB614B614A1B8801331380FDF7B1
:10341000C8BF9BF8063043F040038BF80630CFE777
:103420009BF8063023F004038BF80630B2E7544BC8
:10343000534A1B689BF801109BF800000C33136083
:103440000CF03CFF504A8BF80700937950B303F01F
:10345000BF030106937128D563F07F0393714C4B32
:103460009BF806101A5C484801F0FD038BF8063003
:10347000A2B143F004038371444ABB1C1380FDF7DF
:1034800090BF3F4B41491A68BB1C0B803C49083236
:103490000A60404A01231370FDF783BF21F0060341
:1034A0008371E9E743F0400393719BF8063003F022
:1034B0007F038BF80630D2E7314B34491A68BB1CC6
:1034C0000B802F4908320A60324A02231370FDF73D
:1034D00068BFBB1C2A489AB204682F48930BF91C9A
:1034E00050F82300294B1A8004F11403244CC2F332
:1034F0000D02236089B2805C274A274C8B0B3E1D4E
:1035000052F82320214B1980C1F30D03D35C00EB4B
:10351000032399B2481C8B0B821354F8225054F8A1
:103520002340C0F30D02C1F30D03AA5CE35C17490D
:1035300003EB0223134A0E801380FDF732BF43F0E2
:1035400004039371FFF76FBB43F004039371FFF71C
:10355000C9BB0B4B0D491B68BA1C0A80084A0933CA
:103560001360FDF71EBF064B08491A68BB1C0B8091
:10357000034908320A60074A02231370FDF711BF9E
:10358000C4BD01207CBC0120E0BC01203CBD012069
:103590009063010870BC01200CB70120BB1CB3482C
:1035A0009AB20468B248930BF91C50F82300B14B4F
:1035B0001A8004F11403AD4CC2F30D02236089B2EA
:1035C000805CAB4AAA4C8B0B3E1D52F82320A94BC2
:1035D0001980C1F30D03D35C00EB032399B2481C9F
:1035E0008B0B821354F8225054F82340C0F30D0281
:1035F000C1F30D03AA5CE35C9E4903EB02239BB27B
:103600001A0A0E808BF803308BF80220FDF7C9BE32
:10361000964D9BF804409BF805109BF802209BF800
:1036200003302D689BF80600069543EA022641EA1E
:103630000425C5F30B02C6F30B03134400F001018C
:103640005C18AA19069B1144884A0F331360E304DF
:10365000894A4CBF40F0100320F01003937185EAB3
:103660000603DB0B40F08D8085EA01031C0440F16A
:1036700088809BF8063043F004038BF806307E4ABE
:103680008BF805100B0A8BF804309379C8034CBFF4
:1036900043F0010323F0010393718BB2002B69D037
:1036A0009BF8063023F040038BF806309BF8063079
:1036B0000A044CBF63F07F0303F07F038BF80630EE
:1036C0009BF806306B49BA1C23F002030A808BF882
:1036D0000630FDF766BE654B644C1B689BF8032003
:1036E0009BF801109BF800000C3323600FF0E6F903
:1036F000604B604A1B8801331380FDF752BE5B4B61
:103700005A4A1B689BF801109BF800000C331360A9
:103710000CF0D4FD584A8BF803009379002848D068
:1037200003F0BF030106937146D563F07F039371E5
:10373000524B9BF806101A5C4F4801F0FD038BF8C2
:103740000630002A31D043F004038371494ABB1C80
:103750001380FDF726BE454B1968494B1B788BF843
:10376000073001F109034349BA1C0A803F4A13603C
:10377000FDF717BE9BF8063043F040038BF8063088
:1037800094E79BF8063023F004038BF8063076E7C5
:10379000364B38491A68BB1C0B80344908320A6022
:1037A000384A01231370FDF7FCBD21F00603837135
:1037B000CCE743F0400393719BF8063003F07F039E
:1037C0008BF80630B4E7BB1C28489AB2FB1C99B2B0
:1037D00005682748930B50F82340264B1A8005F1C3
:1037E0001403224D880B2B60214BC2F30D0253F8BA
:1037F0002000204BA45C1980C1F30D039BF804103A
:10380000C25C9BF8053004EB022243EA012390B22C
:103810001CB2B0F5804FA5B223D3B0F5B64F02D29B
:10382000194A01231370830B114AC0F30D0152F89A
:10383000232045F6FE239842545402DC124A012309
:103840001370431C9A13C3F30D01094B53F8222044
:103850002B0A5354074B074A1B8801331380FDF78B
:10386000A0BD43F6FF739842F4D1E7E7C4BD012041
:103870000CB701203CBD0120E0BC01209063010891
:10388000501E002070BC012091000020BD4B9BF811
:1038900006201B68BB4CBC4942F300000F33C50433
:1038A00023604CBF42F0100322F010038B719BF891
:1038B000063023F004038BF80630DFF8CCB2030A9D
:1038C0008BF804309BF806308BF80500C4034CBF1E
:1038D00043F0010323F001038BF8063083B2002B81
:1038E00058D09BF8063023F040038BF806309BF845
:1038F0000630A64900044CBF63F07F0303F07F034A
:103900008BF806309BF80630BA1C43F002030A809D
:103910008BF80630FDF745BD9A4B9A4C1B689BF817
:1039200004209BF801109BF800000C3323600FF07B
:10393000C5F8964B954A1B8801331380FDF731BDBE
:10394000904B904A1B689BF801109BF800000C33C9
:1039500013600CF0B3FC8C4A8BF80400937920B30D
:1039600003F0BF030606937122D563F07F039371C2
:10397000874B9BF806101A5C834801F0FD038BF817
:10398000063072B143F004038371804ABB1C13807C
:10399000FDF707BD9BF8063043F040038BF8063077
:1039A000A5E721F006038371EFE743F0400393712D
:1039B0009BF8063003F07F038BF80630D8E743F01E
:1039C000400393719BF8063003F07F038BF80630B9
:1039D000FFF7D3B99BF8063023F004038BF80630C9
:1039E000FFF71EBA23F040038B71FFF70EBABB1C22
:1039F00064489AB2FB1C99B205686648930B50F86C
:103A00002340624B1A8005F114035E4D880B2B6036
:103A1000604BC2F30D0253F820005C4BA45C19808C
:103A2000C1F30D039BF80210C25C9BF8033004EB5A
:103A3000022243EA012390B21CB2B0F5804FA5B236
:103A400023D3B0F5B64F02D2534A01231370830B30
:103A5000504AC0F30D0152F8232045F6FE23984248
:103A6000545402DC4C4A01231370431C9A13C3F3D1
:103A70000D01484B53F822202B0A5354434B434A21
:103A80001B8801331380FDF78CBC43F6FF7398420B
:103A9000F4D1E7E73B4D9BF804409BF805109BF8F9
:103AA00002209BF803302D689BF80600069543EA38
:103AB000022641EA0425C5F30B02C6F30B03D31A11
:103AC00000F001015C1AAA1B069B511A2D4A0F3304
:103AD0001360E3042C4A4CBF40F0100320F01003A5
:103AE000937186EA05031E0440F1898085EA01038B
:103AF0001D0440F184809BF8063043F004038BF8EA
:103B00000630214A8BF805100B0A8BF804309379A4
:103B1000CC034CBF43F0010323F0010393718BB23C
:103B2000002B65D09BF8063023F040038BF806305D
:103B30009BF8063008044CBF63F07F0303F07F035B
:103B40008BF806309BF806301049BA1C43F002038C
:103B50000A808BF80630FDF724BC0A4B094C1B6821
:103B60009BF802209BF801109BF800000C332360A7
:103B70000EF0A4FF054B054A1B8801331380FDF7A7
:103B800010BC00BFC4BD0120E0BC01203CBD012031
:103B9000906301080CB7012091000020BA4BBA4A8B
:103BA0001B689BF801109BF800000C3313600CF0AD
:103BB00085FBB64A8BF80200937958B303F0BF0334
:103BC0000106937129D563F07F039371B04B9BF885
:103BD00006101A5CAD4801F0FD038BF80630AAB15F
:103BE00043F004038371AB4ABB1C1380FDF7D9BBC0
:103BF0009BF8063043F040038BF8063098E79BF8BB
:103C0000063023F004038BF806307AE721F0060330
:103C10008371E8E743F0400393719BF8063003F0AB
:103C20007F038BF80630D1E7974B9A491B68BA1C83
:103C30000A80954A09331360FDF7B3BB924B95494F
:103C40001A68BB1C0B80904908320A60924A002314
:103C50001370FDF7A6BB914B1C888B4B1D68631C32
:103C600098B2820B05F10E03A10B8D4D55F8211072
:103C700055F82250844A1360C4F30D03C0F30D02BB
:103C8000C95C864B1880AB5C41EA032381490B80F9
:103C9000824BA21C1A80FDF784BBBB1C7A489AB2E7
:103CA00004687F48930BF91C50F82300794B1A8065
:103CB00004F11403744CC2F30D02236089B2805CDA
:103CC000774A774C8B0B3E1D52F82320714B19809D
:103CD000C1F30D03D35C00EB032399B2481C8B0B9B
:103CE000821354F8225054F82340C0F30D02C1F35C
:103CF0000D03AA5CE35C674903EB02239BB21A0A3B
:103D00000E808BF801308BF80020FDF74ABB5E4D2A
:103D10009BF804409BF805109BF800209BF80130AD
:103D20002D689BF80600069543EA022641EA042521
:103D3000C5F30B02C6F30B03134400F001015C183A
:103D4000AA19069B1144504A0F331360E3044F4AEB
:103D50004CBF40F0100320F01003937185EA060376
:103D6000DB0B50D185EA01031D044CD59BF80630CE
:103D700043F004038BF80630444A8BF805100B0A15
:103D80008BF804309379CC034CBF43F0010323F04C
:103D9000010393718BB27BB39BF8063023F0400391
:103DA0008BF806309BF8063008044CBF63F07F03A5
:103DB00003F07F038BF806309BF806303549BA1CB8
:103DC00023F002030A808BF80630FDF7EABA2E4B87
:103DD0009BF800001A689BF8013002F10C041946A8
:103DE0001A46294B1C600EF069FE2A4B294A1B8893
:103DF00001331380FDF7D5BA9BF8063043F040033A
:103E00008BF80630CEE79BF8063023F004038BF8DE
:103E10000630B1E71C4B1C4A1B689BF801109BF84D
:103E200000000C3313600CF049FA184A8BF80100BB
:103E3000937900283CD003F0BF03010693713AD573
:103E400063F07F039371124B9BF806101A5C0F48C6
:103E500001F0FD038BF8063032B343F004038371A5
:103E60000C4ABB1C1380FDF79CBA074B0D4A19681E
:103E70009BF80730137001F109030649BA1C0A8048
:103E8000014A1360FDF78DBAC4BD0120E0BC0120DA
:103E9000906301083CBD012070BC01207CBC012066
:103EA0000CB70120501E002021F006038371D7E7D4
:103EB00043F0400393719BF8063003F07F038BF8C7
:103EC0000630C0E7B04BB1491A68BB1C0B80AE4945
:103ED00008320A60AE4A00231370FDF762BAAD4B98
:103EE0001C88A94B1D68631C98B2820B05F10E0358
:103EF000A10BA94D55F8211055F82250A24A136084
:103F0000C4F30D03C0F30D02C95CA24B1880AB5C77
:103F100041EA03239D490B809E4BA21C1A80FDF7AA
:103F200040BA994B9BF807101B6897489B4A083387
:103F30008029036000F098804B4298B20B0700F094
:103F40009980937943F0100393710E069BF8063025
:103F500040F18580050640F1828043F004038BF830
:103F600006308E4A8BF8070093798849C4054CBF08
:103F700043F0010323F0010393719BF8063010F026
:103F8000FF0F14BF23F0400343F040038BF80630CB
:103F90009BF8063000064CBF63F07F0303F07F03FD
:103FA0008BF806309BF80630BA1C43F002030A80F7
:103FB0008BF80630FDF7F5B9BB1C73489AB2FB1CB1
:103FC00099B205687448930B50F823406F4B1A80E0
:103FD00005F114036C4D880B2B606F4BC2F30D027F
:103FE00053F82000694BA45C1980C1F30D039BF8C2
:103FF0000010C25C9BF8013004EB022243EA01236B
:1040000090B21CB2B0F5804FA5B223D3B0F5B64F35
:1040100002D2634A01231370830B5F4AC0F30D0180
:1040200052F8232045F6FE239842545402DC5C4AA1
:1040300001231370431C9A13C3F30D01564B53F81D
:1040400022202B0A5354514B504A1B8801331380B2
:10405000FDF7A7B943F6FF739842F4D1E7E723F0E1
:1040600004038BF806307CE7937943F004039371E3
:104070004FF680709BF8063023F010038BF8063063
:1040800063E7414D9BF804409BF805109BF8002026
:104090009BF801302D689BF80600069543EA02263E
:1040A00041EA0425C5F30B02C6F30B03D31A00F053
:1040B00001015C1AAA1B069B511A334A0F33136085
:1040C000E304364A4CBF40F0100320F01003937114
:1040D00086EA05031E0450D585EA01031C044CD56D
:1040E0009BF8063043F004038BF806302B4A8BF81C
:1040F00005100B0A8BF804309379C8034CBF43F0CA
:10410000010323F0010393718BB27BB39BF806305C
:1041100023F040038BF806309BF806300A044CBFAE
:1041200063F07F0303F07F038BF806309BF80630C3
:104130001649BA1C43F002030A808BF80630FDF7DB
:1041400030B9114B9BF801101A689BF8003002F14E
:104150000C0418461A460C4B1C600EF0AFFC0B4BBF
:104160000A4A1B8801331380FDF71BB99BF8063000
:1041700043F040038BF80630CEE79BF8063023F07F
:1041800004038BF80630B1E7C4BD01203CBD01201B
:1041900070BC01207CBC01200CB70120E0BC0120D8
:1041A00091000020974B974A1B689BF800009BF8F2
:1041B00001100C3313600CF081F8934A8BF8000067
:1041C000937940B303F0BF030106937126D563F0E2
:1041D0007F0393718D4B9BF806101A5C8A4801F09F
:1041E000FD038BF8063092B143F004038371884AD3
:1041F000BB1C1380FDF7D5B81146864811F054FB5F
:10420000059B1B6898680FF06DFBFDF7CAB821F09D
:1042100006038371EBE743F0400393719BF806308C
:1042200003F07F038BF80630D4E743F0400393712B
:104230009BF8063003F07F038BF80630FDF74DBF87
:10424000734B75481C889BF80650631C9BB29A0BF5
:10425000A11C50F822006E4A1380C3F30D0289B2EC
:10426000805C6D4A8B0B52F82320694B1980C1F397
:104270000D036749D35C00EB032368079EB238D572
:10428000664B604A1B881068013BE11C9AB200F142
:10429000110388B261490A805A49B2F5804F0B6018
:1042A0000DD3B2F5B64F02D25D4901230B70930BCB
:1042B000C2F30D01584A52F82320030A5354574BB6
:1042C0001B88013B9AB2554BB2F5804F1A800CD334
:1042D000B2F5B64F02D2524901230B70930B4E49EF
:1042E000C2F30D0251F823309854494B1E80FDF75C
:1042F00058B8444BE21C1B680A80424A0A331360D8
:10430000FDF74FB83F4B9BF805001968404B1A88E2
:104310009BF803308BF805300B1D3A498BF80300EE
:104320000B603B4B9BF8041001321A809BF8023063
:104330008BF804308BF80210FDF733B8344B9BF840
:1043400006501C882F4B1E68631C9AB2A31C98B29F
:10435000910B314B53F821102D4B1A8006F10A03B3
:10436000284EC2F30D023360895C2B4A830B6D0724
:1043700052F82320264B1880C0F30D03D35C244A47
:1043800001EB03239BB258BFE31C1380FDF709B870
:10439000244B1B78002B00F082801A4B9BF80810EE
:1043A0001B689BF8092017480833036042EA012381
:1043B000174A1380FCF7F5BF9BF806305E077DD5E2
:1043C000164B1C880F4B1D68631C98B2820B05F1BD
:1043D0000B03A10B104D55F8211055F82250094A36
:1043E0001360C4F30D03C0F30D02C95C0B4B1880BE
:1043F000AB5C41EA032306490B80084BA21C1A80E0
:10440000FCF7CFBFC4BD0120E0BC012090630108D0
:104410003CBD0120246301080CB701207CBC0120B5
:1044200091000020C1BD0120844B85491B8808886C
:10443000844A013B99B2431C80481268018081483C
:104440000B32B1F5804F026098B20DD3B1F5B64F83
:1044500002D27D4A012313708B0B7C4AC1F30D01FC
:1044600052F82320030A5354744B1B88013B9AB221
:10447000724BB2F5804F1A800CD3B2F5B64F02D210
:10448000714901230B70930B7049C2F30D0251F86F
:10449000233098546A4A20231380FCF782BF6C4B68
:1044A0001B78BBB1674B9BF80A101B689BF80B206D
:1044B00064480833036042EA012379E7614B6149AC
:1044C0001A685F4B05321B880A605D4A013313800E
:1044D000FCF767BF5B4B9BF804101B689BF805203B
:1044E00058480433036042EA012361E7544B574CB8
:1044F0001D88544B9BF8070019686B1C9BB29A0BE4
:10450000073154F822204E4C23804E4CC3F30D0348
:104510002160D35C4F4A18408BF80700937900283C
:1045200000F0818003F0BF03070693717ED563F02E
:104530007F0393719BF80610474B464C185C01F0C3
:10454000FC0242F010038BF80630002859D042F0EC
:104550001403A3713A4AAB1C1380FCF722BF3F4BF4
:104560001B78002B3ED0374B36481B689BF8081051
:104570009BF809200F33036042EA01202F4B1B8870
:10458000013B9AB22D4BB2F5804F1A800DD3B2F594
:10459000B64F02D22C4901230B70930BC2F30D01CD
:1045A0002A4A52F82320030A5354244B1B88013B08
:1045B0009AB2224BB2F5804F1A800CD3B2F5B64FA7
:1045C00002D2214901230B70930B2049C2F30D0243
:1045D00051F8233098541A4B194A1B880133138021
:1045E000FCF7DFBE1A4B1B788BB1164B15481B68C6
:1045F0009BF80A109BF80B200F33036042EA01205E
:10460000BCE721F0070343F01003A371A2E70D4BB1
:104610000C481B689BF804109BF805200B330360C3
:1046200042EA0120AAE743F0400393719BF8063069
:1046300003F07F038BF806307CE700BF7CBC0120D1
:104640003CBD0120C4BD0120910000200CB7012019
:10465000C2BD0120E0BC012090630108C1BD012062
:10466000A94BAA481C889BF80650631C9BB29A0B66
:10467000A11C50F82200A44A1380C3F30D0289B292
:104680008B0B805CA14A52F823209F4B1980C1F309
:104690000D039D49D35C00EB03239EB26B0738D416
:1046A0009B4B9C4A1B881068013BE11C9AB200F1AD
:1046B000110388B296490A809649B2F5804F0B6083
:1046C0000DD3B2F5B64F02D2934901230B70930B71
:1046D000C2F30D018D4A52F82320030A53548C4B28
:1046E0001B88013B9AB28A4BB2F5804F1A800CD3DB
:1046F000B2F5B64F02D2884901230B70930B834960
:10470000C2F30D0251F8233098547F4B1E80FCF702
:1047100048BE804BE21C1B680A807E4A0A33136045
:10472000FCF73FBE7D4B93F80080B8F1000F44D0FA
:10473000784B784A1B689BF809509BF808E01733C0
:104740001360734B71481A88531C9F13C3F30D0CED
:104750006E4B910B53F8273050F8210013F80C6082
:10476000C2F30D03B2F5804F0693C45C07D3B2F5D4
:10477000B64F02D2684901230B70069BC55443F61D
:10478000FE739A420BDD45F6FE239A4202DC624A32
:10479000012313705D4B53F8273003F80CE0B8F198
:1047A000000F17D08BF809408BF80860564B564A1B
:1047B0001B8801331380FCF7F4BD594B1B788BB178
:1047C000544B544A1B689BF80B509BF80AE0173374
:1047D0001360B6E7524B1B7873B18BF80B408BF824
:1047E0000A60E3E74B4B4B4A1B689BF805509BF86C
:1047F00004E013331360A4E78BF805408BF80460E2
:10480000D4E7414B9BF806501C88424B1E68631C42
:104810009AB2A31C98B2910B3C4B53F821103A4B1F
:104820001A8006F10A033B4EC2F30D023360895C25
:10483000364A830B52F82320334B1880C0F30D0304
:10484000D35C314A01EB032369079BB248BFE31CE9
:104850001380FCF7A6BD314B1B78002B00F09D8028
:104860002B4B1C882B4B1D68631C98B2A10B05F1C8
:104870000E03264D820B55F82150244951F8226031
:10488000244A1360C4F30D03C0F30D01EA5C204B0E
:104890001880735C42EA03231BB2C3F307218BF831
:1048A00009301B4B8BF80810A21C1A80164B164AB5
:1048B0001B8801331380FCF774BD9BF80630580742
:1048C00000F19680124B1C88124B1D68631C98B235
:1048D000820B05F10B03A10B0C4D55F8211055F877
:1048E00022500C4A1360C4F30D03C0F30D02C95CDF
:1048F000074B1880AB5C41EA032303490B80044B50
:10490000A21C1A80FCF74DBD3CBD01200CB7012054
:104910007CBC0120C4BD012091000020C1BD01204C
:10492000C2BD0120B34BB4491B880888B34A013B80
:1049300099B2431CAF4812680180B0480B32B1F500
:10494000804F026098B20DD3B1F5B64F02D2AC4A97
:10495000012313708B0BAB4AC1F30D0152F82320D6
:10496000030A5354A34B1B88013B9AB2A14BB2F5E7
:10497000804F1A800CD3B2F5B64F02D2A049012362
:104980000B70930B9F49C2F30D0251F823309854DA
:10499000994A18231380FCF704BD9B4B1B78002B0E
:1049A00032D0944B1C88954B1D68631C98B2A10BA8
:1049B00005F10E03934D820B55F82150914951F8A2
:1049C00022608E4A1360C4F30D03C0F30D01EA5C4C
:1049D000884B1880735C42EA03231BB2C3F30721A0
:1049E0008BF80B30834B8BF80A10A21C1A805DE702
:1049F000824B82491A68804B05321B880A607E4AC6
:104A000001331380FCF7CDBC7A4B1C887B4B1D68AF
:104A1000631C98B2A10B05F10A037A4D820B55F87D
:104A20002150784951F82260744A1360C4F30D0391
:104A3000C0F30D01EA5C6F4B1880735C42EA0323FC
:104A40001BB2C3F307218BF805306A4B8BF80410B7
:104A5000A21C1A802AE7684B6A4EB3F800E0674B45
:104A60009BF8075018689BF80640684F0EF1010349
:104A70009BB29A0BC3F30D0156F822205E4E338091
:104A8000C31D5E480360505C05F00F0200F00F0389
:104A9000D11A04F001032A1AC91AD31ACA069EB2FF
:104AA0004CBF44F0100324F01003BB7180EA0503EF
:104AB0001B063FD585EA06031F063BD59BF806304B
:104AC00043F004038BF80630504A4B4993798BF836
:104AD0000760F5054CBF43F0010323F00103937118
:104AE0009BF8063016F0FF0F14BF23F0400343F08D
:104AF00040038BF806309BF8063034064CBF63F059
:104B00007F0303F07F038BF806309BF806300EF12D
:104B1000020243F002030A808BF80630FCF741BC26
:104B2000354B35491B885A1C0A80394A01231370BA
:104B3000FCF73DBC9BF8063023F004038BF80630ED
:104B4000C2E72D4B2F481C889BF80650631C9BB274
:104B50009A0BA11C50F82200274A1380C3F30D02C0
:104B600089B2805C274A8B0B52F82320224B198094
:104B7000C1F30D032049D35C00EB0323E8079EB289
:104B800048D51C4B1D4A1B881068013BE11C9AB29A
:104B900000F1110388B217490A801849B2F5804F15
:104BA0000B600DD3B2F5B64F02D2154901230B703D
:104BB000930BC2F30D01134A52F82320030A5354F6
:104BC0000C4B1B88013B9AB20A4BB2F5804F1A80FE
:104BD0000CD3B2F5B64F02D2094901230B70930BE7
:104BE0000849C2F30D0251F823309854024B1E803D
:104BF000FCF7D7BB7CBC01203CBD0120C4BD01201B
:104C0000910000200CB70120C2BD0120E0BC0120B2
:104C1000C1BD0120A74BE21C1B680A80A54A0A33CC
:104C20001360FCF7BEBBA44BA44D1C88A14B9BF8A2
:104C300007001968631C9BB29A0B0B3155F82220B0
:104C40009D4D2B809B4DC3F30D032960D15C0BF070
:104C500035FB994A8BF80700A31C1380FCF7A1BB16
:104C6000954B9BF806501C88924B1E68631C9AB2A9
:104C7000A31C98B2910B914B53F821108E4B1A80C4
:104C800006F10A038B4EC2F30D023360895C8B4A36
:104C9000830BED0752F82320874B1880C0F30D03D8
:104CA000D35C854A01EB03239BB258BFE31C1380FE
:104CB000FCF777BB7F4B9BF8000019687E4B1A8886
:104CC0007F4B1B788BF800300B1D7A490B607A49BB
:104CD0009BF8013001320A80794A10707848517887
:104CE0009BF80220437083788BF8011082709BF848
:104CF0000310C2788BF802309BF80430C1708BF837
:104D0000032001799BF80520037143798BF8041087
:104D100042718BF80530FCF744BB9BF80630DE0788
:104D20005CD5684B1C88634B1D68631C98B2820B72
:104D300005F10B03A10B614D55F8211055F82250D8
:104D40005C4A1360C4F30D03C0F30D02C95C5D4BF4
:104D50001880AB5C41EA032357490B80594BA21CD6
:104D60001A80FCF71EBB574B53491B880888514AD1
:104D7000013B99B2431C5348126801804D480B32E5
:104D8000B1F5804F026098B20DD3B1F5B64F02D2A3
:104D90004D4A012313708B0B484AC1F30D0152F8A1
:104DA0002320030A5354474B1B88013B9AB2454BBF
:104DB000B2F5804F1A800CD3B2F5B64F02D24249F9
:104DC00001230B70930B3D49C2F30D0251F82330C0
:104DD0009854394A10231380FCF7E3BA354B354910
:104DE0001A68354B05321B880A60334A0133138039
:104DF000FCF7D7BA304B314F1E882E4B9BF807403B
:104E00001D683248731C9BB29A0BC3F30D0157F80F
:104E10002220294F3B80EB1D264D2B60515C04F076
:104E20000F0201F00F03D31A13F0100F837914BF90
:104E300043F0100323F01003837181EA0403621A24
:104E40001F0695B240F1868084EA0203180640F1FD
:104E500081809BF8063043F004038BF806308BF812
:104E600007201A4A9379E9054CBF43F0010323F068
:104E7000010393719BF806300F4915F0FF0F14BF23
:104E800023F0400343F040038BF806309BF80630D4
:104E90002F064CBF63F07F0303F07F038BF80630CF
:104EA0009BF80630B21C43F002030A808BF80630F0
:104EB000FCF777BAC4BD01203CBD01200CB701202E
:104EC00060BC01207CBC012091000020E0BC0120DE
:104ED000A34B9BF802101B889BF80320A14842EAD1
:104EE0000122013B9E49006814B29AB20A809D4992
:104EF00000F10B03B2F5804FA0B20B600DD3B2F5F9
:104F0000B64F02D2984901230B70930BC2F30D01E7
:104F1000964A52F82320030A5354914B1B88013BB5
:104F20009AB28F4BB2F5804F1A800CD3B2F5B64FC0
:104F300002D28D4901230B70930B8C49C2F30D02F1
:104F400051F823309C548A4B894A1B8801331380C3
:104F5000FCF727BA9BF8063023F004038BF80630E1
:104F60007DE7834B81481C889BF80650631C9BB2ED
:104F70009A0BA11C50F822007D4A1380C3F30D0246
:104F800089B28B0B805C794A52F82320784B1980C8
:104F9000C1F30D037649D35C00EB03239EB2EB070C
:104FA00038D46F4B6F4A1B881068013BE11C9AB2E2
:104FB00000F1110388B26A490A806A49B2F5804F4C
:104FC0000B600DD3B2F5B64F02D2674901230B70C7
:104FD000930BC2F30D01654A52F82320030A535480
:104FE0005F4B1B88013B9AB25D4BB2F5804F1A8034
:104FF0000CD3B2F5B64F02D25B4901230B70930B71
:105000005A49C2F30D0251F823309854584B1E8070
:10501000FCF7C7B9534BE21C1B680A80514A0A339C
:105020001360FCF7BEB9524B504C1B884D4A0133FC
:105030009BB2990B106854F821104D4C9BF8072037
:105040002380484CC3F30D030B302060C95C9BF8F0
:1050500000000DF033FD464B454A1B880133138099
:10506000FCF79FB9424B9BF806501C883D4B1E68CD
:10507000631C9AB2A31C98B2910B3C4B53F82110BD
:105080003B4B1A8006F10A03364EC2F30D02336021
:10509000895C364A830B52F82320354B1880C0F3C5
:1050A0000D03D35C324A01EB0323E9079BB248BFEF
:1050B000E31C1380FCF775B9294B1D88294B1C682C
:1050C0002B4B1F886B1C98B2A90B04F10A03274CC9
:1050D000820B54F82140254951F82260214A13607F
:1050E000C5F30D03C0F30D01E25C1D4B1880735C2A
:1050F00042EA03231BB2C3F307208BF80330184B9B
:105100008BF80200A91C1980194B7A1C1A80FCF735
:1051100048B99BF80630D80767D4114B1C88114B4F
:105120001D68631C98B2820B05F10B03A10B0F4D98
:1051300055F8211055F822500A4A1360C4F30D03A4
:10514000C0F30D02C95C064B1880AB5C41EA032337
:1051500007490B80024BA21C1A80FCF722B900BF42
:105160007CBC0120C4BD0120910000200CB70120AF
:105170003CBD0120B44BB5491B880888B44A013BAB
:1051800099B2431CB04812680180B1480B32B1F5A6
:10519000804F026098B20DD3B1F5B64F02D2AD4A3E
:1051A000012313708B0BAC4AC1F30D0152F823207D
:1051B000030A5354A44B1B88013B9AB2A24BB2F58D
:1051C000804F1A800CD3B2F5B64F02D2A149012309
:1051D0000B70930BA049C2F30D0251F82330985481
:1051E0009A4A08231380FCF7DCB8994B98491A684F
:1051F000964B05321B880A60944A01331380FCF7F2
:10520000D0B8924B94481F88914B9BF806401B687E
:1052100006937B1C9BB29A0BC3F30D0150F822201E
:105220008A489BF807500380069B89488B4E0733BA
:105230000360505C05F00F0304F001010B4400F023
:105240000F021A4443191944D3064CBF44F010030B
:1052500024F01003B37180EA0503DB0940F08A8073
:1052600085EA01031E0640F185809BF8063043F075
:1052700004038BF80630794A8BF807109379CD0533
:105280004CBF43F0010323F0010393719BF80630F8
:1052900011F0FF0F14BF23F0400343F040038BF8DD
:1052A00006309BF806300C064CBF63F07F0303F01A
:1052B0007F038BF806309BF806306449BA1C23F054
:1052C00002030A808BF80630FCF76BB85F4B1C8832
:1052D0005F4B1D685C4B1E88631C9AB2A31C98B27E
:1052E000910B5D4B53F82110584B1A8005F11103B7
:1052F000574DC2F30D022B608D5C574A830B52F859
:105300002310524B1880C0F30D03721ECB5C05EBCB
:105310000323E11C92B29CB24B4BB2F5804F88B292
:105320001A800DD3B2F5B64F02D24A4901230B7051
:10533000930BC2F30D01484A52F82320030A535439
:10534000414B1B88013B9AB23F4BB2F5804F1A800C
:105350000CD3B2F5B64F02D23E4901230B70930B2A
:105360003D49C2F30D0251F823309854374B1C804D
:10537000FCF717B89BF8063023F004038BF80630CF
:1053800079E7324B34481C889BF80650631C9BB26B
:105390009A0BA11C50F822002C4A1380C3F30D0273
:1053A00089B28B0B805C2C4A52F82320274B198042
:1053B000C1F30D032549D35C6A0600EB03239EB2BB
:1053C00038D5214B224A1B881068013BE11C9AB258
:1053D00000F1110388B21C490A801D49B2F5804FC3
:1053E0000B600DD3B2F5B64F02D21A4901230B70F0
:1053F000930BC2F30D01184A52F82320030A5354A9
:10540000114B1B88013B9AB20F4BB2F5804F1A80AB
:105410000CD3B2F5B64F02D20E4901230B70930B99
:105420000D49C2F30D0251F823309854074B1E80EA
:10543000FBF7B7BF064BE21C1B680A80044A0A331D
:105440001360FBF7AEBF00BF7CBC01203CBD012058
:10545000C4BD0120910000200CB70120E0BC012058
:10546000884B1D781DB9884B1B78002B59D0874B72
:1054700087481A88531C99B2931C9AB28B0B940BD1
:1054800050F82300814B1980C1F30D038049C056A9
:105490007E4B51F824101A80C2F30D03CB5C03F04D
:1054A000F80203F00701382A00F29486DFE812F0D0
:1054B0008C06920692069206920692069206920632
:1054C0008806920692069206920692069206920626
:1054D000840692069206920692069206920692061A
:1054E0000A04920692069206920692069206920686
:1054F0000704920692069206920692069206920679
:10550000BC039206920692069206920692069206B4
:10551000AA039206920692069206920692069206B6
:1055200088005A4B5A481B8801339BB29A0BC3F32D
:105530000D0150F8222055480380535C03F0F80217
:1055400003F00701382A00F2A382DFE812F05A02C2
:10555000A102A102A102A102A102A102A102440191
:10556000A102A102A102A102A102A102A102F100D5
:10557000A102A102A102A102A102A102A1020007AF
:10558000A102A102A102A102A102A102A1020B0299
:10559000A102A102A102A102A102A102A1022F0463
:1055A000A102A102A102A102A102A102A102A700DF
:1055B000A102A102A102A102A102A102A1027800FE
:1055C0000D4606212F4B1B78002B51D09BF808204D
:1055D0009BF809302F4943EA022303440C682C4A04
:1055E00099B28B0BC1F30D0052F8232004F117037D
:1055F000284C2360125C9BF80630D0074CBF43F068
:10560000010323F00103062D8BF806304FEA520008
:105610001DD00BF805009BF8063098B123F040032D
:105620008BF806309BF80620184B02F06D021B88A1
:105630008BF80620154A01331380FBF7B2BE0D46E6
:105640000020BFE743F040038BF80630EAE7B1F5EE
:10565000804FE0D3B1F5B64F02D20F4A0123137049
:105660008B0BC1F30D020A4951F823309854D2E74D
:10567000054B1C78002C00F082869BF80A209BF8D2
:105680000B30A7E7C1BD0120C2BD01203CBD0120F8
:105690000CB70120C4BD0120910000200D46002060
:1056A000A94B1B78002B00F0EB859BF808209BF89A
:1056B0000930A64943EA022303440C68A44A99B27C
:1056C0008B0BC1F30D0052F8232004F117039F4CFC
:1056D0002360125C9BF8063016064CBF43F00103B2
:1056E00023F001038BF80630530043F00100062D30
:1056F00084B200F0B2850BF805009BF806209549AE
:1057000002F0BF0324068BF8063054BF02F03F03BB
:1057100063F07F038B719BF806208F4B22F01202FF
:105720001B888BF806208C4A01331380FBF739BEA7
:105730000E460020844B1B78002B00F09E809BF8C7
:1057400008209BF80930814943EA022303440D688D
:1057500099B2880B7E4B53F8202005F117037B4D3F
:10576000C1F30D042B60125D9BF8063003F00103BA
:1057700043EA4202062E95B271D00BF806209BF840
:105780000630EE054CBF43F0010323F001038BF814
:1057900006309BF8063015F0FF0F14BF23F04003CE
:1057A00043F040038BF806309BF806302D064CBFC3
:1057B00063F07F0303F07F038BF806309BF806202D
:1057C000654B22F012021B888BF80620624A0133D7
:1057D0001380FBF7E6BD0D4600205B4B1B78002BCA
:1057E00079D09BF808209BF80930584943EA0223F6
:1057F00003440C68564A99B28B0BC1F30D0052F862
:10580000232004F11703514C2360125C9BF80630EF
:10581000D0075AD5520843F0010342F080008BF8BC
:105820000630062D5FD00BF805009BF8063060B3FC
:1058300003F0BF030706474A8BF8063029D563F00B
:105840007F0393719BF80620434B22F012021B88C2
:105850008BF80620404A01331380FBF7A2BDB1F557
:10586000804F8CD3B1F5B64F02D23C4901230B7067
:10587000374B53F820301A5581E7394B1B787BB1F1
:105880009BF80A209BF80B305DE743F040038BF850
:1058900006309BF8063003F07F038BF80630D1E723
:1058A000062931D01BF8012028499BF806300968E9
:1058B00003F0010343EA420201F108032349062EE3
:1058C00095B20B607FF459AF59E723F001035008FC
:1058D0008BF80630A5E7224B1C784CB39BF80A20C6
:1058E0009BF80B3081E7B1F5804F9ED3B1F5B64FF1
:1058F00002D21A4A012313708B0BC1F30D02144913
:1059000051F82330985490E79BF804209BF8053019
:105910000E490D6843EA0221880B0D4B53F82020F5
:1059200005F10F03094DC1F30D042B60125D1BE758
:10593000062900F00F85054B04481B681BF8012061
:1059400008332146036061E7C1BD0120C4BD0120C9
:105950000CB70120E0BC01203CBD012091000020DB
:10596000C2BD01200D460020A84B1B78002B00F083
:10597000A3849BF808209BF80930A54943EA022339
:1059800003440C68A34A99B28B0BC1F30D0052F883
:10599000232004F117039E4C2360125C9BF8063011
:1059A00016064CBF43F0010323F00103062D8BF8CC
:1059B00006304FEA420000F06C840BF805009BF8BB
:1059C000063010F0FE0F14BF23F0400343F04003F5
:1059D0008BF806309BF8063004064CBF63F07F035B
:1059E00003F07F038BF806309BF806208A4B22F0E9
:1059F00012021B888BF80620874A01331380FBF7BD
:105A0000D0BC864B1878002800F0A28500209BF8B7
:105A10000A209BF80B307E4C43EA0223034425689E
:105A20007C4A9CB2A30BC4F30D0052F8232005F16D
:105A30001703774D2B60125C150600F17D859BF8EE
:105A40000630520023F0010302F0FE008BF806300E
:105A5000062900F08A850BF801009BF80630002823
:105A600059D003F0BF0304066D4A8BF8063056D5B3
:105A700063F07F0393719BF80620674B22F01202BC
:105A80001B888BF80620644A01331380FBF789BC1E
:105A90000E46002003F0C002802AC3F3C20770D074
:105AA000C02A43D0402A7BF47CAC584B1B78002B97
:105AB00000F091809BF808209BF80930544943EA94
:105AC000022303449BB20C6851489A0BC3F30D01A7
:105AD000504B53F8222004F114030360525C42FA45
:105AE00007F313F0010F9BF806304B4A14BF23F065
:105AF000440343F044038BF806309BF806301188CA
:105B000023F0020343F010028BF80620424A4B1C9C
:105B10001380FBF746BC43F040038BF806309BF83C
:105B2000063003F07F038BF80630A4E7374B1B7871
:105B3000002B00F073849BF808209BF8093034494F
:105B400043EA022303440D6899B2880B314B53F8A2
:105B5000202005F117032E4DC1F30D042B60125DBB
:105B6000012505FA07F31343062E1AB200F0478405
:105B70000BF80620284B284A1B8801331380FBF7BB
:105B800010BC224B1B78002B00F051849BF808209E
:105B90009BF809301E4943EA022303440D6899B279
:105BA000880B1C4B53F8202005F11703184DC1F347
:105BB0000D042B60125D012505FA07F3062E22EA7B
:105BC000030212D00BF80620134B134A1B88013333
:105BD0001380FBF7E6BB114B1B78002B00F03084E1
:105BE0009BF80A209BF80B3068E7B1F5804FEBD3A8
:105BF000B1F5B64F3CBF0B4B1D70064B53F8203030
:105C00001A55E1E70D4606214AE500BFC1BD012056
:105C1000C4BD01200CB701203CBD0120C2BD012044
:105C2000E0BC0120910000200D4606219A4B1B7814
:105C3000002B00F0B1809BF808209BF809309749B1
:105C400043EA022303440C68954A99B28B0BC1F3D3
:105C50000D0052F8232004F11703904C2360125CCE
:105C60009BF80630D0074CBF43F0010323F001033B
:105C70008BF80630130646BF530843F080005008E7
:105C8000062D78D00BF805009BF80630002867D069
:105C900003F0BF030706834A8BF8063064D563F030
:105CA0007F0393719BF806207F4B22F012021B8822
:105CB0008BF806207C4A01331380FBF772BB0D463C
:105CC000062151E60D460621734B1B78002B00F090
:105CD000BA829BF808209BF80930704943EA0223F6
:105CE00003440C686E4A99B28B0BC1F30D0052F855
:105CF000232004F11703694C2360125C9BF8060013
:105D0000C40746BF530843F080045408D3074CBF70
:105D100040F0010320F00103062D8BF8063000F05F
:105D200080820BF805409BF80630002C00F06E8254
:105D300003F0BF0327065B4A8BF8063040F16A8206
:105D400063F07F0393719BF80620574B22F01202F9
:105D50001B888BF80620544A01331380FBF721BBC4
:105D600043F040038BF806309BF8063003F07F03C6
:105D70008BF8063096E7B1F5804F85D3B1F5B64F75
:105D800002D24A4A012313708B0BC1F30D0244491E
:105D900051F82330985477E7454B1C78002C00F0DD
:105DA000FA829BF80A209BF80B3048E70D4600204A
:105DB0003CE73D4B9BF806501C88384B1E68631C23
:105DC0009AB2A31C98B2910B354B53F82110364B65
:105DD0001A8006F10A03314EC2F30D023360895C6A
:105DE0002F4A830B6E0652F823202F4B1880C0F3E6
:105DF0000D03D35C2C4A01EB03239BB258BFE31C79
:105E00001380FBF7CEBA2B4B1C88244B1D68631CF8
:105E100098B2820B05F10A03A10B214D55F8211010
:105E200055F822501D4A1360C4F30D03C0F30D0250
:105E3000C95C204B1880AB5C41EA03231A490B80F4
:105E40001C4BA21C1A80FBF7ACBA9BF806305F060D
:105E50006DD5184B1C88114B1D68631C98B2820BC2
:105E600005F10B03A10B0E4D55F8211055F82250EA
:105E70000A4A1360C4F30D03C0F30D02C95C0D4B55
:105E80001880AB5C41EA032307490B80094BA21C35
:105E90001A80FBF786BA00BFC1BD0120C4BD012036
:105EA0000CB70120E0BC01203CBD01209100002086
:105EB000C2BD01207CBC0120A74BA8491B880888D3
:105EC000A74A013B99B2431CA34812680180A44829
:105ED0000B32B1F5804F026098B20DD3B1F5B64FD9
:105EE00002D2A04A012313708B0B9F4AC1F30D010C
:105EF00052F82320030A5354974B1B88013B9AB254
:105F0000954BB2F5804F1A800CD3B2F5B64F02D242
:105F1000944901230B70930B9349C2F30D0251F87E
:105F2000233098548D4A00231380FBF73ABA8C4BE8
:105F30008B491A68894B05321B880A60874A0133EE
:105F40001380FBF72EBA854B874F1E88844B9BF836
:105F500007401D688548731C9BB29A0BC3F30D0163
:105F600057F822207D4F3B80EB1D7D4D2B60515C0F
:105F700004F00F0201F00F03134413F0100F8379A4
:105F800014BF43F0100323F01003837181EA04036C
:105F90006218DB0995B276D184EA0203180672D53D
:105FA0009BF8063043F004038BF806308BF807208B
:105FB0006E4A9379E9054CBF43F0010323F00103D6
:105FC00093719BF80630654915F0FF0F14BF23F05D
:105FD000400343F040038BF806309BF806302A0656
:105FE0004CBF63F07F0303F07F038BF806309BF810
:105FF0000630B21C23F002030A808BF80630FBF750
:10600000D0B9554B9BF800101B889BF801205448D1
:1060100042EA0122013B5049006814B29AB20A8058
:106020004F4900F10B03B2F5804FA0B20B600DD3C6
:10603000B2F5B64F02D24B4901230B70930BC2F35A
:106040000D01494A52F82320030A5354424B1B883E
:10605000013B9AB2404BB2F5804F1A800CD3B2F597
:10606000B64F02D23F4901230B70930B3E49C2F356
:106070000D0251F823309C54384B384A1B880133A9
:106080001380FBF78EB99BF8063023F004038BF8DE
:1060900006308BE7314B34481C889BF80650631C54
:1060A0009BB29A0BA11C50F822002C4A1380C3F318
:1060B0000D0289B28B0B805C2B4A52F82320274BB0
:1060C0001980C1F30D036D06D35C244900EB032353
:1060D0009EB238D4204B224A1B881068013BE11C39
:1060E0009AB200F1110388B21B490A801C49B2F52B
:1060F000804F0B600DD3B2F5B64F02D21949012380
:106100000B70930BC2F30D01174A52F82320030AB8
:106110005354114B1B88013B9AB20F4BB2F5804F81
:106120001A800CD3B2F5B64F02D20E4901230B7080
:10613000930B0D49C2F30D0251F823309854074BCD
:106140001E80FBF72EB9064BE21C1B680A80044A2E
:106150000A331360FBF725B97CBC01203CBD01204C
:10616000C4BD0120910000200CB70120E0BC01203B
:10617000B94BBA4C1988BA4B1D684B1C9AB28B1C90
:1061800099B2930B880B54F82340B34B1A8005F156
:106190000A03B34D2B60B14BC2F30D0253F820003C
:1061A000AD4BA25C1980C1F30D03C35C02EB03236A
:1061B000A94A1380FBF7F5B80E460621FFF7BABAD5
:1061C0000D460621FFF709BB3DB19BF808209BF85F
:1061D000093020E40E4606215CE4A24B1B78002B1C
:1061E0007FF415AC9BF804209BF805309C4843EAEB
:1061F00002240568994AA30BC4F30D0052F823202A
:1062000005F10F03964D2B60125C15E443F040033B
:106210008BF806309BF8063003F07F038BF80630CE
:1062200091E5B1F5804FFFF47EADB1F5B64F02D2E6
:106230008D4A012313708B0BC1F30D02874951F86E
:1062400023309C546FE5874B1C78002C00F0A08114
:106250009BF80A209BF80B303FE5B1F5804FFFF427
:106260004CAAB1F5B64F02D27F4A012313708B0BB3
:10627000C1F30D02794951F823309854FFF73DBA24
:10628000784B1C780CB39BF80A209BF80B30FFF777
:1062900010BAB1F5804FFFF492ABB1F5B64F02D210
:1062A000714A012313708B0BC1F30D026B4951F836
:1062B00023309854FFF783BB6A4B1C788CB19BF852
:1062C0000A209BF80B30FFF758BB062915D0644B0A
:1062D00063481B681BF80120083321460360FFF761
:1062E000F9B906291ED05E4B5D481B681BF80120DA
:1062F000083321460360FFF751BB9BF804209BF84D
:10630000053057490C6843EA02218B0B534A52F877
:10631000232004F10F03524CC1F30D002360125CE3
:10632000FFF7D8B99BF804209BF805304C490C685E
:1063300043EA02218B0B494A52F8232004F10F0350
:10634000474CC1F30D002360125CFFF727BB0D46DD
:106350000020B9E49BF804209BF8053040490C6804
:1063600043EA02218B0B3D4A52F8232004F10F032C
:106370003B4CC1F30D002360125CFFF747BA0629BE
:1063800014D0374B36481B681BF8012008332146D0
:106390000360FFF730B906291DD0314B30481B6828
:1063A0001BF8012008332146036059E49BF80420C0
:1063B0009BF805302A490C6843EA02218B0B274AD7
:1063C00052F8232004F10F03254CC1F30D00236084
:1063D000125CFFF710B99BF804209BF805302049A8
:1063E0000C6843EA02218B0B1C4A52F8232004F16B
:1063F0000F031B4CC1F30D002360125C30E4B1F5B8
:10640000804FFFF4B7ABB1F5B64F3CBF164B1D70D4
:10641000124B53F820301A55FFF7ACBB114B1B78C9
:1064200023B39BF80A209BF80B30FFF788BB0D4B7A
:106430001B7873B39BF80A209BF80B30FFF7AABBBD
:1064400006293AD0064B1BF801201B680449083383
:106450000B60FFF744BB00BF3CBD01200CB701201F
:10646000C4BD0120C2BD012091000020062939D001
:10647000AE4B1BF8012019680123BB401A4301F100
:106480000803AA49062E12B20B607FF471ABFFF726
:1064900071BB06293BD0A54B1BF8011018680123DE
:1064A00003FA07F221EA0202A04900F10803062ECE
:1064B0000B607FF487ABFFF787BB9BF804209BF84A
:1064C00005309A4943EA022308689A0BC3F30D0189
:1064D000974B53F8222000F10C0394480360525C60
:1064E000FFF7FDBA9BF804209BF805308F490D6833
:1064F00043EA0221880B8E4B53F8202005F10F034D
:106500008A4DC1F30D042B60125DFFF729BB9BF888
:1065100004209BF8053085490D6843EA0221880B69
:10652000834B53F8202005F10F03804DC1F30D0478
:106530002B60125DFFF73FBB9BF80600530043F052
:10654000010240F001038BF80630D0B2FFF780BAA9
:1065500006293FF447AE754B1BF801201B68044623
:10656000724808330360FFF767BAB4F5804FFFF451
:1065700074AAB4F5B64F02D26E4A01231370A30B6E
:106580006B49C4F30D0251F823309854FFF765BAF4
:10659000062905F09980654B64481B681BF80120AB
:1065A000083321460360FFF7A9BB634B9BF80650F5
:1065B0001C885E4B1E68631C9AB2A31C98B2910B98
:1065C0005B4B53F821105C4B1A8006F10A03574EBF
:1065D000C2F30D023360895C554A830B6E0652F894
:1065E0002320554B1880C0F30D03D35C524A01EBB6
:1065F00003239BB248BFE31C1380FAF7D2BE4E4B75
:106600004B4C19884D4B1D784B1C9AB28B1C99B280
:10661000930B880B54F82340474B1A80C2F30D03A9
:10662000434A52F82000E25C434B1980C1F30D034A
:10663000C35C02EB032398B29DB33C4B3B4A1B68FF
:106640009BF809409BF8085014331360B0F5804F55
:1066500022D3B0F5B64F02D2364A01231370830B12
:10666000334AC0F30D0152F8232045F6FE23984229
:10667000545402DC2F4A01231370431C9913C3F3B3
:106680000D022B4B53F821309D542B4B2A4A1B886B
:1066900001331380FAF785BE43F6FF739842F4D1B5
:1066A000E8E7274B1B78002B36D0204B1F4A1B688E
:1066B0009BF80B409BF80A5014331360C6E71F4B3E
:1066C0001B78002B3ED01C4B19481A88174B1D68AD
:1066D000531C9BB2911C9A0B89B250F82240164A67
:1066E000C3F30D00138005F10E03104D2B60235CE6
:1066F0000F488BF809308A0BC1F30D0350F82220A4
:106700000D480180D35C8BF808300B4B0A4A1B887C
:1067100001331380FAF745BE044B044A1B689BF80B
:1067200005409BF80450103313608FE7C4BD01206F
:106730000CB70120910000203CBD0120C1BD01200B
:10674000C2BD0120874B1B78002B68D0864B874841
:106750001A88874B1D68531C9BB2911C9A0B89B2F7
:1067600050F82240804AC3F30D00138005F10E0358
:106770007F4D2B60235C7D488BF80B308A0BC1F377
:106780000D0350F8222078480180D35C8BF80A3042
:10679000BBE7754B754918889BF806501C46431C8F
:1067A0009BB29A0B238051F82210C3F30D03821C75
:1067B000CB5692B2134469069BB253D46C4A2380E1
:1067C000126802F10C036A4A1360FAF7EABD684BDB
:1067D00067481B68674A9BF8061004330360D37947
:1067E000644ACD0746BF5B0843F0800058089BF819
:1067F00007308BF80700DC074CBF41F0010321F0A4
:10680000010393719BF80620574B22F012021B885C
:106810008BF80620544A01331380FAF7C2BD524B5D
:1068200052481A88524B1D68531C9BB2911C9A0BFC
:1068300089B250F822404C4AC3F30D00138005F191
:106840000A034B4D2B60235C48488BF805308A0BBC
:10685000C1F30D0350F8222043480180D35C8BF82C
:10686000043052E7424B22801B68414A07331360D1
:10687000FAF797BD404B1B783BB93A4B1B7823B9CD
:106880003B4B3B4A1B6807331360374B37491C8827
:10689000631C9BB29A0BC3F30D0051F82210324ACD
:1068A00013800B5C8BF803302F4BA21C1A80FAF775
:1068B00078BD314B1B781BB92A4B1B78002B43D07A
:1068C0002B4B2B4A1B68083313609BF803002949A4
:1068D00000F00F035A1E431E9CB28B79D2064CBFA8
:1068E00043F0100323F010038B71C30932D080EA08
:1068F00004031F062ED59BF8063043F004038BF8E3
:1069000006301C4A8BF80340937914F0FF0F14BF34
:1069100023F0400343F0400393719BF806302606B2
:106920004CBF63F07F0303F07F038BF806309BF8C6
:1069300006200D4B42F002021B888BF806200A4A03
:1069400001331380FAF72DBD094B094A1B68043344
:106950001360BAE79BF8063023F004038BF8063087
:10696000CFE700BFC2BD01203CBD01200CB7012014
:10697000C4BD0120E0BC0120C1BD0120A54B1B7896
:106980001BB9A54B1B78002B5CD0A44BA34A1B68FA
:10699000083313609BF80310A14A01F00F03013381
:1069A00013F0100F937914BF43F0100323F010037A
:1069B0009371CB0901F101004AD181EA00031C0661
:1069C00046D59BF8063043F004038BF806309BF85D
:1069D0000610934A8BF8030001F0FD0310F0FF0F3F
:1069E0008BF8063014BF21F0420343F0400393714B
:1069F0009BF806308B4A01064CBF63F07F0303F01F
:106A00007F038BF80630874B1B8801331380FAF71E
:106A1000C8BC9BF802209BF80330804943EA02235C
:106A2000013B9BB209687F4A8BF803301B0A8BF845
:106A300002307A4B1288063119607A4B01321A8083
:106A4000FAF7AFBC754B754A1B6804331360A1E7B6
:106A50009BF8063023F004038BF80630B7E76F4944
:106A60009BF802209BF803300C686E4943EA02232E
:106A700008889A0BC3F30D016B4B53F82220E31DDA
:106A8000664C2360535C674A8BF80730431C1380C5
:106A9000FAF787BC5F4B9BF802009BF803101B784A
:106AA0005F4A41EA0024002B70D05C48117A537A87
:106AB000056843EA0123C3F30B0005F10F011D191B
:106AC000C4F30B03034413F4805F937953488BF8AA
:106AD000095014BF43F0100323F0100393712B0AE5
:106AE00001608BF808309BF806204D4902F0FD0349
:106AF000ED038BF8063054BF22F0030343F001038B
:106B00008B71484B474A1B8801331380FAF749BC05
:106B1000444B454C1888414B1968431C9BB29A0B57
:106B20000C3154F822203F4C23803C4CC3F30D031E
:106B30002160D256831C13443A4A1380FAF731BCC1
:106B4000364B9BF806101B689BF80720334804332C
:106B5000CF0703604FEA420348BF43F00103DE055D
:106B60002F4A8BF807304CBF41F0010321F001039D
:106B700093719BF806202B4B22F012021B888BF896
:106B80000620284A01331380FAF70BBC224B1B78EE
:106B9000002B00F010812148917AD37A056843EAEE
:106BA0000123C3F30B0005F10F011D19C4F30B03FF
:106BB000034413F4805F937918488BF80B5014BF8B
:106BC00043F0100323F0100393712B0A01608BF83C
:106BD0000A3088E70F4B1B783BB90F4B1B7823B962
:106BE0000E4B0E4A1B68073313600E4B0E491C8870
:106BF000631C9BB29A0BC3F30D0051F82210094A93
:106C000013800B5C8BF80230064BA21C1A80FAF73B
:106C1000C8BB00BFC1BD0120C2BD0120C4BD012051
:106C2000E0BC01203CBD01200CB70120AD4B1B781E
:106C300023B9AD4B1B78002B00F0B780AB4BAB4AB0
:106C40001B68083313609BF80210A94A01F00F0378
:106C5000013313F0100F937914BF43F0100323F0A6
:106C600010039371CB0901F1010040F0C38081EA68
:106C700000031F0640F1BE809BF8063043F004037A
:106C80008BF806309BF80610994A8BF8020001F049
:106C9000FD0310F0FF0F8BF8063014BF21F0420304
:106CA00043F0400393719BF80630924A06064CBFAE
:106CB00063F07F0303F07F038BF806308D4B1B8856
:106CC00001331380FAF76DBB864B1B781BB9864BDB
:106CD0001B78002B43D0854B844A1B680833136014
:106CE0009BF80200824900F00F035A1E431E9CB21B
:106CF0008B79D5064CBF43F0100323F010038B7142
:106D0000C30932D080EA040319062ED59BF8063059
:106D100043F004038BF80630754A8BF802409379F0
:106D200014F0FF0F14BF23F0400343F040039371AE
:106D30009BF8063022064CBF63F07F0303F07F030D
:106D40008BF806309BF806206A4B42F002021B8843
:106D50008BF80620674A01331380FAF722BB634B96
:106D6000624A1B6804331360BAE79BF8063023F0CD
:106D700004038BF80630CFE79BF802209BF8033022
:106D80005A4943EA022301339BB20968594A8BF8F6
:106D900003301B0A8BF80230544B128806311960FD
:106DA000544B01321A80FAF7FCBA504B4F4A1B6819
:106DB0000433136047E74D4811795379056843EA76
:106DC0000123C3F30B0005F10B011D19C4F30B03E1
:106DD000034413F4805F937944488BF8055014BF43
:106DE00043F0100323F0100393712B0A01608BF81A
:106DF000043078E69BF8063023F004038BF8063065
:106E000040E73A4B9BF802109BF803201B6842EACC
:106E1000012236490733B2F5804F0B600ED3B2F52D
:106E2000B64F02D2344901230B70930BC2F30D010C
:106E3000324A52F823209BF8073053542D4B2D4AE9
:106E40001B8801331380FAF7ACBA2A4B2B481C88F5
:106E5000264B1D68631C9BB29A0BA11C50F82200A4
:106E6000244A1380C3F30D0205F10A031F4D89B2B2
:106E70002B60855C214A8B0B52F823001D4B198037
:106E8000C1F30D031B49C35C05EB0323E21C9BB25A
:106E90000A801A0A8BF803308BF80220FAF781BABD
:106EA000144B164918889BF800401D46431C9BB2A2
:106EB0009A0B2B8051F82210C3F30D02831C8A56C3
:106EC00099B2631E0A44DBB292B28BF80030002BF9
:106ED00035D0064B2A801B68044A0D331360FAF73D
:106EE00060BA00BFC1BD0120C2BD0120C4BD0120E8
:106EF000E0BC01203CBD0120910000200CB7012026
:106F0000984B9BF807201B68964897490433036009
:106F1000D3071CD58879530863F07F0240F0010342
:106F2000CA718B719BF80620904B22F012021B88CD
:106F30008BF806208D4A01331380FAF732BA894B59
:106F4000884A1B68298008331360FAF72ABA8B79BC
:106F5000520823F00103CA718B71E3E7844B1B785D
:106F60003BB9844B1B7823B97E4B7E4A1B680733A1
:106F700013607E4B80491C88631C9BB29A0BC3F341
:106F80000D0051F82210794A13800B5C8BF8013008
:106F9000764BA21C1A80FAF704BA754B1B781BB902
:106FA000744B1B78002B43D06E4B6E4A1B68083322
:106FB00013609BF801006C4900F00F035A1E431E3A
:106FC0009CB28B79D5064CBF43F0100323F010031D
:106FD0008B71C30932D080EA040319062ED59BF8C1
:106FE000063043F004038BF806305F4A8BF801400B
:106FF000937914F0FF0F14BF23F0400343F04003D4
:1070000093719BF8063022064CBF63F07F0303F0B8
:107010007F038BF806309BF80620544B42F00202A7
:107020001B888BF80620514A01331380FAF7B9B94F
:107030004C4B4C4A1B6804331360BAE79BF806308C
:1070400023F004038BF80630CFE7494B1B781BB9BC
:10705000484B1B78002B5CD0424B424A1B680833DC
:1070600013609BF80110404A01F00F03013313F045
:10707000100F937914BF43F0100323F010039371A2
:10708000CB0901F101004AD181EA00031F0646D570
:107090009BF8063043F004038BF806309BF806108B
:1070A000314A8BF8010001F0FD0310F0FF0F8BF85F
:1070B000063014BF21F0420343F0400393719BF864
:1070C00006302A4A06064CBF63F07F0303F07F03B5
:1070D0008BF80630254B1B8801331380FAF761B912
:1070E0009BF800209BF801301E4943EA0223013B34
:1070F0009BB209681D4A8BF801301B0A8BF80030DF
:10710000184B128806311960184B01321A80FAF7B1
:1071100048B9144B134A1B6804331360A1E79BF86A
:10712000063023F004038BF80630B7E70D499BF8CF
:1071300000209BF801300C680C4943EA02230888C0
:107140009A0BC3F30D010C4B53F82220E31D054CA1
:107150002360535C054A8BF80730431C1380FAF711
:1071600020B900BFC4BD0120E0BC01203CBD01200E
:10717000C1BD0120C2BD01200CB701209B4B9BF873
:1071800000009BF801101B78994A41EA0024002B6B
:107190006AD09848117A537A056843EA0123C3F309
:1071A0000B0005F10F011D19C4F30B03034413F485
:1071B000805F93798F488BF8095014BF43F0100318
:1071C00023F0100393712B0A01608BF808309BF8B1
:1071D0000620874902F0FD03E8038BF8063054BF10
:1071E00022F0030343F001038B71834B824A1B8817
:1071F00001331380FAF7D5B87E4B9BF80700196866
:107200007D4B1A887D4BDB798BF807300B1D794954
:107210000B60794B9BF8061001321A80774B774A46
:107220009B79D07191718BF80630FAF7BAB8714B2F
:107230009BF807201B686F486D49043314060360F0
:1072400034D48B79520023F00103CA718B719BF8FF
:107250000620694B22F012021B888BF80620664A32
:1072600001331380FAF79DB8654B1B783BB3614837
:10727000917AD37A056843EA0123C3F30B0005F141
:107280000F011D19C4F30B03034413F4805F9379BA
:1072900058488BF80B5014BF43F0100323F0100331
:1072A00093712B0A01608BF80A3090E788795300BC
:1072B00043F0010240F00103CA718B71C7E74D48EA
:1072C00011795379056843EA0123C3F30B0005F1F3
:1072D0000B011D19C4F30B03034413F4805F93796E
:1072E00044488BF8055014BF43F0100323F01003FB
:1072F00093712B0A01608BF8043068E73B4B1B78D5
:107300003BB93F4B1B7823B93A4B3A4A1B680733CA
:107310001360394B3B491C88631C9BB29A0BC3F327
:107320000D0051F82210344A13800B5C8BF80030AA
:10733000314BA21C1A80FAF734B82C4B1B781BB9BE
:107340002F4B1B78002B43D02A4B2A4A1B6808334B
:1073500013609BF80000264900F00F035A1E431EDD
:107360009CB28B79D7064CBF43F0100323F0100377
:107370008B71C30932D080EA04031E062ED59BF818
:10738000063043F004038BF80630194A8BF80040AE
:10739000937914F0FF0F14BF23F0400343F0400330
:1073A00093719BF8063025064CBF63F07F0303F012
:1073B0007F038BF806309BF806200F4B42F0020249
:1073C0001B888BF806200C4A01331380F9F7E9BFBC
:1073D000084B084A1B6804331360BAE79BF8063071
:1073E00023F004038BF80630CFE700BFC1BD0120B6
:1073F000E0BC0120C4BD01203CBD012060BC0120D7
:10740000C2BD01200CB70120B44B1B781BB9B44B93
:107410001B78002B5CD0B34BB24A1B680833136057
:107420009BF80010B04A01F00F03013313F0100F66
:10743000937914BF43F0100323F010039371CB0929
:1074400001F101004AD181EA0003190646D59BF8F3
:10745000063043F004038BF806309BF80610A24A6E
:107460008BF8000001F0FD0310F0FF0F8BF80630E1
:1074700014BF21F0420343F0400393719BF80630A0
:1074800002064CBF63F07F0303F07F038BF80630E6
:10749000964B964A1B8801331380F9F782BF9BF8FD
:1074A00000209BF801308F4943EA022301339BB24D
:1074B00009688E4A8BF801301B0A8BF80030894B23
:1074C000128806311960894B01321A80F9F769BFB9
:1074D000844B844A1B6804331360A1E79BF8063091
:1074E00023F004038BF80630B7E77E4B9BF80010BF
:1074F0009BF801201B6842EA01227A490733B2F562
:10750000804F0B600ED3B2F5B64F02D278490123FB
:107510000B70930BC2F30D01764A52F823209BF8AF
:1075200007305354714B714A1B8801331380F9F7AC
:1075300038BF6E4B6F481C886A4B1D68631C9BB23A
:107540009A0BA11C50F82200684A1380C3F30D0265
:1075500005F10A03634D89B22B60855C654A8B0B8C
:1075600052F82300614B1980C1F30D035F49C35CDE
:1075700005EB0323E21C9BB20A801A0A8BF8013048
:107580008BF80020F9F70DBF564B56491A68574B38
:1075900004321B880A60554A01331380F9F701BF92
:1075A000554B56481A8821460EF07EF9059B1B68FC
:1075B00098680CF097F9F9F7F4BE9BF8063023F0C1
:1075C00001038BF80630F9F79FBD9BF807000628EA
:1075D00001F0D5820D2841D0059B1D68A9688B68F4
:1075E000013B002B8B602EDB0A68531C0B60107074
:1075F000059B1B6898680CF075F9F9F785BD039A2F
:10760000C8F30D03D65C3E4B03931A46F9F7A0BFAF
:107610003C4B4B44A3F5B0431B78934279F4A6AF9F
:10762000394B1B78002B7AF407A810067AF504A8CA
:10763000364B1B78002B39F4A1AFC2F3C20402F021
:107640000705F9F79FBF8A69934201DB0A28CBD16E
:107650000A46014628460DF06BFBC9E7059B1D68ED
:10766000A9688B68013B002B8B60C1F245840868D8
:107670000D23421C0A600370059B19688A68936891
:10768000013B002B9360C1F2318410680A23411C36
:1076900011600370ACE7059B1D481B680D22DB6879
:1076A00001210DF001FEF9F733B801340A2005F08D
:1076B000D5F80A2C78F4BBAF164B05931B68164A15
:1076C0001649D8680DF090FD059B15481B681B22D4
:1076D000DB6801210DF0E8FDF9F71AB8C1BD012002
:1076E000C2BD0120C4BD0120E0BC01203CBD012081
:1076F000910000200CB701202CBD01204863010837
:1077000000400010541E0020680300205421002077
:107710005C5F010824010020E45E0108EC5E0108C2
:10772000405F0108C34FDFF83CB3DFF83CA30A23F6
:107730004FF00008B9463E460393DAF83030BE4CAD
:1077400043F00103CAF830304FF4C053032212A9AA
:107750002046129302238DF84D208DF84C308DF881
:107760004E808DF84F8005F0C5F94FF480524FF4EC
:10777000006363836420628305F070F8636A23F416
:1077800070436362636A43F420436362636A23F471
:1077900070236362636A43F420236362DAF844303F
:1077A00043F48043CAF84430DAF8343043F08003BD
:1077B000CAF834300BF0E8FCA04BCBF87C30A04B7F
:1077C000CBF88030C7F81083002202F1C40307EB26
:1077D000830302F1D401C3F80480BB1801320F2ADD
:1077E00047F8218083F88C83EFD108230122A6F883
:1077F000B23333704023B270F272B38004224FF47C
:10780000A0737270F38002228E4B32728E4A336103
:1078100003F54073B261736520322033F261B365C2
:10782000203220333262F3652032203372623366B5
:10783000A2F5AC62A3F5E4637261C6F8CC3002F540
:107840008072E033C6F89020C6F89430403240335E
:10785000C6F89820C6F89C3040324033C6F8A020C5
:10786000C6F8A430403240334FF0A041C6F8A820FB
:10787000C6F8AC3002F5246203F5D1534FF0000096
:10788000C6F8D020C6F8D43002F5005203F50053F4
:10789000F070F160C6F8D820C6F8DC308A6803F5CD
:1078A0000053C6F8E43022F001038B60CA68674BCE
:1078B000C6F8E83042F04003CB60654A654BC6F835
:1078C000EC204FF05021C6F8E010C6F80C3108F05B
:1078D0003BFC737AFA68002B0CBF4FF434134FF45F
:1078E00074139363142006F0F5F8FB78012B07D18D
:1078F000F9688B68052262F3440343F020038B6030
:10790000FA68D3686FF39E7343F00053D36032205C
:1079100006F0E0F8D7F80C3100241C603B7A012B0C
:10792000254600F0E380D9F814100B68012262F3B9
:1079300001030B603F4806F0E5F87A6913686FF3BE
:1079400082031360FB7A012B0FD18021E023D9F849
:107950000C2061F30F0463F30F05C0F26004C0F262
:10796000600551629462C2F80051CDF84080109BCE
:10797000F96843F020031093109B102262F38A13DE
:107980001093109B0B610B69334A1093109B980660
:1079900003D50B691093013AF8D108F0CBFBCDF871
:1079A00038800E9BFA682C4943F010030E930E9B0F
:1079B000136113690E930E9BDB0603D513690E93B7
:1079C0000139F8D108F0B6FB3B786BB12333234A79
:1079D00009EB83004FF0FF3152F8043F99601368C0
:1079E0009042C3F80C80F7D1D7F8CC201C4C136818
:1079F0006FF382036FF341036FF3C3036FF3451318
:107A0000DD045CBF43F480531360C82006F062F8C5
:107A1000FA68F878002393614FF0FF3353615360A5
:107A2000F968002814BF002310236FF080424A61D8
:107A30001CE000BFE4BD0120000002400000002067
:107A4000180000200008005000090050007000508D
:107A500000800050000E0050400D030070BE012059
:107A600000080080A8C301200038024043F00C53F6
:107A70008C618A6943F4001343F0080313438B615C
:107A80008B6843F001038B60DBF880301B689847FC
:107A9000BD4BBE49D96001224321032312A88DF8B2
:107AA00049208DF84B208DF848108DF84A3005F0AC
:107AB00075F8322004F0D2FE942407F08DFFB44B09
:107AC0001B78012B4FF0050039F4CBA904F0C6FE5A
:107AD000013CF2D1AE4B1B78012B39F4C2A9039BB8
:107AE000013B03937FF429AEF9F7BBB9D9F8142011
:107AF000136864F3010313601CE72046A5490DF0E9
:107B00007FFF002879F438A8A34A82F88000F9F7AB
:107B100033B8A24912A80DF073FF064600284FD0D3
:107B20009F4912A80DF06CFF70BB9E4920460DF0D6
:107B300067FF48B9984B984AD3F8C43043F0010323
:107B4000C2F8C430F9F718B8974920460DF058FF2D
:107B500048B9914B904AD3F8C43043F00203C2F8BD
:107B6000C430F9F709B8204690490DF049FF0028C4
:107B700079F402A8884B884AD3F8C43043F0040350
:107B8000C2F8C430F8F7F8BF894912A80DF038FFE1
:107B900000B3884912A80DF033FF002878F4ECAF49
:107BA00020460BF075FD844B7B4A0340002B03DA23
:107BB000013B63F00103013382F8C830F8F7DCBF02
:107BC00021463F227D480DF061FF734B83F8C06072
:107BD000F8F7D2BF20460BF05BFD794B6E4A0340AD
:107BE000002B03DA013B63F00303013382F8C93051
:107BF000F8F7C2BF21463F2272480DF047FF664B9F
:107C000083F87F60F8F7B8BF21463F2262480DF045
:107C10003DFF614B83F83F60F8F7AEBF3B2112A8F0
:107C20000DF00CFF002838F4BAAF0470F8F7B7BFB6
:107C300003F80119C34278F4BBAFF8F7C7BF624934
:107C400062480BF0BBFF0446002800F08F81604BB8
:107C50009BF807001B7821465D000DF0A9F921462D
:107C60009BF806000DF0A4F921469BF801000DF0E9
:107C70009FF921469BF800000DF09AF921469BF8E8
:107C800005000DF095F921469BF804000DF090F9E0
:107C9000214600200DF08CF9214600200DF088F9D6
:107CA0004C4B204619880AF0E3FF4B4B21461878CD
:107CB0000DF07EF9214600200DF07AF9214605F0FD
:107CC000FE000DF075F921469BF803000DF070F9E8
:107CD00021469BF802000DF06BF9404B2146587885
:107CE0000DF066F93D4B214618780DF061F93B4BDC
:107CF0002146D8780DF05CF9384B214698780DF084
:107D000057F9364B214658790DF052F9334B21463D
:107D100018790DF04DF9314B2146D8790DF048F91D
:107D20002E4B214698790DF043F921469BF80B0024
:107D30000DF03EF921469BF80A000DF039F9214675
:107D40009BF809000DF034F921469BF808000DF06E
:107D50002FF9234B214618780DF02AF9214B2146A3
:107D600018780DF025F9204B214618780DF020F9F0
:107D7000362120460AF07CFF1C4B204619880AF069
:107D800077FF002501263EE000ED00E00006FA0541
:107D900034BD01200C62010838B7012010620108CF
:107DA0001C620108286201082C6201083062010887
:107DB000346201084062010801000080B9B7012067
:107DC0000300008078B701200863010858010020F3
:107DD0007EBC01207CBC0120501E002060BC012024
:107DE00071BC01205521002070BC01203CBD012048
:107DF000022B00F0C0800DF0DBF8342E00F0A680DE
:107E0000731C9EB2013521460020ABB2002DEFD18C
:107E1000B24B1B68B3F5804F0CBF03460423B1E09F
:107E2000B72300923821F722482005F0D9FE3821E7
:107E3000084607F033FDF721482007F01BFD4FF0FF
:107E4000C0422C231380B0234FF60002A449013B0B
:107E50000A80FBD1B721084607F020FDF721482012
:107E600007F008FD4FF0C0422C231380B0234FF6DB
:107E700000029B49013B0A80FBD1B721382007F063
:107E80000DFD4821084607F0F5FC4FF0C0422C23B9
:107E9000138080234FF600029149013B0A80FBD1F9
:107EA000B721382007F0FAFCF721084607F0E2FC7A
:107EB0004FF0C0422C23138080234FF600028849E4
:107EC000013B0A80FBD11846864B196809F0C4FDB6
:107ED000079B1B680BB109F097FD0027DFF804A290
:107EE000DFF83882DFF8389216E05A2A00F027814E
:107EF00040F22281B2F5B97F00F0148140F275138F
:107F00009A4206D12FB1774B013F3846196809F0E4
:107F1000A3FD012005F014FE09F0F4FD76280246C9
:107F2000E3D1704BFF20196809F096FD079B6E495D
:107F30001A6800230B600AB109F066FD6B49012243
:107F40000A706B4A00231360F9F751B8634B1B6842
:107F5000B3F5804F1DD00025E9B2204601350AF067
:107F60004FFE082DF8D120460BF002FC614A002399
:107F70001360F9F741B8594B1B68B3F5804F06D031
:107F80005D4B1B78184621460DF012F838E70023A8
:107F9000F8E7204601210AF033FE204602210AF0CC
:107FA0002FFE052120460AF02BFEDCE7534A9BF802
:107FB00003309BF802109BF808409BF809001268F8
:107FC00043EA012A9BF80730069340EA0428002A76
:107FD00040F0C1809BF8063023F001038BF8063097
:107FE000474B484C1888431C820B99B28B0B54F8B2
:107FF0002240444A52F82350C0F30D03C1F30D024E
:10800000E45C3F4B1980AB5C3F4944EA03230B809F
:108010003B4B821C1A80F8F7E3BF3C4B9BF808608F
:108020009979DA793A4B9BF809509BF802409BF812
:1080300003001B6845EA062512F10008069540EA90
:10804000042A01F0010918BF4FF00108002BC1D02C
:10805000304B314A1B6814782E4E002B00F0B6824C
:10806000012C00F0C182022CB4D10024294B1A68E3
:108070001D465368013B002B5360C0F2EE8211682D
:108080004B1C13600A78A2F11003222B00F28B82A2
:10809000DFE813F06602FE01F00189029E01890209
:1080A0008902890289028902890289028902890278
:1080B0008902890237012C0144018902890289025F
:1080C0008902890289028902890289028902890258
:1080D0008902890213018902050100BF78BC0120D1
:1080E000000008606403002034B8012078000020FC
:1080F0001CB70120582100203EBD01202C1E00206D
:108100007CBC01200CB701203CBD012060BC0120DB
:108110004C1E00205C020020301E002038B70120D9
:10812000C0000020052F3FF6F4AEA34B01373846C0
:10813000196809F091FCECE6292A7FF4EAAE062FD3
:108140003FF6E7AEDFE817F0F903D803C6038E0366
:10815000530343033503994B984D1B68002B00F0E4
:10816000E182964B1968059B18688B68013B002BD0
:108170008B60C0F2A08208681023421C0A60037062
:108180008E4B1C68059B1A68A3680AF10205013B27
:108190004FEA2529002BA3605FFA89F7EEB2C0F2FF
:1081A000AB822168E8234A1C22600B70A368059A01
:1081B000013B002B1268A360C0F267822168032391
:1081C0004A1C22600B70A368059A013B002B1268C1
:1081D000A360C0F29B822268531C23601570A368C1
:1081E000059A013B002B1268A360C0F258822268F6
:1081F000531C236082F80090A3680699059A013BFE
:10820000FF290CBFFF260026002B1268A360C0F2D6
:1082100069822268531C23601670BAF1000F1DD0CA
:1082200008EB0A039FB266494FEA9833C8F30D0280
:1082300051F82330A1689D5C059B18684B1E002BEC
:1082400086EA0506A36020DB2268531C23601570B4
:1082500008F101031FFA83F8B845E4D1A368059A31
:10826000013B002B1068A360C0F298822268531C67
:1082700023601670514B18680BF034FB9BF80630E6
:1082800043F001038BF80630AAE6A269934229461F
:10829000224601DB0A2DD7D10CF04AFDD8E7494B25
:1082A00018681D4605F014FD044600287FF4DDAE75
:1082B00028680BF05DFA2C608CE6424B1C680DF1CF
:1082C0002A01204605F0EAFC00283FF4CEAE9DF8D6
:1082D0002A20531E12A920468DF82A30002A3FF486
:1082E000C4AE05F0DBFC0028F1D1BEE6354B1F68BB
:1082F0000DF12A01384605F0D1FC0346D0B91C46E1
:10830000B4E6304B12A9186805F098FC0346002823
:10831000F5D0BDF848102C480DF0C6FA9BF8063091
:1083200043F0010200238BF806208BF802308BF813
:10833000033055E69DF82A1024480DF0B5FA9DF853
:108340002A30DBB1002612A9384605F0A7FC034607
:108350000028D4D0059B9DF8485018688468A3680D
:10836000013B002BA36017DB2268531C23601570B0
:10837000721C9DF82A30D6B2B342E4D8059B196826
:108380008A689368013B002B93600FDB10680A2317
:10839000411C11600370C1E7A2699342294622463D
:1083A00001DB0A2DE0D10CF0C3FCE1E708460A210D
:1083B0000CF0BEFCB2E700BF6403002038250020AB
:1083C0000CB701205C020020C0620108CC620108E9
:1083D000BD4B1D680AA9284605F030FC00283FF473
:1083E00044AE0DF12A01284605F028FC00283FF490
:1083F0003CAE0DF12601284605F050FC00283FF464
:1084000034AE12A9284605F019FC00283FF42DAE21
:108410000DF12501284605F041FC00283FF425AE6A
:108420000DF1250128469DF8256005F037FCD8B1EF
:108430009DF825300DF1250128461C0205F02EFC83
:1084400000283FF412AE9DF8253044EA03431E4352
:108450000AD000240DF12701284605F01FFC631CFB
:108460009CB208B1A642F5D8059B1B6898680BF032
:1084700039FAFAE5944B1C6812A9204605F0DEFB98
:1084800000283FF4F2AD204612A905F0D7FBECE539
:108490008D4B1C6812A9204605F0D0FB034600282E
:1084A0003FF42DAF12A9204605F0C8FB0346002873
:1084B0003FF425AF12A9204605F0C0FB0346002873
:1084C0003FF41DAF12A9204605F0B8FB0346002873
:1084D0003FF415AF12A9204605F0B0FB0346002873
:1084E0003FF40DAF12A9204605F0A8FB0346002873
:1084F0003FF405AF0DF12A01204605F0CFFB0346FE
:1085000000283FF4FCAE12A9204605F097FB034675
:1085100000283FF4F4AE6168013900296160C0F2BF
:1085200032812268531C236016780139002961606A
:10853000C0F21E812268531C236015784B1E002B4D
:108540006360C0F20B812268531C23601278CDF85F
:10855000008046EA052343EA02430193204618E0DF
:10856000594B1C6812A9204605F068FB03460028F9
:108570003FF4C5AE0DF12A01204605F05FFB03462E
:1085800000283FF4BCAEBDF82A30CDF8008020466C
:1085900001934B465246069905F0CCFB0128044650
:1085A0007FF464ADBAE6059B48491B68D8680CF0B7
:1085B0001BFE059B1B68D8680BF094F9424B1868AA
:1085C0000BF0D6F8404A0023136003E540494148C8
:1085D0000BF0F4FA0546306000283FF4FBAC022CA7
:1085E0001BD0012C7FF4F6AC374B1D6812A928462E
:1085F00005F024FB00283FF4EDACBDF848400194A1
:10860000CDF800804B4652460699284605F092FB6D
:108610000446002C3FF4DEAC80E612AC214628462E
:1086200005F03CFB013400283FF4D4AC0DF15203BB
:108630009C42F3D10722284912A80CF043FED8B976
:108640009DF84F301A2B3FF410AD059A234912685C
:10865000D0681A460CF0C8FDBCE4059B11461868AA
:108660000BF0B8FF411C02467FF40DAD28680BF0FB
:108670007FF800232B60CCE7059B19481B68162266
:10868000DB6801210CF010FEA4E4A1698B42BFF667
:1086900095AD1046032122460CF04AFB93E5A169F3
:1086A0008B4202DB0A2F7FF4A2AD394610462246E8
:1086B0000CF03EFBA0E58A699342BFF65CAD0A462A
:1086C00010210CF035FB5BE55C020020E062010844
:1086D000446201085C210020786201089862010868
:1086E00080620108A1698B42BFF693AD1046314606
:1086F00022460CF01DFB90E5A1698B42BFF651ADFF
:108700001046E82122460CF013FB4FE5A1698B428D
:1087100002DB0A2E7FF45FAD3146104622460CF094
:1087200007FB5CE5AA49AB480BF048FA0446286011
:1087300000283FF44FAC034607220121A6480CF065
:10874000B3FD21461A200CF033FC214601200CF029
:108750002FFC214610200CF02BFC02E5059B214646
:1087600018680BF037FF024601307FF4F0AE7CE46E
:10877000059B214618680BF02DFF471C05463FF46A
:1087800074AC6168DAE6059B214618680BF022FF9D
:10879000431C06463FF469AC6168C6E6A269934291
:1087A00002DB0A2E7FF462AD224631460CF0C0FA9D
:1087B00060E58A4B93F8803033B3002388F880302B
:1087C000874B0620196809F047F9FFF7A2BB012083
:1087D00009F07CFAE0B1014682480DF047F9824A7F
:1087E00001231360012005F0ABF9FFF79ABB7C4B26
:1087F0001C681D469CB17D4B00241C60754B1C7091
:1088000005F010FA2C60EDE7012388F88030D7E7F7
:10881000734B0520196809F01FF9FFF77ABB204652
:1088200009F054FA0546B0B1704B1C60694B1C70DE
:1088300005F0F8F928460DF021F904286B4C06D90B
:108840002946FF2263480DF021F901232360644A81
:1088500001231360C6E7DAF80010042009F0FCF8E1
:10886000FFF757BB002009F01FFB0646002846D043
:108870000DF004F90428B5D95D4B5E4A5D4F1268CE
:1088800000241C605C4B1C705C4B051F1C601AB103
:1088900010460AF06DFF3C607419204658490DF0EF
:1088A000AFF800283ED0574920460DF0A9F868B32C
:1088B000204655490DF0A4F8002893D1534C4E485A
:1088C0000323FF22314623700DF0E0F84B4A0123C9
:1088D000136087E7012009F0E7FA044600283ED03C
:1088E0000DF0CCF804287FF67DAF21468022484861
:1088F0000DF0CCF80AF0CAF90AF06CFA72E7384BBE
:108900000320196809F0A8F8FFF703BB3F4C3A4869
:108910000223FF22314623700DF0B8F8344A0123B8
:1089200013605FE7394B344801243146FF221C7045
:108930000DF0ACF82E4B1C6054E7364B354A1B78D3
:108940000133DBB2042B137004BF002389F800301D
:10895000234B0020196809F07FF8FFF7DABA204BA3
:108960000220196809F078F8FFF7D3BA2A4A137081
:10897000F8F727BF012129480CF096FF059B1B68DB
:1089800098680AF0AFFF0125F8F7D0BE012325460D
:108990008DF82530F8F7CABE1D480BF011FCF8F72A
:1089A0009CBA12A938460AF00DF9BDF848301C49A6
:1089B000172B38460CBF022503250AF003F9BDF832
:1089C0004830023B9BB2ADF84830002B3CD155E01B
:1089D00008630108600200207862010838B70120AE
:1089E0006403002058010020582100202C1E002084
:1089F0004C1E00205C0200205C210020341E002060
:108A00000C630108146301081C630108301E002078
:108A100040BD0120C000002071BC01204862010857
:108A20003CBD01209DF82630012B40F2F880022D3C
:108A300000F0A880043B012B40F2A880621CBDF826
:108A4000483094B2A34219D90DF1260138460AF0F4
:108A50009FF8002CE6D0022CF0D1A24B1B68B3F596
:108A6000004FEBD19DF82620FD217F200AF026F84B
:108A7000621CBDF8483094B2A342E5D80023DFF869
:108A800094A28DF828308DF82A3012A938460AF0C1
:108A900099F80DF12A0138460AF07AF8BDF8483005
:108AA0004FF6FF72934204BF4FF48043ADF8483055
:108AB0008C4B1B680CBF4FF000094FF00109B3F558
:108AC000804F9DF82A3050D0033B874A52F82380CC
:108AD000BDF8483023B300252C460DE09DF82660F4
:108AE000ED2E2BD06B1C08F805609DB2621CBDF802
:108AF000483094B2A34213D90DF1260138460AF04A
:108B000047F8B9F1000FE9D19DF8263008F8053093
:108B10006B1C9DB2621CBDF8483094B2A342EBD8E6
:108B20007B68013B002B7B604CDB3A68531C3B604D
:108B30001378184639460CF0F3F8A6E70DF1260134
:108B400038460AF025F89DF82620631CED2A99B2D4
:108B500042D008F805606B1C9AB29DF8263008F8E0
:108B60000230AB1C0C469DB2C0E7052B66D0082B2B
:108B700061D0042B0CBFD0464FF00008A8E70920B5
:108B8000FEF72ABD033B012B3FF658AF554B1B6840
:108B9000B3F5804F7FF452AF544B1B78002B38D085
:108BA000534B0093534A514B534880210CF0F6FE2F
:108BB0000028F8F692A90AF069F84A4B186807F0FD
:108BC0001FFB3BE7059B394618680BF003FD034686
:108BD000013038F426AEACE70AA9384609F0D8FFD0
:108BE0000DF12601384609F0D3FF9DF82820E31C3B
:108BF0009CB2002A3FF47AAF00219DF8263008F895
:108C000005309DF8282001316B1C91429DB2F4DBA8
:108C10006CE78022394938480CF038FFCBE7314BFC
:108C20001B68B3F5804F3FF409AF304B1B78002B26
:108C3000EFD0324BB5E7DDF80C8049E7DFF8D8809C
:108C400046E72F4803F0E8FE0BADF7F7E3BCFB2245
:108C5000022112A88DF849308DF848200AF02EFA2A
:108C6000002877F4C8ACFA23012112A88DF8483007
:108C70000AF024FA002877F4BEAC4FF400300AF072
:108C80007FF90028F9D11F4C1F4823889BB243F479
:108C9000807323800AF0FCF9002837F4ACACA523DC
:108CA00023821A480AF0F4F9002837F4A4AC238B85
:108CB00023889BB243F4806312AD238027462E465F
:108CC000012413480AF0E4F9631C0E4A002837F423
:108CD00092AC398A06F8011B062B00F049811C462C
:108CE000EFE700BF78BC01208873010838B7012086
:108CF000706201086862010840BD0120D861010866
:108D00008C5E0108005400400100001002000010B9
:108D1000400000100080001000C000100B600AF03E
:108D200023F92B6B844C43F002032B632B6B43F032
:108D300002032B63204612A94FF480758DF84C80F6
:108D40008DF84E808DF84F608DF84D60129503F0D0
:108D5000D1FE4FF40073204612A912938DF84E6095
:108D60008DF84C608DF84F608DF84D6003F0C2FEB9
:108D700023699A0503D46583404603F06FFD4FF4E1
:108D800080766D4C374609250120278303F066FD68
:108D900023699B054FF0010004D4668303F05EFD58
:108DA000013DF1D1644C654D4FF48076268301205E
:108DB00003F054FD23692B6B43F002032B632B6BF1
:108DC00043F002032B632B6A43F400132B622B6ADC
:108DD00023F400132B62636A23F00F036362636A58
:108DE00043F004036362636A23F0F0036362636A1F
:108DF00043F04003636202220123204612A98DF84A
:108E00004C208DF84D208DF84E308DF84F30129655
:108E100003F070FE4FF4007312A92046129303F082
:108E200069FE296C464B474A41F4001129641A60D7
:108E300006F048FDF7F7D1BB12A803F0AFFEF7F735
:108E400028BBC9003231A3FB0113C3F3421343EA29
:108E50000201F7F7E4BA59685A685B684C024CBFE4
:108E600039493A4902F03F02B1FBF2F2334949680D
:108E7000C3F3881302FB03F2C1F30141344B013108
:108E80004900B2FBF1F21A60F7F7F8B9304B2E4AFD
:108E90001A60F7F7F3B92F4BEB6031238DF8497067
:108EA0008DF84A708DF84B808DF84830F7F7DEBAB0
:108EB000059B29481B681B22DB6801210CF0F4F993
:108EC000F7F726BC059B25481B681122DB680121AA
:108ED0000CF0EAF9F7F71CBC059B21481B68362209
:108EE000DB6801210CF0E0F9F7F712BC08460A2113
:108EF0000BF01EFFFEF77CBB8A699342BEF6B7AB50
:108F00000A46014628460BF013FFFEF7B5BB154B8A
:108F10001548059321460CF0C7FC01233B60F7F789
:108F2000F7BB059B11481B680E22DB6801210CF082
:108F3000BBF9F7F7EDBB00BF000402400038024068
:108F400068220020801A060000127A000024F40033
:108F5000700000200006FA05AC6101082C5F0108D2
:108F6000F45E010824010020C05E0108C861010808
:108F7000138823F480631B041B0C138013889BB29B
:108F800043F4007313804FF4003009F0F9FF002818
:108F9000F9D1AA480AF07CF8002837F42CABA84B8A
:108FA00012A91A8A0A551A8892B242F480621A806B
:108FB0000CA806220CF086F900287DD1A14E0123D1
:108FC00033609F4CA048A588A04BDFF8C092A04F0B
:108FD000A049A14ADFF8B882ADB245F40065A5808A
:108FE000046B9E4D44F400140463186820F00100E3
:108FF00018601868002420F001004FF0210A186062
:109000001C605C609C60DC601C61C3F814A0C9F843
:109010000C70186801400A431A605A699049079118
:1090200022F0070242F001025A615C60C3F8088036
:10903000DD601A680BAD42F010021A60012711239F
:1090400028462B706C70AC70EF7003F0A7FD854B59
:1090500085491A6822F001021A601A6822F001029A
:109060001A603D221C605C609C60DC601C61C3F87F
:1090700014A0C9F808201868764A024042F000722D
:1090800042F482321A605A6922F007023A435A6166
:109090005C60C3F80880D9601A6842F010021A6058
:1090A00028460B232B706C70AC70EF7003F076FDCC
:1090B000079B1F60F7F7A7BA062212A90EA80CF0AB
:1090C00001F928B1062212A910A80CF0FBF818B972
:1090D0005C4E0223336074E7644803F09DFC0DF19D
:1090E0004E0415F8011B624803F074FCAC42F8D141
:1090F000604803F091FCF7F77EBA5F4B1B7804F0F1
:109100000701A3B15D4B5D481B6803F108020B1F0B
:10911000012B026000D80431594B1A881BF801302A
:109120008BF80130531C564A1380F8F73AB9554B67
:109130001B78002B02F08380504B50481A680B1F9D
:10914000DBB20832012B0260E6D88B1DD9B2E3E70F
:10915000494B1B7804F00705002B5ED0474B47496D
:109160001B6803F108022B1F012B0A6000D804358D
:109170009BF806009BF807601BF80540424F06F07D
:109180000F0300F00101CA1804F00F031A44331949
:109190001944D3064CBF40F0100320F01003BB71FC
:1091A0001BF80530384A7340DB0940F0E68086EA58
:1091B00001031C0640F1E180937943F004039371AD
:1091C000314A8BF807109379C8054CBF43F001036F
:1091D00023F0010393719BF8063011F0FF0F14BFC9
:1091E00023F0400343F040038BF806309BF8063031
:1091F0000A064CBF63F07F0303F07F038BF8063051
:109200009BF806201E4B22F002021B888BF80620DA
:109210001B4A01331380F8F7C4B81A4B1B78002B94
:1092200000F0D780154B15491A682B1FDBB20832A6
:10923000012B0A609CD8AB1DDDB299E740000010FD
:109240000054004030B8012000380240A0600240C5
:1092500000003D203F801CF04004010260220020FD
:1092600020B80120106002403C1E00203C5E010836
:10927000545E010874730108C1BD0120C4BD012002
:109280003CBD0120C2BD0120E0BC012000600240C5
:1092900010540040A74B1B78002B7CD0A64BA74A4C
:1092A0001B881168A6489BF8084001339BB29A0BB3
:1092B000133150F82200A04A1380C3F30D029F4BD4
:1092C00019609BF80930825643EA042313449BB289
:1092D0009A0BC3F30D019A4B9BF8074053F82230C9
:1092E000585C984900F00F0204F00F03134413F088
:1092F000100F8B7914BF43F0100323F010038B7110
:1093000080EA04032218DB0995B23DD184EA020306
:10931000180639D59BF8063043F004038BF8063065
:109320008BF80720874A9379E9054CBF43F0010386
:1093300023F0010393719BF8063015F0FF0F14BF63
:1093400023F0400343F040038BF806309BF80630CF
:109350002A064CBF63F07F0303F07F038BF80630CF
:109360009BF80620744B22F002021B888BF8062023
:10937000714A01331380F8F714B89BF8063023F0D4
:1093800004038BF806301BE79BF8063023F0040338
:109390008BF80630C4E76C4B1B7803B3664B674A07
:1093A0001B88116866489BF80A4001339BB29A0BF0
:1093B000133150F82200604A1380C3F30D025F4B53
:1093C00019609BF80B30825643EA042313449BB286
:1093D0007EE75A4B594A1B6804331360C8E6574B63
:1093E0009BF804101B689BF8052054480733036062
:1093F00042EA01236CE7504B514C19884F4B1D68D2
:109400004B1C9AB28B1C99B2930B880B54F82340D7
:10941000494B1A8005F10D03484D2B60484BC2F3B0
:109420000D0253F82000444BA25C1980C1F30D03D8
:10943000C35C02EB03239AB2B2F5804F0ED3B2F5B0
:10944000B64F02D2414901230B70930BC2F30D01B9
:109450003B4A52F823209BF807305354364B364A88
:109460001B8801331380F7F79CBF334B34481C88AB
:10947000324B1D68631C9BB29A0BA11C50F8220052
:109480002D4A1380C3F30D0205F10A032B4D89B257
:109490002B60855C2A4A8B0B52F82300264B1980DF
:1094A000C1F30D032449C35CE21C0A80284A05EB82
:1094B00003231380F7F775BF1F4B214918889BF8CA
:1094C00006501C46431C9BB29A0B238051F8221075
:1094D000C3F30D03821CCB5692B21344EF079BB229
:1094E0001FD4164A2380126802F10C03134A13603A
:1094F000F7F757BF114B9BF8062018680E4B9BF8E7
:1095000007101B880D4C42F012028BF806200A4A05
:109510000430C943013320608BF807101380F7F73C
:1095200040BF064B22801B68044A07331360F7F7DD
:1095300038BF00BFC1BD01203CBD0120C4BD01201A
:109540000CB70120E0BC0120C2BD01209100002029
:109550007CBC01209D4B1B78002B63D09C4B9C4A0C
:109560001B680B33136009249A4B9B491D886B1CA5
:109570009BB29A0BC3F30D0051F82210954A138049
:109580000B5C0BF80430934BAA1C1A80F7F709BF49
:109590008E4B1B78002B00F0C6808D4B8C4A1B68CD
:1095A0000833136009241BF804208C4802F00F03D1
:1095B000591E531E9DB28379884ACE064CBF43F094
:1095C000100323F0100383711BF80430D90935D040
:1095D0006B40190632D5937943F0040393710BF86D
:1095E00004507E4A937915F0FF0F14BF23F0400317
:1095F00043F0400393719BF806302A064CBF63F09A
:109600007F0303F07F038BF806309BF80620714B35
:1096100042F002021B888BF806206E4A0133138049
:10962000F7F7BFBE6E4B1B78002B00F08680684BAF
:10963000674A1B680B3313600B2495E79BF80630D1
:1096400023F004038BF80630C9E7604B1B78002B2E
:1096500000F081805E4B5E4A1B680833136009206E
:109660001BF800205D4902F00F03013313F0100FC7
:109670008B7914BF43F0100323F010038B711BF898
:109680000030D90902F10104544A45D163401B0658
:1096900042D5937943F0040393710BF800409BF893
:1096A00006204E4902F0FD0314F0FF0F8BF8063040
:1096B00014BF22F0420343F040038B719BF8063045
:1096C000444A27064CBF63F07F0303F07F038BF807
:1096D0000630404B1B8801331380F7F762BE3B4BCB
:1096E0001B78002B41D09BF808209BF809303849A3
:1096F00043EA0223013B9AB209688BF80920130A56
:109700008BF80830324B0A311960324B314A1B88D2
:1097100001331380F7F745BE9BF8063023F00403AE
:109720008BF80630B9E72E4B1B786BB1284B284AD3
:109730001B68083313600B2435E7254B244A1B684C
:109740000733136005240FE7214B214A1B680433BC
:109750001360052427E7224B1B78E3B11C4B1C4AFE
:109760001B68083313600B207AE71D4B1B78CBB1C5
:109770009BF80A209BF80B30154943EA0223013B72
:109780009AB209688BF80B20130A8BF80A30104B39
:109790000A311960B9E70E4B0D4A1B680433136098
:1097A00005205DE79BF804209BF80530084943EA53
:1097B0000223013B9AB209688BF80520130A8BF843
:1097C0000430034B063119609FE700BFC1BD012083
:1097D000C4BD01203CBD01200CB70120E0BC01202C
:1097E000C2BD0120884B89481988894B874D1E7856
:1097F0004B1C9AB28B1C99B2930B8C0B50F8230024
:10980000814B1A80C2F30D03804AC05C7E4B52F834
:1098100024201980C1F30D03D35C00EB032398B21D
:10982000002E57D07B4A411C1768820B8B13C1F363
:109830000D0455F82210774A55F8236007F11403F8
:109840001360C0F30D03325DCB5C03EB02239BB2CC
:109850001A0A8BF809308BF808206B4B6A4A1B8870
:1098600001331380F7F79DBD694B1B78002B51D056
:1098700068499BF809300C689BF808206649654DDB
:1098800043EA022204F10F032B608B7917054FEA9C
:1098900042004CBF43F0100323F010038B71030A06
:1098A00004468BF809008BF808309BF806205A49CB
:1098B00002F0FD03E0038BF8063054BF22F00303EF
:1098C00043F001038B71504B4F4A1B8801331380C7
:1098D000F7F767BD514B1B78411C002B3CD04D4A1C
:1098E0001768820B8B13C1F30D0455F82210494AF7
:1098F00055F8236007F114031360C0F30D03325DC4
:10990000CB5C03EB02239BB21A0A8BF80B308BF86B
:109910000A20A2E7414B1B78002B38D03D499BF829
:109920000B300C689BF80A203B493A4D43EA02226F
:1099300004F10F032B608B7916054FEA42004CBFF0
:1099400043F0100323F010038B71030A04468BF8D5
:109950000B008BF80A30A8E72E4A1768820B8B138E
:10996000C1F30D0455F822102A4A55F8236007F177
:1099700010031360C0F30D03325DCB5C03EB0223D5
:109980009BB21A0A8BF805308BF8042065E7214951
:109990009BF805300C689BF804201F491D4D43EAD5
:1099A000022204F10B032B608B7915054FEA42006C
:1099B0004CBF43F0100323F010038B71030A0446DD
:1099C0008BF805008BF804306FE70F4B0F491888B0
:1099D0009BF806501C46431C9BB29A0B238051F8FF
:1099E0002210C3F30D03821CCB5692B213446906B6
:1099F0009BB26FD5074A2380126802F10C03054A17
:109A00001360F7F7CEBC00BF3CBD01200CB70120AE
:109A1000C1BD0120C4BD0120E0BC0120C2BD0120A8
:109A2000AE4B9BF806101B68AC48AD4A0433CF061A
:109A3000036057D4D37903F00F03092B8CBF06249E
:109A40000024CE0703D49BF80730992B06D904F1E4
:109A5000600241F00103D4B28BF806309BF8061087
:109A60009F4A01F01203022B4BD0122BD37903F043
:109A70000F0344D0092B44D941F0100393719BF894
:109A800006009BF80730964A850746BF1B1B99B214
:109A90001919CCB28BF807406CB320F040039371D6
:109AA0009BF8063008064CBF63F07F0303F07F038A
:109AB0008BF806308B4B1B5DB3B19BF8063043F03F
:109AC00004038BF80630884B874A1B8801331380C8
:109AD000F7F767BC814B22801B68804A073313600D
:109AE000F7F75FBC0624ACE79BF8063023F00403CD
:109AF0008BF80630E7E740F040039371D0E7052B81
:109B0000BAD921F010039371B9E7784B1B78002B79
:109B100063D0724B714A1B680B3313600824724B7D
:109B200073491D886B1C9BB29A0BC3F30D0051F84F
:109B300022106D4A13800B5C0BF804306A4BAA1C90
:109B40001A80F7F72EBC694B1B78002B00F0D480ED
:109B5000624B624A1B680833136008241BF8042018
:109B60005F4802F00F03591E531E9DB283795C4A71
:109B7000CE064CBF43F0100323F0100383711BF893
:109B80000430D90935D06B40190632D5937943F0AA
:109B9000040393710BF80450514A937915F0FF0FA9
:109BA00014BF23F0400343F0400393719BF8063049
:109BB0002A064CBF63F07F0303F07F038BF8063067
:109BC0009BF80620484B42F002021B888BF80620C7
:109BD000454A01331380F7F7E4BB464B1B78002B53
:109BE00000F094803D4B3D4A1B680B3313600A2400
:109BF00095E79BF8063023F004038BF80630C9E79D
:109C00003A4B1B78002B00F08F80344B334A1B6893
:109C10000833136008201BF80020314902F00F03BD
:109C2000013313F0100F8B7914BF43F0100323F0AE
:109C300010038B711BF80030D90902F10104284A86
:109C400045D163401B0642D5937943F004039371D9
:109C50000BF800409BF80620214902F0FD0314F0A8
:109C6000FF0F8BF8063014BF22F0420343F040038D
:109C70008B719BF806301C4A27064CBF63F07F03AC
:109C800003F07F038BF80630174B1B8801331380DA
:109C9000F7F787BB154B1B78002B4FD09BF808209C
:109CA0009BF809300D4943EA022301339AB209684F
:109CB0008BF80920130A8BF80830084B0A31196019
:109CC000094B094A1B8801331380F7F76ABB9BF8DD
:109CD000063023F004038BF80630B9E7C4BD012039
:109CE000E0BC0120906301083CBD0120C1BD012002
:109CF0000CB70120C2BD0120A04B1B786BB1A04B5B
:109D00009F4A1B68083313600A2427E79C4B9C4A30
:109D10001B6807331360042401E7994B984A1B68BA
:109D200004331360042419E7944B1B78E3B1944B7C
:109D3000934A1B68083313600A206CE78F4B1B782B
:109D4000CBB19BF80A209BF80B308D4943EA0223E4
:109D500001339AB209688BF80B20130A8BF80A308A
:109D6000874B0A311960ABE7854B854A1B68043382
:109D7000136004204FE79BF804209BF805308049CE
:109D800043EA022301339AB209688BF80520130ACB
:109D90008BF804307A4B0631196091E7794B7A4C95
:109DA0001888774B1D68431C9BB29A0B811C54F892
:109DB0002240744A1380C3F30D0205F10D03704D68
:109DC00089B22B60A45C704A8B0B033052F82320BD
:109DD0006C4B1980C1F30D03D35C04EB03239BB2DE
:109DE000990BC3F30D02684B53F821309B5C8BF841
:109DF0000730644B1880F7F7D4BA644B1B78002BFC
:109E000069D063499BF808209BF809305C480988B1
:109E10000568604843EA02235C18C3F30B02C1F3F0
:109E20000B0357498BF809401A4405F10F030B60E7
:109E30008379D2044CBF43F0100323F010038371E5
:109E4000230A25468BF808309BF80620514902F07A
:109E5000FD03E8038BF8063054BF22F0030343F000
:109E600001038B71474B474A1B8801331380F7F777
:109E700098BA444B444918889BF806501C46431C2A
:109E80009BB29A0B238051F82210C3F30D03821C5E
:109E9000CB5692B21344E9079BB243D5384A23808C
:109EA000126802F10C03364A1360F7F77ABA9BF88E
:109EB00006303449324A0888126823F0120343F00E
:109EC00001018BF806102E4904320A602D4A431C0A
:109ED0001380F7F766BA294B1B785BB32C499BF8C4
:109EE0000A209BF80B30264809880568294843EA70
:109EF00002235C18C3F30B02C1F30B0320498BF858
:109F00000B401A4405F10F030B608379D7044CBF53
:109F100043F0100323F010038371230A25468BF8C6
:109F20000A3091E7164B22801B68154A07331360ED
:109F3000F7F737BA16499BF804209BF8053010480C
:109F400009880568134843EA02235C18C3F30B022F
:109F5000C1F30B030A498BF805401A4405F10B03C2
:109F60000B608379D6044CBF43F0100323F0100339
:109F70008371230A25468BF8043065E7C2BD0120B2
:109F8000C4BD01203CBD01200CB70120C1BD012092
:109F90007CBC0120E0BC0120854B1B78002B3DD010
:109FA000844B854A1B88116884489BF8084001331C
:109FB0009BB29A0B133150F822007E4A1380C3F3F0
:109FC0000D027D4B19609BF80930825643EA042349
:109FD000134498B2774B794C1B8801339BB29A0B90
:109FE000C3F30D0154F82220724CB0F5804F23804A
:109FF000515C0CD3B0F5B64F02D2714A01231370F5
:10A00000830BC0F30D026D4850F823309954694B0F
:10A01000684A1B8801331380F7F7C3B9694B1B7873
:10A02000002B00F0AC80634B634A1B8811686348C7
:10A030009BF80A4001339BB29A0B133150F822006F
:10A040005C4A1380C3F30D025B4B19609BF80B3025
:10A05000825643EA0423134498B2BBE7544B1B785F
:10A06000002B6ED0534B544A1B88116853489BF801
:10A07000084001339BB29A0B173150F822004D4A29
:10A080001380C3F30D024C4B19609BF809308256C4
:10A0900043EA0423134498B2830B484AC0F30D06E5
:10A0A00052F82350A95D01F00F035A1E4B1E9CB2BB
:10A0B0009BF80630D2064CBF43F0100323F0100388
:10A0C0008BF80630CB0935D081EA04031F0631D561
:10A0D0009BF8063043F004038BF80630B0F5804F50
:10A0E00006D3B0F5B64F02D2354A01231370AC55F2
:10A0F0009BF8063014F0FF0F14BF23F0400343F029
:10A1000040038BF806309BF8063020064CBF63F006
:10A110007F0303F07F038BF806309BF80620254B66
:10A1200042F002021B888BF80620224A013313807A
:10A13000F7F737B99BF8063023F004038BF80630A5
:10A14000CCE7204B1B7833B31A4B1B4A1B88116892
:10A150001A489BF80A4001339BB29A0B173150F80A
:10A160002200144A1380C3F30D02134B19609BF8AD
:10A170000B30825643EA0423134498B28CE70E4B0B
:10A180000D481B689BF804109BF805200A330360F8
:10A1900042EA01201EE7084B07481B689BF80410A1
:10A1A0009BF805200B33036042EA012074E700BFEF
:10A1B000C1BD01203CBD0120C4BD01200CB7012060
:10A1C00091000020C2BD0120924B1B78002B6DD066
:10A1D000914B924A1B88116891489BF808400133C3
:10A1E0009BB29A0B173150F822008B4A1380C3F3AD
:10A1F0000D028A4B19609BF80930825643EA04230A
:10A20000134499B28B0B864AC1F30D0552F82340D3
:10A21000625D02F00F03013313F0100F9BF806305C
:10A2200014BF43F0100323F010038BF80630D3095A
:10A2300002F1010033D182EA00031E062FD59BF8FC
:10A24000063043F004038BF80630B1F5804F06D397
:10A25000B1F5B64F02D2734A0123137060559BF8D3
:10A260000620714902F0FD0310F0FF0F8BF8063055
:10A2700014BF22F0420343F040038B719BF8063079
:10A28000654A01064CBF63F07F0303F07F038BF840
:10A290000630614B1B8801331380F7F782B89BF8B7
:10A2A000063023F004038BF80630CEE75F4B1B78B3
:10A2B000002B2BD0584B594A1B88116858489BF8E3
:10A2C0000A4001339BB29A0B173150F82200524AD0
:10A2D0001380C3F30D02514B19609BF80B3082566B
:10A2E00043EA0423134499B28CE74C4B4B4819685A
:10A2F0004F4B06311A88484B01604D491B8801328B
:10A300000A80454A01331380F7F74BB8434B9BF85B
:10A3100004101B689BF8052040480B33036042EA99
:10A3200001216FE73B4B1B783BB9404B1B7823B9AE
:10A330003A4B3A4A1B6807331360374B38491C883D
:10A34000631C9BB29A0BC3F30D0051F82210324AE2
:10A3500013800B5C8BF807302F4BA21C1A80F7F789
:10A3600020B82C4B1B781BB9304B1B78002B43D0EB
:10A370002A4B2A4A1B68083313609BF807002A49B6
:10A3800000F00F035A1E431E9CB28B79D5064CBFBA
:10A3900043F0100323F010038B71C30932D080EA1D
:10A3A000040319062ED59BF8063043F004038BF8FE
:10A3B00006301D4A8BF80740937914F0FF0F14BF45
:10A3C00023F0400343F0400393719BF806302206CC
:10A3D0004CBF63F07F0303F07F038BF806309BF8DC
:10A3E00006200D4B42F002021B888BF806200A4A19
:10A3F00001331380F6F7D5BF084B084A1B680433B6
:10A400001360BAE79BF8063023F004038BF806309C
:10A41000CFE700BFC1BD01203CBD0120C4BD01206C
:10A420000CB7012091000020E0BC0120C2BD01203A
:10A430007CBC0120A54B1B781BB9A54B1B78002BBE
:10A4400054D0A44BA34A1B68083313609BF8071031
:10A45000A14A01F00F03013313F0100F937914BFD9
:10A4600043F0100323F010039371CB0901F10100B5
:10A4700042D181EA00031F063ED59BF8063043F027
:10A4800004038BF806309BF80610934A8BF80700FC
:10A4900001F0FD0310F0FF0F8BF8063014BF21F020
:10A4A000420343F0400393719BF806308B4A060643
:10A4B0004CBF63F07F0303F07F038BF80630874BBC
:10A4C0001B8801331380F6F76CBF824B81481968F3
:10A4D000834B06311A88814B016081491B88013A00
:10A4E0000A807E4A01331380F6F75BBF794B794AC5
:10A4F0001B6804331360A9E79BF8063023F00403BC
:10A500008BF80630BFE7714B1B7804F00701A3B14D
:10A51000704B70481B6803F108020B1F012B02608F
:10A5200000D804316D4B1A881BF801308BF80030CD
:10A53000531C6A4A1380F6F734BF654B1B783BB354
:10A54000644B64481A680B1FDBB20832012B0260AF
:10A55000E8D88B1DD9B2E5E75E4B9BF806201B6857
:10A560005C485D4904330360D3074CBF22F001030C
:10A5700042F001038B719BF80620584B22F0020237
:10A580001B888BF80620554A01331380F6F709BF64
:10A59000504B504A1B6804331360C3E74B4B1B7886
:10A5A0004BB34E4B4B4A1B8811684E489BF80840F2
:10A5B00001339BB29A0B133150F82200474A1380A3
:10A5C000C3F30D02434B19609BF80930825643EAEE
:10A5D000042313449BB29A0BC3F30D01414B53F870
:10A5E00022303E4A5B5C12888BF80030531C3B4A99
:10A5F0001380F6F7D6BE364B1B78002B00F0C783CE
:10A60000364B344A1B88116836489BF80A400133A0
:10A610009BB29A0B133150F82200304A1380C3F3D7
:10A620000D022C4B19609BF80B30825643EA042331
:10A6300013449BB2CFE7254B1B7804F00701002B96
:10A6400030D0244B23481B6803F108020B1F012B59
:10A65000026000D804311BF801209BF807301E4926
:10A660005A408BF807208B79002A45D003F0BF03AE
:10A6700017068B7143D563F07F038B711A4B9BF8E0
:10A6800006109A5C144801F0EC038BF80630C2B156
:10A6900043F004038371114B104A1B88013313806C
:10A6A000F6F77FBE0A4B1B7803B30A4B09481A68BA
:10A6B0000B1FDBB20832012B0260CCD88B1DD9B244
:10A6C000C9E721F017038371E5E700BFC1BD012091
:10A6D000C2BD0120C4BD0120E0BC01203CBD012061
:10A6E0007CBC01200CB7012090630108B54BB54A32
:10A6F0001B6804331360AEE743F040038B719BF893
:10A70000063003F07F038BF80630B7E7AE4B1B78BB
:10A7100004F00700002B00F01E86AA4BA9491B6815
:10A7200003F10802031F012B0A603AD90922A74B43
:10A7300019881BF800300BF80230A44A4B1C138018
:10A74000F6F72FBEA04B1B78002B00F014869F4B12
:10A750009C4A1B8811689E489BF8084001339BB2B5
:10A760009A0B133150F82200984A1380C3F30D025C
:10A77000944B19609BF80930825643EA0423134432
:10A780009BB29A0BC3F30D01914B53F822308F4AC1
:10A790005B5C12888BF80430531C8C4A1380F6F7EC
:10A7A00000BE04300922C2E7874B1B7804F007047F
:10A7B000002B5AD0834B83491B6803F10802231FE7
:10A7C000012B0A6000D804349BF807501BF80410D2
:10A7D000804805F00F0201F00F03D31A13F0100F99
:10A7E00083797C4A14BF43F0100323F01003837174
:10A7F0001BF804306B40691A18068EB240F10584CC
:10A8000085EA0103190640F10084937943F00403BB
:10A8100093719BF80630F2054CBF43F0010323F01F
:10A8200001038BF806309BF8063016F0FF0F14BFBB
:10A8300023F0400343F040038BF806309BF80630CA
:10A8400037064CBF63F07F0303F07F038BF80630BD
:10A850009BF806205D4B42F002021B888BF8062015
:10A860005A4A01331380F6F79CBD5B4B1B78002BD3
:10A8700000F0D284534B53491A68231FDBB20832CD
:10A88000012B0A60A0D8A31DDCB29DE74E4B1B78BC
:10A8900004F00701A3B14B4B4A481B6803F10802BF
:10A8A0000B1F012B026000D80431484B1A881BF89B
:10A8B00001308BF80730531C444A1380F6F771BD02
:10A8C000454B1B7893B13F4B3E481A680B1FDBB2D8
:10A8D0000832012B0260E8D88B1DD9B2E5E7394B6D
:10A8E000384A1B6804331360F6F75BBD354B354AB5
:10A8F0001B6804331360D8E7334B1B7804F007045C
:10A90000002B6BD02F4B2F491B6803F10802231F2C
:10A91000012B0A6000D804349BF807501BF8041080
:10A920009BF806002B4E01F00F0305F00F02D21A20
:10A9300000F00103D21A691ACB1AD70699B24CBF9C
:10A9400040F0100320F01003B3711BF80430214ACB
:10A950006B401E0640F1FC8785EA01031D0640F1AD
:10A96000F787937943F0040393711A4A8BF8071021
:10A970009379CC054CBF43F0010323F0010393719D
:10A980009BF8063011F0FF0F14BF23F0400343F093
:10A9900040038BF806309BF8063008064CBF63F086
:10A9A0007F0303F07F038BF806309BF80620074BEC
:10A9B00042F002021B888BF80620044A0133138000
:10A9C000F6F7EFBCC4BD0120C1BD01203CBD012094
:10A9D0000CB70120E0BC0120C2BD0120984B1B78C0
:10A9E000002B00F00185974B96491A68231FDBB2B4
:10A9F0000832012B0A608FD8A31DDCB28CE7924B82
:10AA00001B7804F00701A3B18E4B8E481B6803F13D
:10AA100008020B1F012B026000D804318B4B1A88EF
:10AA20001BF801308BF80330531C884A1380F6F76B
:10AA3000B8BC834B1B78002B39D0824B81481A68F5
:10AA40000B1FDBB20832012B0260E7D88B1DD9B295
:10AA5000E4E77D4B1B78002B2FD07C4B794A1B8879
:10AA600011687B489BF8084001339BB29A0B133165
:10AA700050F82200754A1380C3F30D02714B196020
:10AA80009BF80930825643EA042313449BB29A0B85
:10AA9000C3F30D016E4B53F822306C4A5B5C128895
:10AAA0008BF80230531C694A1380F6F77ABC654B69
:10AAB000644A1B6804331360B0E7614B1B78002BBA
:10AAC00001F00481614B5F4A1B88116860489BF864
:10AAD0000A4001339BB29A0B133150F822005B4AB3
:10AAE0001380C3F30D02574B19609BF80B3082564D
:10AAF00043EA042313449BB2C9E79BF806305F0680
:10AB000000F1D283534B1C884E4B1D68631C98B2D6
:10AB1000820B05F10B03A10B4D4D55F8211055F893
:10AB20002250484A1360C4F30D03C0F30D02C95C00
:10AB3000484B1880AB5C41EA032344490B80454BEA
:10AB4000A21C1A80F6F72DBC3F4B1B7804F00704BB
:10AB5000002B59D03B4B3B491B6803F10802231FD4
:10AB6000012B0A6000D804349BF807501BF804102E
:10AB7000394805F00F0201F00F03134413F0100FD2
:10AB80008379354A14BF43F0100323F01003837117
:10AB90001BF804306B402944DB098EB243D185EAAF
:10ABA00001031F063FD5937943F0040393712A4AAA
:10ABB0008BF807109379F5054CBF43F0010323F0A0
:10ABC000010393719BF8063016F0FF0F14BF23F0BA
:10ABD000400343F040038BF806309BF80630340600
:10ABE0004CBF63F07F0303F07F038BF806309BF8C4
:10ABF0000620164B22F002021B888BF80620134A0F
:10AC000001331380F6F7CDBB0D4B1B7893B10D4B81
:10AC10000C491A68231FDBB20832012B0A60A3D843
:10AC2000A31DDCB2A0E79BF8063023F004038BF8E9
:10AC30000630BCE7034B034A1B680433136093E7F9
:10AC4000C2BD0120C4BD0120C1BD01203CBD012009
:10AC50000CB701207CBC0120E0BC0120994B1B7883
:10AC600004F00701002B36D0974B97481B6803F17F
:10AC700008020B1F012B026000D804311BF80120D1
:10AC80009BF8073091491A408BF807208B79002AEE
:10AC900000F0D48503F0BF0314068B7140F1D18519
:10ACA00063F07F038B719BF80610894B874C985C8F
:10ACB00001F0FC0242F010038BF80630002800F08F
:10ACC000918542F01403A371824B824A1B880133A1
:10ACD0001380F6F766BB804B1B78002B00F0918049
:10ACE000794B79481A680B1FDBB20832012B0260DE
:10ACF000C4D88B1DD9B2C1E7724B1B78002B62D030
:10AD0000744B714A1B88116874489BF808400133E2
:10AD10009BB29A0B133150F822006E4A1380C3F392
:10AD20000D02694B19609BF80930825643EA0423EF
:10AD300013449BB29A0BC3F30D01684B53F82230B6
:10AD40009BF807205B5C61491A408BF807208B79E0
:10AD50007AB303F0BF0310068B712DD563F07F0328
:10AD60008B719BF806105A4B584C985C01F0FC0212
:10AD700042F010038BF80630A8B142F01403A3711F
:10AD8000544B544A1B8801331380F6F70ABB4E4BD1
:10AD90009BF804101B689BF805204B4807330360A1
:10ADA00042EA012317E421F0070343F01003A371E3
:10ADB000E6E743F040038B719BF8063003F07F0316
:10ADC0008BF80630CDE7444B1B7803B3414B3E4A2A
:10ADD0001B88116841489BF80A4001339BB29A0BCB
:10ADE000133150F822003B4A1380C3F30D02364B57
:10ADF00019609BF80B30825643EA042313449BB23C
:10AE000098E7314B304A1B680433136036E72E4B0A
:10AE10009BF804101B689BF805202B480733036040
:10AE200042EA012386E7274B1B7804F00700002B3A
:10AE300000F04583244B24491B6803F10802031FDB
:10AE4000012B0A603AD90822224B19881BF80030DE
:10AE50000BF802301F4A4B1C1380F6F7A2BA194BAD
:10AE60001B78002B00F040831A4B174A1B8811688F
:10AE70001A489BF8084001339BB29A0B133150F8E3
:10AE80002200144A1380C3F30D020F4B19609BF884
:10AE90000930825643EA042313449BB29A0BC3F34E
:10AEA0000D010E4B53F822300A4A5B5C12888BF876
:10AEB0000330531C074A1380F6F773BA0430082294
:10AEC000C2E700BFC1BD0120C4BD0120E0BC01201C
:10AED000906301083CBD0120C2BD01200CB70120D8
:10AEE000994B1B7804F00701002B34D0974B9748FF
:10AEF0001B6803F108020B1F012B026000D804310C
:10AF00001BF801209BF8073091491A438BF8072062
:10AF10008B79002A00F01E8703F0BF0315068B71A2
:10AF200040F11B8763F07F038B718A4B9BF80610FF
:10AF30009A5C874801F0EC038BF80630002A00F099
:10AF4000148743F004038371834B834A1B880133C6
:10AF50001380F6F726BA814B1B78002B00F089800E
:10AF60007A4B7A481A680B1FDBB20832012B026059
:10AF7000C6D88B1DD9B2C3E7734B1B78002B5AD0B0
:10AF8000754B724A1B88116875489BF8084001335D
:10AF90009BB29A0B133150F822006F4A1380C3F30F
:10AFA0000D026A4B19609BF80930825643EA04236C
:10AFB00013449BB29A0BC3F30D01694B53F8223033
:10AFC0009BF807205B5C62491A438BF807208B795A
:10AFD0003AB303F0BF0314068B7125D563F07F03EA
:10AFE0008B715C4B9BF806109A5C594801F0EC039E
:10AFF0008BF806308AB143F004038371564B564AEE
:10B000001B8801331380F6F7CCB99BF8063023F088
:10B0100004038BF80630FFF7FCBB21F017038371A4
:10B02000ECE743F040038B719BF8063003F07F039D
:10B030008BF80630D5E7494B1B7803B3464B434AA0
:10B040001B88116846489BF80A4001339BB29A0B53
:10B05000133150F82200404A1380C3F30D023B4BDA
:10B0600019609BF80B30825643EA042313449BB2C9
:10B07000A0E7364B354A1B680433136040E7334B77
:10B080009BF804101B689BF80520304807330360C9
:10B0900042EA01238EE72C4B1B7804F00705002BB6
:10B0A00032D02D4B294A1B8811682D489BF8084047
:10B0B00001339BB29A0B133150F82200264A1380B9
:10B0C000C3F30D02214B19609BF80930825643EA05
:10B0D000042313449AB2B2F5804F0ED3B2F5B64FA3
:10B0E00002D2204901230B70930BC2F30D011C4ABD
:10B0F00052F823201BF805305354174B164A1B886F
:10B1000001331380F6F74DB9144B1B78002B59D03F
:10B11000114B0E4A1B88116811489BF80A400133F5
:10B120009BB29A0B133150F822000B4A1380C3F3E1
:10B130000D02064B19609BF80B30825643EA04233C
:10B1400013449AB2C7E700BFC1BD0120C4BD0120AE
:10B15000E0BC0120906301083CBD0120C2BD01207C
:10B160000CB7012091000020A34B1B78002B35D099
:10B17000A24BA34A1B881168A2489BF808400133E0
:10B180009BB29A0B133150F822009C4A1380C3F3F0
:10B190000D029B4B19609BF80930825643EA042349
:10B1A00013449BB29A0BC3F30D01964B53F8223014
:10B1B000924A5B5C12888BF80530531C8F4A1380CF
:10B1C000F6F7EFB88E4B9BF804101B689BF8052030
:10B1D0008B480733036042EA01227CE78A4B1B78E5
:10B1E0000BB3864B864A1B88116886489BF80A4039
:10B1F00001339BB29A0B133150F822007F4A13801F
:10B20000C3F30D027E4B19609BF80B30825643EA64
:10B21000042313449BB2C5E7794B794A1B68043376
:10B220001360FFF7D1BA764B9BF804101B689BF8AC
:10B23000052073480733036042EA0123B2E7704BED
:10B240006F4A1B6804331360FDF766BF6A4B1B78B7
:10B25000002B35D0694B6A4A1B88116869489BF8F6
:10B26000084001339BB29A0B133150F82200634A15
:10B270001380C3F30D02624B19609BF809308256AC
:10B2800043EA042313449BB29A0BC3F30D015D4BB5
:10B2900053F82230594A5B5C12888BF80730531CF4
:10B2A000564A1380F6F77DB8554B55491A68534BEB
:10B2B00005321B880A60514A01331380F6F771B8D2
:10B2C000514B1B78002B00F0CF804C4B4C4A1B8815
:10B2D00011684C489BF80A4001339BB29A0B13311A
:10B2E00050F82200454A1380C3F30D02444B196005
:10B2F0009BF80B30825643EA042313449BB2C3E706
:10B300003D4B1B7804F00701A3B13D4B3C481B6843
:10B3100003F108020B1F012B026000D80431374BE8
:10B320001A881BF801308BF80230531C334A138003
:10B33000F6F737B8344B1B78002B00F0CF80304B3A
:10B340002F481A680B1FDBB20832012B0260E6D8C7
:10B350008B1DD9B2E3E72C4B1B78002B2FD0284B49
:10B3600027491A68031FDBB20832012B0A6021D972
:10B370000B22FFF7DCB9244B1B7843B31F4B204A49
:10B380001B8811681F489BF80A4001339BB29A0B37
:10B39000133150F82200194A1380C3F30D02184BE1
:10B3A00019609BF80B30825643EA042313449BB286
:10B3B000FFF7E7B9831DD8B20B22FFF7B8B9104BDE
:10B3C0000F4A1B68043313600522FFF7B0B90C4B1A
:10B3D0009BF804101B689BF805200948073303609D
:10B3E00042EA0123FFF7CDB9054B054A1B68043338
:10B3F0001360FFF791BA00BFC1BD01203CBD012021
:10B40000C4BD01200CB70120C2BD0120A74B1B7891
:10B41000002B35D0A64BA74A1B881168A6489BF87D
:10B42000084001339BB29A0B133150F82200A04A16
:10B430001380C3F30D029F4B19609BF809308256AD
:10B4400043EA042313449BB29A0BC3F30D019A4BB6
:10B4500053F82230964A5B5C12888BF80130531CFB
:10B46000934A1380F5F79DBF924B9BF804101B681D
:10B470009BF805208F480733036042EA012303E766
:10B480008E4B1B78002B4DD0894B8A4A1B88116844
:10B4900089489BF80A4001339BB29A0B133150F84C
:10B4A0002200834A1380C3F30D02824B19609BF87C
:10B4B0000B30825643EA042313449BB2C4E77F4B0C
:10B4C0001B78002B4AD07B4B7A491A68031FDBB2EA
:10B4D0000832012B0A603DD90A22B5E4754B754A42
:10B4E0001B68043313601AE7744B1B7833B3704B3B
:10B4F000704A1B88116870489BF80A4001339BB260
:10B500009A0B133150F82200694A1380C3F30D02DD
:10B51000684B19609BF80B30825643EA04231344AE
:10B520009BB2BBE4634B9BF804101B689BF805209F
:10B5300060480733036042EA012385E75D4B9BF8CF
:10B5400004101B689BF805205A480733036042EA41
:10B550000123A3E4831DD8B20A2275E4554B554A52
:10B560001B680433136004226EE4504B1B7804F014
:10B570000704002B5BD04F4B4E491B6803F10802B8
:10B58000231F012B0A6000D804341BF804109BF819
:10B5900007504B4805F00F0201F00F03D31A13F0C8
:10B5A000100F8379464A14BF43F0100323F01003B1
:10B5B00083711BF804306B40691A1C068EB240F18F
:10B5C0007A8285EA0103180640F17582937943F087
:10B5D000040393713A4A8BF807109379F1054CBF35
:10B5E00043F0010323F0010393719BF8063016F03A
:10B5F000FF0F14BF23F0400343F040038BF80630E5
:10B600009BF8063037064CBF63F07F0303F07F03DF
:10B610008BF806309BF80620254B42F002021B886F
:10B620008BF80620224A01331380F5F7BABE234B6C
:10B630001B78002B00F07C831E4B1E491A68231FC9
:10B64000DBB20832012B0A609FD8A31DDCB29CE755
:10B650001C4B1D88174B1C68154B1F886B1C98B220
:10B66000A90B04F10A03144C820B54F8214012492F
:10B6700051F822600F4A1360C5F30D03C0F30D01AA
:10B68000E25C104B1880735C42EA03231BB2C3F3E5
:10B6900007208BF801300B4B8BF80000A91C198098
:10B6A000034B7A1C1A80F5F77CBE00BFC1BD012098
:10B6B0003CBD0120C4BD01200CB70120C2BD01204A
:10B6C000E0BC01207CBC01209BF804209BF80530E5
:10B6D000B7490C6843EA02218B0BB64A52F8232083
:10B6E00004F10F03B24CC1F30D002360125CFAF7B2
:10B6F00005BBB14B1B78002B00F08280AF4BAC4AEE
:10B700001B881168AB489BF8084001339BB29A0B29
:10B71000133150F82200A94A1380C3F30D02A44B41
:10B7200019609BF80930825643EA042313449BB204
:10B730009A0BC3F30D019F4B9BF8074053F822303F
:10B740009BF806005D5C9E4E05F00F0204F00F03AF
:10B75000991A00F00103621BC91AC906A2EB030380
:10B760009FB24CBF40F0100320F01003B37185EA84
:10B7700004031A063DD584EA07031B0639D59BF856
:10B78000063043F004038BF806308D4A8BF80770BF
:10B790009379FE054CBF43F0010323F0010393713D
:10B7A0009BF8063017F0FF0F14BF23F0400343F05F
:10B7B00040038BF806309BF806303D064CBF63F023
:10B7C0007F0303F07F038BF806309BF806207B4B4A
:10B7D00042F002021B888BF80620784A013313805E
:10B7E000F5F7DFBD21F0070343F01003A371FFF766
:10B7F0006BBA9BF8063023F004038BF80630C4E7DD
:10B80000704B1B782BB36D4B694A1B8811686948D4
:10B810009BF80A4001339BB29A0B133150F8220077
:10B82000664A1380C3F30D02614B19609BF80B301D
:10B83000825643EA042313449BB279E743F0400362
:10B840008B719BF8063003F07F038BF80630FFF70F
:10B850002ABA574B9BF804101B689BF805205448E4
:10B860000733036042EA012362E7534B1B78002B46
:10B870007DD0524B4E4A1B8811684E489BF80840B9
:10B8800001339BB29A0B133150F822004B4A1380BC
:10B89000C3F30D02464B19609BF80930825643EA08
:10B8A000042313449BB29A0BC3F30D01414B9BF845
:10B8B000074053F82230585C414900F00F0204F071
:10B8C0000F039B1A13F0100F8B7914BF43F0100372
:10B8D00023F010038B7180EA0403221A1E0695B22E
:10B8E0003ED584EA020318063AD59BF8063043F0A9
:10B8F00004038BF806308BF80720314A9379E90569
:10B900004CBF43F0010323F0010393719BF8063011
:10B9100015F0FF0F14BF23F0400343F040038BF8F2
:10B9200006309BF806302A064CBF63F07F0303F015
:10B930007F038BF806309BF80620204B42F0020272
:10B940001B888BF806201D4A01331380F5F729BDAB
:10B950009BF8063023F004038BF80630FFF705B898
:10B960009BF8063023F004038BF80630C3E7154B31
:10B970001B78002B00F0A680104B0D4A1B88116825
:10B980000C489BF80A4001339BB29A0B133150F8D4
:10B9900022000A4A1380C3F30D02054B19609BF87D
:10B9A0000B30825643EA042313449BB27BE700BF6B
:10B9B000C4BD01200CB70120C1BD01203CBD012048
:10B9C000E0BC0120C2BD0120B94B1B78002B00F068
:10B9D0008C80B84BB84A1B881168B8489BF808405F
:10B9E00001339BB29A0B133150F82200B14A1380F5
:10B9F000C3F30D02B04B19609BF80930825643EA3D
:10BA0000042313449BB29A0BC3F30D01AB4B9BF879
:10BA1000060053F822309BF807505C5CA84E00F0FB
:10BA2000010105F00F030B4404F00F021A446319DF
:10BA30001944D3064CBF40F0100320F01003B3713B
:10BA400084EA0503DB0949D185EA01031F0645D5D0
:10BA50009BF8063043F004038BF80630984A8BF8C5
:10BA600007109379CE054CBF43F0010323F0010387
:10BA700093719BF8063011F0FF0F14BF23F04003C1
:10BA800043F040038BF806309BF806300D064CBFA0
:10BA900063F07F0303F07F038BF806309BF80620EA
:10BAA000844B22F002021B888BF80620814A013366
:10BAB0001380F5F776BC9BF8063023F004038BF86F
:10BAC000063087E57C4B9BF804101B689BF805202B
:10BAD00079480733036042EA0123E4E69BF8063025
:10BAE00023F004038BF80630B8E7764B1B78002B65
:10BAF00000F040816F4B704A1B8811686F489BF8BB
:10BB00000A4001339BB29A0B133150F82200694A64
:10BB10001380C3F30D02684B19609BF80B308256FB
:10BB200043EA042313449BB26DE7614B1B78002B5F
:10BB300000F03A815F4B604A1B8811685F489BF8B0
:10BB4000084001339BB29A0B133150F82200594A36
:10BB50001380C3F30D02584B19609BF809308256CD
:10BB600043EA042313449BB29A0BC3F30D01534BD6
:10BB700053F822309BF807205B5C51495A408BF800
:10BB800007208B79002A00F0058103F0BF03160619
:10BB90008B7140F1028163F07F038B714A4B9BF8FC
:10BBA00006109A5C464801F0EC038BF80630002A38
:10BBB00000F0EC8043F0040383713E4B3D4A1B8848
:10BBC00001331380F5F7EDBB394B1B78002B00F0E8
:10BBD0009180384B384A1B88116838489BF80840D8
:10BBE00001339BB29A0B133150F82200314A138073
:10BBF000C3F30D02304B19609BF80930825643EABB
:10BC0000042313449BB29A0BC3F30D012B4B9BF8F7
:10BC1000074053F82230585C294900F00F0204F025
:10BC20000F039B1A13F0100F8B7914BF43F010030E
:10BC300023F010038B7180EA0403221A1E0695B2CA
:10BC400051D584EA020318064DD59BF8063043F01F
:10BC500004038BF806309BF80630E9054CBF43F02F
:10BC6000010323F001038BF806309BF8063015F032
:10BC7000FF0F14BF23F0400343F040038BF806305E
:10BC80009BF806302A064CBF63F07F0303F07F0366
:10BC90008BF806309BF80620064B42F002021B8808
:10BCA0008BF80620034A01331380F5F77ABB00BFF7
:10BCB000C1BD01203CBD0120C4BD01200CB7012045
:10BCC000E0BC0120C2BD0120906301084B4B9BF8F2
:10BCD00004101B689BF8052048480733036042EABC
:10BCE0000123FEF7D4BE9BF8063023F004038BF843
:10BCF0000630B0E7424B1B7803B3424B3F4A1B88E8
:10BD0000116841489BF80A4001339BB29A0B1331EA
:10BD100050F822003B4A1380C3F30D02374B1960E1
:10BD20009BF80B30825643EA042313449BB26AE724
:10BD3000324B324A1B680433136026E42F4B9BF8C6
:10BD400004101B689BF805202C480733036042EA67
:10BD5000012358E743F040038B719BF8063003F052
:10BD60007F038BF80630FFF7E0B821F017038371EB
:10BD7000FFF7EAB8214B9BF804101B689BF80520DD
:10BD80001E480733036042EA01233CE621F0170313
:10BD9000837112E743F040038B719BF8063003F088
:10BDA0007F038BF80630F9E6154B1B78D3B1154BA2
:10BDB000124A1B88116814489BF80A4001339BB251
:10BDC0009A0B133150F822000E4A1380C3F30D0270
:10BDD0000A4B19609BF80B30825643EA0423134444
:10BDE0009BB2C1E6054B9BF804101B689BF805202D
:10BDF00002480733036042EA0123B5E6C4BD0120CF
:10BE0000C2BD01203CBD01200CB70120016809B36F
:10BE100010B40C78202C09D93A2C16D00A4601E02F
:10BE20003A2B07D012F8013F202BF9D800205DF8FB
:10BE3000044B704701318A4207D1302C05D10132C1
:10BE400002605DF8044B002070474FF0FF305DF852
:10BE5000044B70474FF0FF30704700BF2DE9F041B1
:10BE600007468846066861BBF5681DB3B3699D4205
:10BE700028BF012533690BB3B3692C4606E00128BE
:10BE800015D0013058D0AC4218D0B36901349C426F
:10BE900002D3012D12D902242146386806F080F918
:10BEA0000028ECD1012C02D9B3699C422CD301208B
:10BEB000BDE8F08133690125002BDDD10020BDE80C
:10BEC000F081304606F06CF90128F0D9421C33D0DD
:10BED000B369984243D33269002AEFD008F10104D4
:10BEE000A34298BF02242146386806F059F9012878
:10BEF000DDD0431C20D0A0B3F568B369012D33D940
:10BF00009D4228BF4546B8E74FF0FF3221463046F4
:10BF100006F0A8F970B9B8F1000F11D0B8F1010F0F
:10BF2000C5D9B3699845C2D241462246304606F08B
:10BF300099F928B10128BAD14FF0FF30BDE8F0815E
:10BF4000B3693269F460023B9A4201D8013A326126
:10BF5000337943F0010333712046BDE8F081BDE839
:10BF6000F081002C9ED1B369454686E708B10420D4
:10BF700070472DE9F04FDFF86892904E904C914D4C
:10BF800030704FF0010E2060C5F800E0C9F82C00B9
:10BF9000D9F83C70DFF854828B4BDFF854C247F479
:10BFA0004A7747F00207C9F83C704FF07469C8F847
:10BFB00008901F6827F001071F601F6827F001071E
:10BFC0001F602127186058609860D86018615F6111
:10BFD000C8F80890D3F800907C487D4F09EA0C0C13
:10BFE0004CEA00001860D3F814C07A48A8F59B38D2
:10BFF000A8F5C0784CF0070C4FF40079C3F814C0D2
:10C00000C3F80490C3F80880D960196841F01001A2
:10C010001960196841F020011960196841EA0E01A0
:10C020001960C7F800E0036883B05202022B009247
:10C0300000F0A380684F00224FF0100B4FF4007AFD
:10C040004FF040094FF48068FA6087E8000CC7F8A9
:10C050000890C7F8108006F0B1FF584602F096F835
:10C06000002841D05D490B687BB923686BB93378F0
:10C070005BB94FF0FF3305E0226832B9327822B95C
:10C08000013B02D00A68002AF6D00023544A0B6014
:10C09000536B13F4805400F086804FF0FF3401E0BE
:10C0A000002C6DD0536B13F4805704F1FF34F7D19B
:10C0B0002A68444D012A6ED0002C6AD03846484B7D
:10C0C0003E4940F2FF529A6333785BB10878C4B2BC
:10C0D00002F0E8F80028FBD1201C18BF012003B0B3
:10C0E000BDE8F08F0446F3E73E4AF8601268C7F8EF
:10C0F000089002FA0BF24FF0370BC7F8108087E870
:10C10000040806F05BFF584602F040F80028A9D169
:10C1100017224FF0010BF8607A600192C7F808907F
:10C12000C7F81080C7F800B006F048FF019A104623
:10C1300002F02CF8002895D11922009BF8607A6053
:10C1400000923B60C7F80890C7F8108006F036FFF1
:10C15000009A104602F01AF8002883D1224B4FF0C3
:10C16000FF319022C3F804A0D8601861C3F814B05E
:10C1700019609A6006F03CFF74E7530A009359E790
:10C180002B68104D012B04D102F076F82C600028AA
:10C1900095D1042093E702F06FF82F60002C8ED128
:10C1A00000288CD1F5E72B68064D012B01D02046E5
:10C1B00085E702F061F82C6081E700BF442500208C
:10C1C0003C25002094240020586402404054A308D9
:10C1D0008C8525422C250020D0BD0120482500203B
:10C1E000002C01403025002090C301200064024053
:10C1F0003F801CF083690BB9042070472DE9F04F94
:10C2000005692035B5F5001F83B003D3042003B0C2
:10C21000BDE8F08FC5F308068846044607684EBBA4
:10C2200041690133836161B3B7F80A9009F1FF39BD
:10C2300019EA55291ED1384605F0B2FF0128824679
:10C2400027D9B0F1FF3F34D0BB69984223D2831E77
:10C25000019307F13408C4F814A0BB690199023BAB
:10C26000994204D2B7F80A90FB6A01FB0939C4F875
:10C27000189001E007F134084644E661256100208A
:10C28000C5E73B89B3EB551FF4D80023A361042015
:10C29000BDE70220BBE7B8F1000FF6D06169204688
:10C2A000FFF7DCFD824630B90720B0E77889834587
:10C2B000D1D00120ABE70128EBD0B0F1FF3FF8D09F
:10C2C000FB7843BBBB69AAF10202023B9A4201928E
:10C2D00027D300230093009B3B6307F134084346B8
:10C2E00007F50D71002203F8012B9942FBD14FF0A5
:10C2F000000B06E07878FFF739FE0028D6D10BF165
:10C30000010B7889009B834503EB0B0241464FF0FC
:10C310000103EFD3CBE7384606F032F80028D1D03E
:10C32000C7E77A89FB6A019901FB02330093D2E7E0
:10C3300008B1042070472DE9F04FDFF810927B4DD3
:10C340007B4C7C4E28704FF0010C2060C6F800C07A
:10C35000C9F82C00D9F83CE0DFF8F481764B774F30
:10C360004EF44A7E4EF0020EC9F83CE04FF074697C
:10C37000C8F80890D3F800E02EF0010EC3F800E0F2
:10C38000D3F800E02EF0010EC3F800E04FF0210ECC
:10C39000186058609860D8601861C3F814E0C8F855
:10C3A00008901868DFF8AC91DFF8ACE1DFF8AC81F9
:10C3B000074047F00A6040F45530186058694FF460
:10C3C000007740F0070058615F60C3F80890D960BB
:10C3D00019685B4F41F010011960196841F02001A4
:10C3E0001960196841EA0C011960C8F800C0DEF84C
:10C3F000003083B0022B4FEA422B4FF000034FF482
:10C4000000724FF010084FF0400A4FF480693A6014
:10C41000019208BF4FEA5B2BFB60C7F80480C7F8A6
:10C4200008A0C7F8109006F0C9FD404601F0AEFE26
:10C43000019AF8B9434B01905A604FF0FF319022B6
:10C4400019609A60022101221861D9604FF0120828
:10C450005A6106F0CDFD0198F860C7F800B0C7F842
:10C4600008A0C7F81090C7F8048006F0A7FD404662
:10C4700001F08CFE34490B687BB923686BB92B78CB
:10C480005BB94FF0FF3305E0226832B92A7822B950
:10C49000013B02D00A68002AF6D000232B4A0B6029
:10C4A000536B13F4005437D04FF0FF3400E004B363
:10C4B000536B13F4005704F1FF34F8D132681D4E6A
:10C4C000012A21D0F4B13846204B184940F2FF52DE
:10C4D0009A632B785BB10878C4B201F0E3FE0028C0
:10C4E000FBD1201C18BF012003B0BDE8F08F04462B
:10C4F000F3E733680F4E012B04D101F0BDFE346029
:10C500000028E1D10420DFE701F0B6FE3760002CFF
:10C51000DAD10028D8D1F5E73368064E012B01D0D7
:10C520002046D1E701F0A8FE3460CDE74425002085
:10C530003C25002094240020586402403F801CF0D9
:10C54000D0BD012090C3012048250020002C0140CF
:10C5500000640240802C01402C2500208C8525425F
:10C5600038B5036B8B4218D0C37804460D467BB9AF
:10C570002A46012304F134016078FFF7D9FE002830
:10C5800018BF4FF0FF3525630CBF0020012038BDD8
:10C5900005F0F6FE0028EBD038BD002038BD00BF06
:10C5A00000224FF0FF3310B5C27003630446FFF75B
:10C5B000D7FF08B1042010BD94F8331294F832323A
:10C5C0004AF6552243EA0123934201D0032010BDCD
:10C5D00094F83430EB2B05D01833DBB2012B01D9A2
:10C5E000022010BD94F86A30462B07D194F86B30C6
:10C5F000412B03D194F86C30542B15D094F886302D
:10C600000A4904F18702463B8B34002BE8D112F82B
:10C61000013B11F8010FA242A3EB0003F5D1002B5F
:10C6200014BF0220002010BD002010BD10650108BD
:10C630002DE9F84F0B78D0F800902F2B0C4682464E
:10C6400041D05C2B3FD0D9F81430836023781F2B66
:10C6500043D90AF120080AF12B062025434603F8A6
:10C66000015BB342FBD123782E2B3ED00027384606
:10C6700004F1FF3E4FF0080C1EF8013F202B00F1A3
:10C68000010040F2C9802F2B4AD05C2B48D02E2BC2
:10C690003AD0BC4535D91A063DD4222B31D06D494C
:10C6A00001E09A422DD011F8012F002AF9D1A3F10F
:10C6B0006102192A01D8203BDBB208F807300137A4
:10C6C000DAE714F8013F2F2BFBD05C2BF9D00023C5
:10C6D000CAF8083023781F2BBBD880238AF82B3068
:10C6E0005046BDE8F84F06F09DBC8AF820306378CC
:10C6F0002E2B40F09E808AF82130A3782E2B40F01C
:10C7000092800620BDE8F88FBCF10B0FF9D0082706
:10C710004FF00B0CB0E703F07F034F4AD35CBCE74C
:10C720002044044610F8012B2F2AFAD05C2AF8D0B6
:10C73000002FE6D09AF82020E52A04BF05228AF8C7
:10C740002020202B8CBF002304238AF82B30504656
:10C75000DAF8007006F066FC60BBDAF818103846AC
:10C76000FFF7FEFE30BBDAF81C201378002B49D00F
:10C7700092F80BC00CF03F038AF80630D37A1B07FF
:10C7800012D496469AF820101EF80B3B01325B1A21
:10C790000AF1210143B912F8013B11F801BB96459A
:10C7A000CBEB0303F6D1A3B100215046FFF722FDE6
:10C7B0000028D2D004289AF82B302FD198063CD5E7
:10C7C00059077FF54BAF80238AF82B300020BDE856
:10C7D000F88F9AF82B305B072DD41CF0100F1FD068
:10C7E000DAF8103099F8001009F13402C3F30803A5
:10C7F00013440329D87E9A7E42EA002205D0CAF863
:10C8000008202BE79AF82B30D8E7597D1B7D43EAA7
:10C81000012342EA0342F2E7044489E7BDE8F88FC6
:10C820000520BDE8F88F03222F2B0BD114442023C1
:10C830008BE70222F8E7BDE8F88F5A07F0D504200D
:10C84000BDE8F88F5C2BF1D0202B3FF65AAF144493
:10C8500024237AE71865010890640108044B054A0F
:10C860001B6803FB00F010601368002BFCD17047BD
:10C870007400002080240020064B074A1B68012B0F
:10C8800018BFB0FBF3F0013010601368002BFCD12F
:10C89000704700BF1400002080240020034B1A685A
:10C8A00012B11A68013A1A60704700BF8024002054
:10C8B00030B42B4B99891A888C0602D592B2900617
:10C8C00023D4274A9189138809069BB201D51B06F8
:10C8D00001D430BC70474FF67F73224913800B6838
:10C8E000002B31D02048214B02689B5C0132FE2A8C
:10C8F000026004BF002202600A681948DBB29BB2E2
:10C90000013A0A60838030BC70474FF6DF71184AE5
:10C9100019809B8812689BB212B9DAB2032A1AD026
:10C92000144A11687F29CCD81349144D0C68DBB226
:10C93000601C2B557F2888BF0023086088BF0B60D0
:10C94000136801331360BCE70D4A136823F08003BA
:10C95000136030BC70470B4A01211160E0E700BF53
:10C9600000440040842400207C2400207C220020FD
:10C970007C000020481E002088240020AC1D0020E0
:10C980000C440040902400200E4A1368FD2BFCD874
:10C9900030B40D4B0D4D1C68611CFD291960C0B2EF
:10C9A00088BF0021285588BF196072B6136801330B
:10C9B000136062B6064A136843F08003136030BC0C
:10C9C000704700BF842400208C2400207C2200209B
:10C9D0000C4400400FB430B583B006AB0D4C53F897
:10C9E000042B01934FF48071204609F08DF8204606
:10C9F00009F044F80546207828B1FFF7C5FF14F880
:10CA0000010F0028F9D1284603B0BDE8304004B03A
:10CA1000704700BF7C23002010B50446007828B181
:10CA2000FFF7B2FF14F8010F0028F9D110BD00BFC5
:10CA3000034B5B6B034214BF01200020704700BF13
:10CA4000002C0140044B82B0034400220192019368
:10CA5000019B186802B07047142C014010B4214C9F
:10CA6000A36803F00C03042B1BD0082B1CD01E4B17
:10CA700003601C4A1D499468C4F303140C5DE34031
:10CA800043609468C4F382240C5D23FA04F4846048
:10CA900092685DF8044BC2F342328A5CD340C360B3
:10CAA0007047134B0360E4E76368616813F4800F19
:10CAB000636818BF0E4C01F03F020CBF0A49B4FB7B
:10CAC000F2F1C3F3881308BFB1FBF2F101FB03F2EB
:10CAD000044B5B68C3F3014301335B00B2FBF3F328
:10CAE0000360C6E7003802400024F4008000002004
:10CAF00000127A000022F0B513460126032704E055
:10CB00000133102B02F102022FD00D6806FA03F454
:10CB100034EA0505F4D1D0F800E007FA02F5ED4358
:10CB20000EEA050EC0F800E091F804E0D0F800C06D
:10CB30000EFA02FE4EEA0C0EC0F800E091F804E096
:10CB40000EF1FF3EBEF1010F07FA02FC0ED9C468D8
:10CB500024EA0C04C460CC79C568944001332C43AA
:10CB6000102BC46002F10202CFD1F0BDD0F808E072
:10CB700005EA0E05856091F805E085680EFA02FE6B
:10CB80004EEA05058560456825EA040444608C7911
:10CB900045689C40A4B22C434460D8E7F0B4114BE4
:10CBA0004578D968827807780F4EC943C1F30221CE
:10CBB000C1F10404E4B20F2305FA04F40B41E4B21A
:10CBC00013402343F2191B01DBB282F800330378D0
:10CBD000012203F01F015B098A4046F82320F0BCC4
:10CBE000704700BF00ED00E000E100E02DE9F04FEC
:10CBF00000238FB00B600C46FFF708F9002813DB09
:10CC0000784B53F820509DB125602B781BB16B7881
:10CC1000002B00F0D480C0B2002368702B7058B194
:10CC200003200FB0BDE8F08F0B200FB0BDE8F08FF0
:10CC30000C200FB0BDE8F08F6B4B6C4E596A7060E2
:10CC400041F400615962596A694AB06021F4006197
:10CC5000596230605368674F674CF06023F4FD43BE
:10CC600023F07F0343F07603536003210123116017
:10CC70003B6076224FF4806323613061327520601F
:10CC80006060A060E06006F099F94FF4803308938B
:10CC9000089B2BB909E0089B013B0893089B23B133
:10CCA0008020FFF7C5FE0028F5D0089B002BB7D0E9
:10CCB0004F4F40F2FF53BB634FF4D5730820402120
:10CCC000002223604FF4806323616060A160E26012
:10CCD00006F074F94FF4803309937B6B13F0450F22
:10CCE0000CD1099A52B1394601E0099A32B1099B37
:10CCF000013B09934B6B13F0450FF6D0099A12B123
:10CD0000580740F1FF833A4B04229A6300274FF003
:10CD1000370840224FF480632760E760C4F804803E
:10CD2000A260236106F04AF94046019701F02EFA0D
:10CD30000023372740214FF480622360E36067605F
:10CD4000A160226106F03AF9384601F01FFA002886
:10CD50007FF466AF284FDFF898A006958046002341
:10CD60004FF037094FF0400B4FF480652360E360CC
:10CD7000C4F80490C4F808B0256106F01FF94846CD
:10CD800001F004FA00287FF44BAF019BC7F808B00C
:10CD900043F0004343F480132922F8603D613B6077
:10CDA0007A6006F00BF9DAF8340010F0450FFAD08B
:10CDB00010F0040005D00E4B04229A6330E71846A9
:10CDC0002FE740F2FF53CAF83830FFF73BFE002848
:10CDD00008F10108064B11DB4FF6FF739845BED1F1
:10CDE0001EE700BF441E002000380240142500202A
:10CDF000002C0140A0802542D0BD01204FF6FF72DB
:10CE00009045069D3FF40CAF420040F1AB82DFF845
:10CE1000A8830222C8F800201B689F073FF400AFD8
:10CE2000914600230221C0222360E3604FF4806317
:10CE30006160A260236106F0C1F801F08FF900285B
:10CE40007FF4EEAEFFF7FEFDD64F38600420FFF70B
:10CE5000F9FD78600820FFF7F5FDB8600C20FFF7BA
:10CE6000F1FDB9F1020FF86003D9B9F1060F40F0F6
:10CE7000EE830023402203212360E3604FF48063AC
:10CE8000A2606160236106F099F8C74A536B13F002
:10CE9000450FFBD058078ED413F0010040F0D0832B
:10CEA000C14A1369DBB2032B7FF4BAAE40F2FF53E1
:10CEB0009363FFF7C7FD10F4604F7FF4B1AE030C2E
:10CEC000BA4A0692190413600922C0236260A36063
:10CED00000224FF480632160E260236106F06EF867
:10CEE00001F03CF900287FF49BAEB14B0193FFF7B2
:10CEF000A9FDAF4B81460420C3F80090FFF7A2FDC7
:10CF0000AB4B58600820FFF79DFDA94B98600C20A3
:10CF1000FFF798FDA64BD8600023A3483360426812
:10CF2000337522F4FD4222F07F024260019AA1494A
:10CF30005268D8F8008073604FEA196E5FFA8EF07D
:10CF40004FEA901A4FEA126C81F800A0C9F3074B20
:10CF5000C9F3072A4FEA0C1CCEF3830E00F003003E
:10CF60005FFA89F981F801E0887081F803B00698CA
:10CF700081F804A081F80590A1F806C0B1F806C0B8
:10CF8000D0F800B0B360100AC2F307491FFA8CFC56
:10CF90005FFA80FE4CEA191C4FEADE1A09F00F090D
:10CFA000A1F806C0B8F1010F81F80890C0F3801C09
:10CFB00081F809A0C0F34019C0F3001A81F80AC033
:10CFC000F36081F80B90336181F80CA081F85680F2
:10CFD000A1F854B0DFF8D8C14B7340F2D582B8F154
:10CFE000020F00F09B82DCF80800019A4FEA4E0322
:10CFF00003F07E03CEF3801E81F819E0D2F80CA076
:10D000008B7691F81AE03A684FEA1A63C0B24EEA9A
:10D01000D01E4FEA830C00F07F0081F81AE00CF07C
:10D020000C0CC8764FEAD31EC3F34110C3F382033E
:10D0300081F81CE048778B7781F81FC091F81FE0DA
:10D040004FEA1A4C5FFA8CF94FEA1A234EEA991EFE
:10D05000CCF3401C81F81FE009F0010981F820C0E1
:10D060005FFA83FE4FF0000C81F821C081F8229016
:10D070004FEADE1981F82390C3F3801981F82490D8
:10D08000C3F3401981F82590CAF34600C3F3001991
:10D09000C2F3074AC3F3810381F826904FEA0A2AB4
:10D0A00081F827300EF0030E130E4FF0010981F8BE
:10D0B00028E081F8290081F82A9081F82C30A1F825
:10D0C0002EA0CB8D7868DFF8F4A01FFA83FEC2F3A0
:10D0D00007234EEA03031206CB850A630A6B4FEA65
:10D0E000106E42EA0E420A630B6BC4F80CC04FEAA2
:10D0F000102C0CF47F4C4CEA03030B630B6BBA68E7
:10D10000FF68C0F3072C4CEA030C4FEA124EC1F83B
:10D1100030C04FEA0E634FEA126CC0B281F834009F
:10D1200081F835C08B63886B4FEA022E0EF47F0EB8
:10D130004EEA00008863886B120202F47F420243C9
:10D140008A638A6B42EA17628A6391F83CE03A0C80
:10D15000C2F3031012024EEA000002F4706281F87A
:10D160003C00CA87CA8FC7F3072E92B24FEA0B4022
:10D1700042EA0E024FF0070BC7F3460E40234FF46E
:10D180008067CA87206081F840E0C4F804B0A360DB
:10D1900081F84190276105F011FF584600F0F6FF35
:10D1A0000EE000BF00250020002C014030250020AB
:10D1B000F0240020982400202C250020D0BD012040
:10D1C00000287FF42DADB8F1030F3FF429ADB8F17D
:10D1D000020F00F2BA80FFF735FC10F000707FF408
:10D1E0001FAD4FF0100B40234FF008080A900B9032
:10D1F000CAF80C00CAF80830CAF810708AE80009AA
:10D2000005F0DCFE584600F0C1FF00287FF408ADB1
:10D21000069BCAF80C001A68CAF8107002FA0BF2E2
:10D2200040234FF0370B8AE80408CAF8083005F0AD
:10D23000C5FE584600F0AAFF834600287FF4F0ACF4
:10D24000C84A30204FF0FF330221C2F80480136037
:10D250009060C2F810B0C2F814904FF03308D1605B
:10D2600005F0C6FE4023CAF800B0CAF80830CAF874
:10D270000CB0CAF81070CAF8048005F09FFE404652
:10D2800000F084FF00287FF4CBACDFF8DC820DF1E6
:10D290002409C24604E0FFF7CBFB002840F0D98107
:10D2A000D8F83420B04F40F22A6313404FF40010F6
:10D2B000002BF0D00820FFF7BBFB002800F0138202
:10D2C0000823BB63ACE440F2FF53BB630A9B1BBA69
:10D2D00059037FF5A5AC069BE0601B684FF0370A49
:10D2E0001B044FF040094FF4806884E80804C4F838
:10D2F0000890C4F8108005F061FE504600F046FF2B
:10D300009A4B00287FF48CAC02220624D860C3F824
:10D310000890C3F8108083E8140005F04FFE204603
:10D3200000F034FF00287FF47BAC30607B68307500
:10D3300023F4FD4323F07F0343F400634FF40062C2
:10D340007060B06030617B60F26000212846FFF7BA
:10D3500027F902281AD0042838D0012840F2008189
:10D360000D205EE41B689B073FF45AACDFF8108287
:10D37000D8F80090B9F1040F7FF453AD7C4B0193C2
:10D38000D3F800907B4B7C4F0693C5E50AAC26464C
:10D3900005F5FE7005F50F7710F8063C43B10188DE
:10D3A00010F8012C10F8023C42EA012243EA022361
:10D3B0001030B84246F8043BEED10EAF54F8046B7F
:10D3C00036B90320A742F9D10428C9D1012028E4A5
:10D3D00031462846FFF7E4F80128F3D895F84020B5
:10D3E00095F83F3043EA0223B3F5007FB8D195F8B2
:10D3F0004B1095F84A3053EA012340F02681B5F8E6
:10D400005A1095F8593095F8582043EA012342EA1A
:10D41000032195F84470E9617B1E012BAF709FD802
:10D4200095F841309AB201FB07F76A81002A97D03C
:10D430005A1E1A4294D195F8452095F8464042EA82
:10D44000042422072C818BD195F8480095F84720B9
:10D4500052EA002209D1B5F856E095F8550095F842
:10D46000542040EA0E2042EA002295F843E095F865
:10D47000420050EA0E203FF473AF00EB141EBE448E
:10D480007245FFF46DAFDFF8FCC0CEEB0202B2FBD9
:10D49000F3F35A1E62453FF663AF4FF6F5729342BF
:10D4A00000F2EC8040F6F572934200F2D78002332E
:10D4B00030440EEB0602AB616862EA622E62002C19
:10D4C0003FF44EAF03EB4302384403F0010303EB98
:10D4D0005203A862012203F2FF13B1EB532FFFF4B2
:10D4E0003FAF4FF0FF3380212B61EB60297123495F
:10D4F0002A700B8801339BB200200B80EB8068619F
:10D50000FFF78FBB590602D5174B40229A631C4B7D
:10D5100001221A604FF08043019309E4130403F4DD
:10D520007C130B61DCF808000B69020E43EA02234E
:10D530000B610B69C0F3074213430B610A690023B7
:10D54000013243F10003DB0443EA52334FF4007C21
:10D55000D204CB648A64C0F3072EC1F850C044E5FE
:10D5600000263BE790C30120002C0140D0BD0120E4
:10D57000F024002030250020002500201025002068
:10D580002C250020F4FFFF0F830203F440630B619E
:10D590000B69DCF80800920002F47F7213430B6100
:10D5A000D1F810C0020E030C5FFA82FE4FEA430965
:10D5B0004CEA9E1C0EF0070A09F00609C2F3C20EDF
:10D5C000C3F34212C3F38203C1F810C081F814E020
:10D5D00081F815A08A75CB7581F818900B7EC0F381
:10D5E000072E43EADE130B760B6907930B7E91F847
:10D5F00008904FF0010C02330CFA03F30CFA09FC0B
:10D600004FEAE37AA3FB0C23CDE90423CDE90223FF
:10D61000079BC1F850C003F10109059B0CFB0A33BD
:10D620000393029BA3FB0923CDE90423059A039BE3
:10D6300009FB03230593DDE90423C1E91223D4E4A4
:10D640005A4B01229A63FFF7EBBA1946E1E6012330
:10D6500036E4DAF8803049F8043F21E602333044FA
:10D660000EEB0602AB616862EA622E62002C3FF4A8
:10D6700077AE3844A8625B0002222CE795F85F7011
:10D6800095F85E202E6202333044B64452EA0722F7
:10D69000AB616862C5F82CE07FF462AE002C7FF4C9
:10D6A0005FAEB5F8627095F8610095F860209B0058
:10D6B00040EA072003F2FF1342EA0022B1EB532FA6
:10D6C000AA62FFF44DAE95F8651095F8643043EA10
:10D6D00001234FF0FF328021012B2A61EA6029717A
:10D6E0000AD0032203E70220FFF7A2F9002849D05D
:10D6F0000223BB63FFF794BA711C2846FEF730FF84
:10D700000028EED195F8332295F832322C7143EA95
:10D7100002234AF655229342E3D1E88E95F835204C
:10D7200095F83430224942EA002243EA02238B4230
:10D73000D7D1B5F81A0295F8192295F8183201F1E7
:10D74000FF5101F5005142EA0022203143EA022351
:10D750008B42C6D1B5F81E6295F81D02B5F822427B
:10D7600095F8211295F81C2295F8203240EA0620FF
:10D7700041EA042142EA002243EA01232A61EB60E4
:10D780000322B4E62020FFF753F918B12023BB632E
:10D79000FFF746BA4FF40070FFF74AF900283FF44C
:10D7A00092AD4FF40073BB63FFF73ABA002C01400F
:10D7B0005252614143695869704700BFC368586954
:10D7C0009B691840704700BFC368586900F00100AA
:10D7D000704700BF00EB81014FF00043D1F890206B
:10D7E000012060F3DC431361D1F89020136800201E
:10D7F00043F0004360F39E731360704700EB8101B8
:10D8000086B0D1F89020136843F0404359030AD5FD
:10D8100041690969C1F3074109B96FF3DF7300205A
:10D82000136006B07047C168C96AC1F30741002997
:10D83000F3D00020136006B0704700BFF0B54C0174
:10D84000051987B0D5F8BC330022D3B1B5F8B2635F
:10D85000013B3344B3FBF6F39BB2B3F5807F64D94D
:10D860003602C5F8BC6305194FF4807795F8AE63AE
:10D870003B466EB1B5F8B26303FB06F3C5F8BC33A3
:10D8800008E001273B46051995F8AE63002EF1D15B
:10D89000D5F8BC3301F1150600EB461500EB81010C
:10D8A00063F3120295F814E1D1F8903067F3DC428B
:10D8B0006EF35E721A61C378012B39D0D1F89050A3
:10D8C00042692B68926802F0010282F0010262F361
:10D8D0005D7343F000436FF39E732B60C3780BBB03
:10D8E000021992F8AE33EBB9D2F8BC33D3B192F847
:10D8F000B123032A2BD8DFE802F02102210242697A
:10D9000015690195DA1CADB2C2F38F0295421ED2A1
:10D91000C268936943F0806393610444C278D4F889
:10D92000BC33A2B1002007B0F0BDC3F30907AAE7DA
:10D93000D1F89030D5F818215A61BFE7C768FD6A61
:10D940000395DA1CADB2C2F38F02954211D300EBFE
:10D950004610D1F8D040D0F8182198B2033080108A
:10D96000E0D00023013352F8041B21609842F9D122
:10D97000D8E7BB6943F02003BB610444C278D4F804
:10D98000BC33002ACED1E2E7F0B400EB81054FF0C2
:10D99000FF34D5F890204B019460C418C27894F8F5
:10D9A000B163012A14BF002404240022032E13D8DB
:10D9B000DFE806F002550249C61844F4936496F86D
:10D9C000AE7344F00104002F46D196F8B06344F0E2
:10D9D00040040EB144F02004D5F89060F46047692B
:10D9E0000126BC6906FA01F12143B961C468A16945
:10D9F000184441F00073A36190F8AC7390F8AF3312
:10DA000090F8AD6390F8AE4390F8B113B0F8B2035C
:10DA100067F39C52A3F1020366F3CE22B3FA83F3B9
:10DA200064F3CF325B0963F3514261F3934260F3D5
:10DA30000A02D5F89030032908BF42F000521A605C
:10DA40000020F0BC7047C61844F4D36496F8AE6367
:10DA500044F00104002EBFD044F48074BCE7C61823
:10DA600044F4087496F8AE6344F00104002EB3D079
:10DA700044F4C074B0E700BF4269136861F3010366
:10DA80001360704730B403329210D0F8D05009D0F0
:10DA90000846002301332C6840F8044B9A42F9D120
:10DAA00001EB8201084630BC704700BF30B4C47837
:10DAB0006CB900EB820003339B10D0F8D05006D035
:10DAC0002246013251F8040B28609342F9D100201C
:10DAD00030BC7047094A0A4B02FB00F0A3FB00234D
:10DAE000C21A82B003EB5202002392080193019BF9
:10DAF00001339A420193FAD202B07047C0D40100B8
:10DB00002549922410B504460A20D4F8CC20136885
:10DB10006FF382036FF341036FF3C3036FF3451396
:10DB200043F480711160FFF7D5FFD4F8CC306FF368
:10DB3000082119601420FFF7CDFF012010BD00BFA0
:10DB40002DE9F843044601F047FF1D4B1B78012BDC
:10DB500010D01C4A1178994218BF13701A4B1A68DA
:10DB60000AB9BDE8F88319494020002208831A60E9
:10DB7000BDE8F883144A1168E1B1154E154D3168BE
:10DB8000DFF85880144FA9462B688B4203F101023D
:10DB9000E7D0202A38F8130008D0C9F800200CB1CB
:10DBA0003860F1E701F0F6FA3168EDE70023C9F8D3
:10DBB0000030F4E70549402048831360DDE700BFEB
:10DBC00034BD0120900000203425002000000240D8
:10DBD000C8BD01204C25002040250020ECBC0120C0
:10DBE000F8B505465C1A0F46164619463846531BCB
:10DBF000013403FB044401F051FE3146284601F094
:10DC000039FE4FF0C0432C221A803CB10449BDF8C4
:10DC10001820002301339C420A80FBD1F8BD00BFCD
:10DC20000000086010B5044C206818B105F0A0FD94
:10DC30000023236010BD00BF3825002070B5436865
:10DC4000013B002B04460E46436010DB0268511C6A
:10DC500001601578013B002B636012DB23685A1CBE
:10DC60002260187845EA00253580012070BD0A4BF6
:10DC70000146186806F0AEFC421C05460AD1002099
:10DC800070BD054B2146186806F0A4FC431CE9D181
:10DC9000002070BD6368DDE72401002010B54368F3
:10DCA000013B002B0C46436006DB03685A1C0260F4
:10DCB00018782070012010BD044B0146186806F04A
:10DCC00089FC431CF5D1002010BD00BF24010020B9
:10DCD00030B5C3B00DF106010446FFF7AFFF10B930
:10DCE000002043B030BD0DF103012046FFF7D6FF01
:10DCF0000028F5D09DF803300025C3B10DF10501D2
:10DD00002046FFF7CBFF013501A90028E8D02046C7
:10DD1000FFF7C4FF234601210028E1D09DF804202D
:10DD200002A805F0A7FF9DF80330AB42E6DC012016
:10DD3000D7E700BF2DE9F04F85B00F460DF10E017A
:10DD4000904600939DF838600546FFF7A7FF00282E
:10DD50005CD00F9B9DF80EA09C1EBAF1000F59D10C
:10DD6000002E40F08E800DF10F067CB3B94601976E
:10DD7000009FD3460DF10F0631462846FFF78EFF70
:10DD80000BF1010109F10102002840D0D8451FFA2A
:10DD900081FB12D98FB1B9F5804FC9F38F30C9F328
:10DDA0000D010AD3B9F5B64FC0F099806A4B9DF8C2
:10DDB0000FE053F8200000F801E09DF80F105C45DB
:10DDC0001FFA82F98AEA010AD6D8019F6249B80B84
:10DDD000C7F30D0251F82000825C002A00F0858014
:10DDE000012431462846FFF759FF78B19DF80F20EE
:10DDF000524572D0594C5A4823682322DB680121CE
:10DE000007F052FA2368D86805F06CFD002005B0D1
:10DE1000BDE8F08F002E49D00DF10F06002CDFD0A9
:10DE20004FF0000B0DF10F064FF001093146284667
:10DE3000FFF734FF0BF101017A1C0028E7D0D84529
:10DE40001FFA81FB15D9009B9BB1B7F5804F4FEAB4
:10DE50009730C7F30D010CD3B7F5B64F38BF414B20
:10DE60009DF80F7038BF83F800903B4B53F82000AB
:10DE700047549DF80F105C4597B28AEA010AD5D83D
:10DE8000AEE7002C60D057460DF10F0605E09DF877
:10DE90000F30BC428AEA030A1DD931462846FFF7F3
:10DEA000FDFE0137BFB20028F1D1AFE7002C48D00A
:10DEB00037460DF10F0605E09DF80F30BC428AEAA7
:10DEC000030A08D931462846FFF7E8FE0137BFB2FA
:10DED0000028F1D19AE7002483E7204697E7214BF9
:10DEE0004FF0010E83F800E060E71F4A92F88020AF
:10DEF000002A7FF475AF43F6F272974228DD45F6AB
:10DF0000F222974202DC174A0120107007F10D023D
:10DF10009013C2F30D0251F8204045F6F1204FF066
:10DF2000000E874204F802E002DC0E4A0120107065
:10DF30000E37BA13C7F30D0751F822208021D155AF
:10DF40004EE70DF10F064CE754460DF10F0648E77A
:10DF50007FF446AFE9E700BF0CB7012024010020A1
:10DF6000286501089100002038B701203F49404B47
:10DF7000D1F888203F4842F47002C1F888201A681E
:10DF8000002142F001021A6099601A6822F084723E
:10DF900022F480321A6058601A6882B022F480221B
:10DFA0001A60D960009101911A6842F480321A60B7
:10DFB00003E0009AB2F5C06F09D01A6802F400328B
:10DFC0000192009A01320092019A002AF1D0284B66
:10DFD0001B6813F4003318BF01230193019B012B2D
:10DFE00000D0FEE7224B24491A6C42F080521A649A
:10DFF0000A6842F480420A609A689A609A6842F419
:10E0000000429A609A6842F4A0529A601A6822F01C
:10E0100080721A601968164A8801FBD4174B536046
:10E02000136843F0807313601168114B8901FBD5AD
:10E03000134A40F205711160126802F00702052AC6
:10E0400000D0FEE79A6822F003029A609A6842F0D4
:10E0500002029A609A6802F00C02082AFAD1034B75
:10E060004FF000629A6002B0704700BF00ED00E020
:10E07000003802401030002400700040042A40079D
:10E08000003C0240054B1A6812F0C05F05D00449FD
:10E0900001204FF0046208609A60704700640240FB
:10E0A0004825002038B54FF48070FEF7C1FC38BB1E
:10E0B0000220FEF7BDFCA8B90820FEF7B9FC002835
:10E0C00030D12020FEF7B4FC28BB1020FEF7B0FCB6
:10E0D00000282ED14FF40070FEF7AAFC00282FD1A3
:10E0E0001B4904E01B4A1A49022393630B70194A27
:10E0F000D36B23F4434323F03A03D3630B7838BD47
:10E1000013491448144B00254FF4807401220D70FC
:10E1100084631A60EBE70F4A0D49202006239063C1
:10E120000B70E4E70B4A0A490820042390630B7044
:10E13000DDE7084A06491020052390630B70D6E7F7
:10E14000044A03494FF40070072390630B70CEE735
:10E1500044250020002C01403C2500200A4A536B36
:10E1600013F0450FFBD05A0709D413F00100064BFA
:10E1700015BF012040F2FF5298639A637047024B2B
:10E1800004229A6303207047002C014008B5384AE6
:10E19000536B13F0450FFBD059070DD413F0010357
:10E1A00006D133490A69D2B290420AD0102008BD84
:10E1B0002F4B0120986308BD2D4B04229A63032046
:10E1C00008BD40F2FF5218468A63FEF73BFC294B1C
:10E1D00003402BB1002805DB420005D5092008BD0E
:10E1E000184608BD1C2008BD830001D50A2008BDC3
:10E1F000C10001D50B2008BD020101D50C2008BDCE
:10E20000430101D50D2008BDC10101D50E2008BD77
:10E21000020201D50F2008BD4302C7D4810201D5F7
:10E22000112008BDC20201D5122008BD030301D58B
:10E23000132008BD410301D5142008BD820301D578
:10E24000152008BDC30301D5162008BD010401D562
:10E25000172008BD420401D5182008BD830401D54C
:10E26000192008BD10F0080F0CBF00201A2008BDAF
:10E27000002C014008E0FFFD10B5094B40200022B2
:10E280000C244FF4806198605C6019611A60DA6058
:10E2900004F094FE2046BDE81040FFF777BF00BFB2
:10E2A000D0BD012038B50F4A0F4B12680020120470
:10E2B0004FF480610D244025D8601A609D6019617B
:10E2C0005C6004F07BFE2046FFF760FF08B102208F
:10E2D00038BDFEF7B7FBC0F34320043818BF012058
:10E2E00038BD00BF30250020D0BD012080B586B0EC
:10E2F00000AF786000237B6100233B617868FFF703
:10E3000059FA0346FB6000237B612AE0BB891A4669
:10E310007B6942FA03F303F00103002B1ED07A68F5
:10E320007B6922339B0013449B681B68BB607B7A2C
:10E3300023F07F03DBB2002B08D07969786802F004
:10E34000E1FA02463B6913433B6107E0796978686B
:10E3500002F0B2FD02463B6913433B617B69013326
:10E360007B617B681B781A467B699A42CED83B69F1
:10E3700018461837BD4680BD80B584B000AF7860C0
:10E380000023FB600023BB607868FFF71DFA03469B
:10E39000002B71D07868FFF711FA0346BB60BB68A9
:10E3A000002B01D1002368E03B7A03F00803DBB2C5
:10E3B000002B06D0786803F07FFA0246FB6813430F
:10E3C000FB603B7A03F01003DBB2002B06D07868C9
:10E3D00002F0CCF90246FB681343FB603B7A03F082
:10E3E0002003DBB2002B06D0786803F087F90246E1
:10E3F000FB681343FB60FB7A03F00403DBB2002BE2
:10E4000006D0786803F0B6F80246FB681343FB6059
:10E41000FB7A03F00203DBB2002B06D07868FFF72B
:10E4200065FF0246FB681343FB60FB7A03F00103C0
:10E43000DBB2002B06D0786802F0E8FF0246FB68EA
:10E440001343FB60FB7A03F02003DBB2002B06D002
:10E45000786803F017FA0246FB681343FB60BB7A47
:10E4600003F02003DBB2002B06D0786802F056F9E7
:10E470000246FB681343FB60FB6818461037BD4635
:10E4800080BD00BF0148FFF777BF00BFE4BD01209A
:10E49000104B114A18681168890600D47047C106EC
:10E4A000FCD510B420210D48916002880C490D4C18
:10E4B00092B242F4007202801A6822F001021A60DD
:10E4C0000B6823F001030B60002222605DF8044B0F
:10E4D000704700BF106002400060024000540040DE
:10E4E000A0600240DC360020094A0A4B11685A68D5
:10E4F000900201D5CA0600D47047074A4FF40011B4
:10E50000D96013889BB243F400731380704700BF37
:10E51000A0600240006002400054004038B52B4C1F
:10E520002368012B00D038BD294804F029FD0128BB
:10E5300009D1284B1B7813B3274B284A1B6803F0DB
:10E54000FE03138238BD254D254AAB8A288B9BB22A
:10E5500043EA004311461A408A4218D0214804F089
:10E560000FFD0028DFD01B4B1A78002ADBD01E4A93
:10E57000127802F0FF01A2B10023236038BD164BD0
:10E58000164A1B6843F00103DBB2138238BD114BFE
:10E590001B78002BC7D0154A136843F001031360A2
:10E5A00038BD1348026842F001020260AA8892B2A4
:10E5B00042F480524FF6FB70AA801970A8822B8813
:10E5C0009BB243F480732B8038BD00BFDC36002043
:10E5D00001000010C2360020CC360020005400405C
:10E5E0008200070004000010C8360020A06002402E
:10E5F0001060024002288CBF00200120704700BF3D
:10E60000022838B51ADD0338072817DC124C4FF4FE
:10E610000B7505FB0040D0F82842E3070ED5012A10
:10E620000B4614D0022A0FD062B903F0F1FE48B1B4
:10E6300005F032F84FF4FA63036003E005F02CF8BC
:10E6400009230360002038BDC1681944EDE7416922
:10E65000194403F0DDFEEAE75425002000286AD0C3
:10E66000F0B5012883B00C46154624D002284BD0C3
:10E670000338072862DC3A4B4FF40B7606FB003672
:10E68000D6F82832DB0759D50027B5F5007F5ADDCB
:10E6900001AB4FF400722146304603F075FF50BBCA
:10E6A000019BB3F5007FA5EB03051C441F44ECD28E
:10E6B000384603B0F0BD002A1ADD2A4E8F1806E056
:10E6C000FEF762F914F8013B3360A74210D02078BE
:10E6D0000A28F5D133680D2BF2D00D20FEF754F93E
:10E6E0002078FEF751F914F8013B3360A742EED1D0
:10E6F000284603B0F0BD04F0CFFF4FF4FA63036087
:10E700004FF0FF3003B0F0BD002AF1DD164E8F1838
:10E7100006E0FEF739F914F8013B3360BC42E7D05C
:10E7200020780A28F5D133680D2BF2D00D20FEF7A2
:10E730002BF92078EDE74FF0FF30704704F0ACFF85
:10E7400009230360DCE7002DB2DD2A46214630466E
:10E7500001AB03F019FF0028CDD1019B1F44A7E7AF
:10E7600054250020B436002050250020022834DD36
:10E77000F0B50338072883B02ADC204B4FF40B7721
:10E7800007FB0037D7F82832DB0721D50C461546A2
:10E790000026B5F5007F23DD01AB4FF40072214662
:10E7A000384603F0BDFF50B9019BB3F5007FA5EBE0
:10E7B00003051C441E44ECD2304603B0F0BD04F007
:10E7C0006BFF4FF4FA6303604FF0FF3003B0F0BD0E
:10E7D00004F062FF09230360F6E74FF0FF30704753
:10E7E000002DE9DD2A462146384601AB03F098FFAB
:10E7F0000028E4D1019B1E44DEE700BF5425002021
:10E800002DE9F043022883B040F39880C41E072C02
:10E8100000F394804FF40B75794F05FB04F57E19D6
:10E82000D6F82832D90740F1898001A9304603F093
:10E83000D3FD002850D1337C5A0663D51B066DD416
:10E840004FF40B7505FB04F507EB05080198D8F8A4
:10E850002010DFF8AC91FDF783FE00283CD1D8F8FA
:10E860002430DA7A42F02002DA72D8F8082059F817
:10E8700005109A76C2F30720D876097803296AD062
:10E880004FF40B7202FB0472CB21D2681A77100A84
:10E890005877100C120E9877DA7799750022B22506
:10E8A000422050219A74DA74DD7518765976019BEE
:10E8B0000122DA70019DEB78002B46D12B78032BD7
:10E8C0004ED06B78022B15D94FF40B7303FB0473F6
:10E8D0001A7C22F040021A744FF40B7000FB04748F
:10E8E0000020D4F8283223F00103C4F8283203B002
:10E8F000BDE8F0834FF40B7303FB04731A7C22F022
:10E9000040021A7401A9304603F066FD0028E3D1E5
:10E910004FF40B7303FB04F3F850DDE7019BF2693E
:10E92000587805F1280139440123FDF71FFB002821
:10E93000D2D1337C03F07F03337481E704F0ACFE63
:10E94000092303604FF0FF30D1E7284603F018FD9C
:10E950000028B9D1B2E7120C110A1A7559758FE760
:10E960002B79012BADD105F134010B4605F50D7066
:10E97000002203F8012B83424FF00008F9D12869E7
:10E98000EB6885F81C024FEA102E85F81DE24FEA6D
:10E99000104E000E2A6A85F81EE285F81F024FEA23
:10E9A000132E180C85F820321B0E85F821E285F80D
:10E9B00022024FF0550EAA2085F82332522301324D
:10E9C00085F832E285F833024FF0610E412085F878
:10E9D000343085F83530722385F8370085F81A020F
:10E9E00085F8183285F819322A6385F836E085F8FB
:10E9F0001BE201236878FDF7B9FA85F8048060E727
:10EA0000542500200EB42DE9F04F8EB0179B03F073
:10EA10000302012A43D0022A35D032B14FF0FF3031
:10EA20000EB0BDE8F04F03B070470126AB4D07466E
:10EA300000242B46D3F8282212F0010F03F50B73A4
:10EA40000DD00134082CF5D104F026FE1723036005
:10EA50004FF0FF300EB0BDE8F04F03B070473246C4
:10EA600001A968460097FEF7C1F800282FD04FF49F
:10EA70000B7000FB04F400232B5104F00DFE4FF447
:10EA8000FA630360CAE79C051BD413F4806F0CBFC4
:10EA900003260B2613F0080F18BF3326C6E79D0583
:10EAA00009D413F4806F0CBF02260A2613F0080F56
:10EAB00018BF3226BAE713F4806F0CBF12260A265D
:10EAC000F4E713F4806F0CBF13260B26E2E79DE8F2
:10EAD0000A0002A80293FDF7ABFD002871D19DF951
:10EAE0003330002BC3DB16F01C0F00F0D7809DF8ED
:10EAF0000E3013F0110FBAD1300700F1F180DDF8BC
:10EB000004E0DEF83010099B4FF40B7202FB045254
:10EB1000116253629EF80000D97E9A7E032842EA71
:10EB2000012100F0D3804FF40B7202FB04F2A8180D
:10EB300002F128078160597FB3F81EC01B7F45F89A
:10EB400002E041EA0C2243EA0223C360BEF8063029
:10EB5000838000222F44067407F500713B464274FF
:10EB6000C261426103F8012B8B42FBD1B10640F137
:10EB700085804FF40B7909FB04F905EB0903DE6886
:10EB8000002E7BD05E61BEF80A8099684FEA482863
:10EB900046454DD9C8EB060602E0464548D91E4613
:10EBA00055F8090003F0FCFA01280146C8EB0603FA
:10EBB00001D9421CF1D14FF40B7303FB045399614B
:10EBC00055E716F01C0F3FF452AF04287FF44FAF07
:10EBD00002A8029F04F026FA00287FF448AF0899A3
:10EBE0003846FDF7BDFC00287FF441AF099B1B7838
:10EBF000E52B03D0012102A8002B62D108993846E9
:10EC0000FDF7AEFC00287FF432AF099B024603F10A
:10EC1000200103F8012B8B42FBD10B220AA9099892
:10EC200003F0D0FB46F008060123F6B2FB7063E761
:10EC30004FF40B7000FB0450C6F308038161EBB185
:10EC4000DDF804E0DEF818300239023B9942BFF4E7
:10EC50000EAFBEF80A30DEF82C2001FB0322002A9A
:10EC60003FF405AF02EB5622C2619EF8010039461F
:10EC70000123FDF75DFB00287FF4F9AE4FF40B7321
:10EC800003FB0453E01CD3F8282242F00102C3F82E
:10EC900028220EB0BDE8F04F03B070479DF80E304B
:10ECA000D9063FF5E4AEB20702D5DF073FF5DFAE88
:10ECB0003007DDF804E07FF524AF46F04006F6B2F9
:10ECC0001FE7FDF797FA002889D0D0E6587D1A7D16
:10ECD00042EA002241EA024125E700BF5425002014
:10ECE0000199099B0A78DF7E987E032A40EA07276C
:10ECF00070D0CB229A73422050224FF0B20E5A7439
:10ED000083F80FE01874099B2022DA72099B002215
:10ED10009A76DA760878032804BF1A755A75099B23
:10ED2000002201201A775A779A77DA77C87017B9D4
:10ED3000DDF804E0C1E7012F7FF699AEDDF8088029
:10ED4000D8F818309F42BFF492AE019B4046D3F8EA
:10ED500030B0B9462BE001283FF489AEB0F1FF3F57
:10ED60003FF485AEB9F1010F7FF681AED8F81830C7
:10ED70009945BFF47CAE49460022404603F072FA42
:10ED800000287FF474AED8F81810D8F810308A1E16
:10ED9000934208D298F80420013342F00102C8F8E7
:10EDA000103088F804208A4507D20298D146494697
:10EDB00003F0F6F982460028CDD159460198FDF7B7
:10EDC000CFFBDDF804E0013FCEF80C7000283FF4E3
:10EDD00074AF4CE6587D1A7D42EA002247EA0247AA
:10EDE00087E700BF2DE9F04F85B00C46039101780D
:10EDF00002900093002944D002F10803224D0193B0
:10EE000004F10C060198EF2EA0F1080730D8B0F5F8
:10EE1000A07F2DD21D4BDDF80CB00C2202FB01327D
:10EE200002F1FF3A00F1FF394FF0C0485946584609
:10EE30001AF8014F00F032FD3846494600F01AFD3D
:10EE40002C23A8F80030BDF838C0BDF800E0072337
:10EE5000012000FA03F2224214BFA5F800E0A5F851
:10EE600000C013F1FF33F4D20BF1010BB345DDD138
:10EE7000029B13F8011F0293019B083301930029A1
:10EE8000C0D105B0BDE8F08F000008604C650108F6
:10EE900010B4A44CFF2323706370C30511D5B0F5E3
:10EEA000B97F44D024D8B0F58A7F3DD040F26B13AF
:10EEB000984203D100223423227063705DF8044B22
:10EEC00070477F28FAD8984B1B78EBB9974B03EB28
:10EED000400213F810305278D9071DD50023237053
:10EEE000FF2A18BF0123E9D0E2545DF8044B7047B4
:10EEF000B0F5BA7F20D040F275139842DED10022DF
:10EF0000432322706370D9E7894B03EB400213F867
:10EF100010305278D907E1D403F0020303F0FF0167
:10EF20007BB171232370DBE771232370C6E70022D6
:10EF3000442322706370C1E7002242232270637071
:10EF4000BCE7FF2A40F0078169381428B6D801A32E
:10EF500053F820F013F00008BDEE000837F0000869
:10EF600001F00008BDEE0008BDEE0008BDEE00088F
:10EF700025F00008BDEE0008EFEF0008EFEF0008F5
:10EF8000DDEF0008CBEF0008BDEE0008BDEE000885
:10EF9000BDEE0008BDEE0008B9EF0008BDEE0008A8
:10EFA000BDEE0008A9EF0008624B1B78032B85D843
:10EFB000DFE803F0AEA9A49F5E4B1B78032B3FF65E
:10EFC0007DAFDFE803F0918C87825A4B1B78032BCF
:10EFD0003FF674AFDFE803F041535956554B1B78A9
:10EFE000032B3FF66BAFDFE803F03538476D514B2D
:10EFF0001B78032B3FF662AFDFE803F0292C613565
:10F000004C4B1B78032B3FF659AFDFE803F0504B16
:10F010004641484B1B78032B3FF650AFDFE803F027
:10F0200096918C7D434B1B78032B3FF647AFDFE86F
:10F0300003F00B0B17433F4B1B78032B3FF63EAF00
:10F04000DFE803F00E0517144023237036E744234E
:10F05000237033E74223237030E7432323702DE7E7
:10F06000342323702AE78223237027E78123237028
:10F0700024E73023237021E7312323701EE7412347
:10F0800023701BE78323237018E73323237015E7CE
:10F09000812283232270637010E730223323227091
:10F0A00063700BE7442241232270637006E7342229
:10F0B00043232270637001E784232370FEE632232A
:10F0C0002370FBE680232370F8E6802282232270DF
:10F0D0006370F3E64322422322706370EEE631222E
:10F0E000322322706370E9E6422244232270637067
:10F0F000E4E68022832322706370DFE6312233232B
:10F1000022706370DAE64322412322706370D5E6F1
:10F110004222432322706370D0E681228223227030
:10F120006370CBE6C0360020D43600204C72010854
:10F130004C710108C000002030223223227063701D
:10F14000BCE64422422322706370B7E63422442393
:10F1500022706370B2E60B46E254C6E64FF080437D
:10F160004FF6FE7208481A82084903680A6801339C
:10F170000132B3F57A7F0A6003D1054A01210023E9
:10F1800011600360704700BFD83600205401002092
:10F190005C22002000F4007292B210B5C2B9592866
:10F1A0002AD00D2837D005283BD0062848D004287F
:10F1B0002DD0294CFFF76CFE2078FF2812D001F0EB
:10F1C0005FF86078FF280DD0BDE8104001F058B816
:10F1D000C0F30800592813D01F4CFFF759FE2078C0
:10F1E000FF2800D110BD01F02DF86078FF28F9D07C
:10F1F000BDE8104001F026B8184B01221A7010BD6E
:10F20000002001F01FF8154B00221A7010BDBDE858
:10F21000104003F091BD1249124B012008601A7092
:10F2200010BD114991F8C9300133DBB2042B14BF72
:10F2300081F8C93081F8C920BDE8104000F0B6BFA0
:10F24000094991F8C8300133DBB2022B14BF81F8B1
:10F25000C83081F8C820EFE7C0360020D43600203F
:10F2600034B801207800002038B701202DE9F041A2
:10F27000214C236882B01BB1002002B0BDE8F081B0
:10F280001E4E3368002BF7D11D4A4FF40030137027
:10F2900003F076FE07460028EED1DFF88080D8F82C
:10F2A0000030012BE8D001251F2301A88DF8043080
:10F2B0008DF805708DF806708DF80750FDF76EFC1F
:10F2C000104B1149114A12484FF0A40EC3F800E048
:10F2D000104BC8F800500D70177006210E4A45609B
:10F2E000596013889BB243F48073284613803560BD
:10F2F000256002B0BDE8F0812CB80120C4360020A2
:10F3000060220020CC360020C2360020C836002003
:10F31000A06002401060024000540040DC36002033
:10F320002DE9F8439D4C2368012B02D00020BDE855
:10F33000F8839B4B1A68012AF8D19A4A1268002A6E
:10F34000F4D1994D2A68022A00F096819749984A8B
:10F350004E790F7849785170D1881770B7074CBF34
:10F3600021F4807141F4807189B2F607D1804CBFDD
:10F3700021F0800141F08001D1800021196020B985
:10F38000002323600120BDE8F8832B68022B13784B
:10F3900000F0AF80A02B00F2A680602B34BF0425C4
:10F3A00000255378A02B40F2998045F00105D388C1
:10F3B0001E0648BF45F01005D80500F196807D4F28
:10F3C0003E68AE42DCD06E4071070DD57A4B6A07BD
:10F3D0001B7840F10C81032B06D8DFE803F07B6B30
:10F3E0006702812000F04CFF33070DD5724B2807D0
:10F3F0001B7840F1E580032B06D8DFE803F0676354
:10F400005F02802000F03CFFF1070DD56A4BEA0750
:10F410001B7840F11A81032B06D8DFE803F03B4349
:10F420003F02832000F02CFFB3070DD5624BA807E5
:10F430001B7840F1F380032B06D8DFE803F0271F89
:10F440001B02822000F01CFFF1060DD55A4BEA0684
:10F450001B7840F19080032B06D8DFE803F002020E
:10F460001307402000F00CFF3D6089E7842000F086
:10F4700007FFF9E7322000F003FFE5E7422000F044
:10F48000FFFEE1E7342000F0FBFEEDE7442000F052
:10F49000F7FED9E7432000F0F3FEC5E7332000F084
:10F4A000EFFEC1E7412000F0EBFEBDE7302000F0A9
:10F4B000E7FE99E7442000F0E3FE95E7312000F0F5
:10F4C000DFFEA1E7432000F0DBFE9DE7422000F0D5
:10F4D000D7FE99E7342000F0D3FE85E75F2B98BF75
:10F4E00045F0020563E708255BE7344B00221A70FC
:10F4F00065E7282B00F2F380182B34BF04250D4656
:10F5000053782B49282B32D8172B40F2EA8085BB41
:10F510008B78142B00F2EB800B2B8CBF002504257D
:10F52000D3782349142B22D80B2B40F2DA80CE88D3
:10F5300065B9B70700F1E28016F4004F0CBF002553
:10F540000825F00740F1D58045F0010542F2FC2383
:10F5500033400BB145F01005F20400F1C5803305CE
:10F56000C3D477057FF52BAF03F0F2FB27E745F017
:10F570000105D688EAE7032B3FF676AFDFE803F014
:10F5800002020A06402000F05DFE6DE7842000F0D4
:10F5900059FE69E7342000F055FE65E72CB80120DC
:10F5A000C4360020DC36002030B801203C1E00208C
:10F5B000B8360020D0360020C0000020780000209F
:10F5C000032B3FF621AFDFE803F00E0A060280208E
:10F5D00000F038FE18E7312000F034FE14E7432035
:10F5E00000F030FE10E7422000F02CFE0CE7032B69
:10F5F0003FF6FAAEDFE803F00E0A0602812000F0C3
:10F6000021FEF1E6302000F01DFEEDE6442000F082
:10F6100019FEE9E6342000F015FEE5E6032B3FF67F
:10F6200013AFDFE803F00E0A0602822000F00AFEA4
:10F630000AE7322000F006FE06E7422000F002FE54
:10F6400002E7442000F0FEFDFEE6032B3FF6ECAEA1
:10F65000DFE803F00E0A0602832000F0F3FDE3E684
:10F66000332000F0EFFDDFE6412000F0EBFDDBE6AC
:10F67000432000F0E7FDD7E6214E224A96F800C06D
:10F6800096F801E0B77896F804904FEAEC084FEA54
:10F690006E1108F0180801F0060148EA01010CF0AB
:10F6A0003F0C96F80380767982F800C04FEAA70CE9
:10F6B00008F0070846EA09260CF0180C41EAD711B1
:10F6C0000EF03F0EF64307F01F074CEA080C82F8D5
:10F6D00001E09170D77082F804C0D6804DE608250D
:10F6E0000EE745F0020544E703F026FB37E708255F
:10F6F00016E7710448BF45F0020527E7042520E717
:10F700003C1E0020B8360020104A1378A02B02D9E6
:10F710004FF4BA7070475F2B02D840F26B107047FD
:10F720005378A02B02D940F2751070475F2B02D896
:10F730004FF4B9707047D3881A0601D55A20704724
:10F7400013F4807F0CBF002076207047B83600206D
:10F7500010B5304A304C13680133022B13601FD9A7
:10F7600023782D4A282B0CD8172B13D8A3782A4A94
:10F77000142B40F26B100AD80B2B2CD840F26B10D4
:10F7800010BD4FF4BA70A378234A142BF4D94FF468
:10F79000BA7010BD5378282B17D940F27510F2E7D4
:10F7A00021781E48FDF716F961781D48FDF712F91A
:10F7B000A1781C48FDF70EF9E1781B48FDF70AF91E
:10F7C000E1881A48FDF706F9CAE7172B8CBF00201D
:10F7D0004FF4B970D7E7D378142B02D940F27510E3
:10F7E00010BD0B2B02D84FF4B97010BDD3889A0707
:10F7F000C4D41C04CBD4D907F0D45A04F3D442F2B5
:10F80000FC221A400AB15A2010BD13F4E05F18BF61
:10F81000762010BDE0360020B83600204C73010879
:10F82000547301085C730108647301086C73010868
:10F830000E4B1A6812F0010F14BF002308231007A3
:10F8400044BF43F02003DBB2910758BF43F04003AD
:10F85000520748BF43F080034FF0C04204483621AE
:10F860009BB2118003801180704700BFEC360020EE
:10F870000000086070B4084B4FF0C045C0F30F247F
:10F880002B26C1F30F22C0B2C9B22E801C80188073
:10F890001A80198070BC70470000086070B4084B73
:10F8A0004FF0C045C0F30F242A26C1F30F22C0B287
:10F8B000C9B22E801C8018801A80198070BC7047D5
:10F8C00000000860F0B585B003F04EFB304D314BC1
:10F8D000AC881E686846FDF7C1F8029A2E482F4B87
:10F8E000A0FB021024F03F042404800C240C87B2F7
:10F8F0003C43AC80298821F001010904090C9E4297
:10F90000298029D87300B2FBF3F39BB2032B07F1D4
:10F91000010798BF04232F841D4A938313889BB249
:10F9200043F001031380138823F4816323F002035F
:10F930001B041B0C43F480634FF48041138011813E
:10F9400093889BB243F40073938013889BB243F077
:10F950000103138005B0F0BD06EB4603B2FBF3F3E1
:10F960009BB2C3F30B020AB943F001034FF4967143
:10F970000B4C074D01FB00F284FB0201D217C2EBD6
:10F98000A112013292B243F400432A84C4E700BFBB
:10F99000005400406822002083DE1B43A086010043
:10F9A000D34D621008B50B4A13889BB243F4007321
:10F9B000138013886FEA43436FEA53439BB213806B
:10F9C0001388C3F30E03138003F0CEFABDE808409A
:10F9D000FFF778BF005400402DE9F04194B00223B6
:10F9E000AD4D8DF80F30D5F81023AC4C2ABB2278E2
:10F9F000002A3FD09A4200D02370D4F880301B698F
:10FA0000984703F0C1FBD4F880305B689847E36FF8
:10FA1000A3495B68A04898470023A5F89035A5F84E
:10FA20009235A5F89435A5F89635A5F89835A5F83A
:10FA30009A35237014B0BDE8F08123780A2BF9D8E9
:10FA400001A252F823F000BF75FA0008D1FA0008AD
:10FA5000FBF9000835FA00084DFB00086DFB0008B3
:10FA600089FB0008ABFA000889FA000835FA00089B
:10FA7000A5FB0008D5F81033002BDBD00123642050
:10FA80002370FEF727F8D5E7D4F88030834C9B6BC2
:10FA900098470128CED1E36F7F481B6821469847DD
:10FAA0000028C7D105232370C4E7237F0022013B30
:10FAB000A2740A2BBED8DFE813F0C7010402E501E7
:10FAC000620236027A021902AB018C017A016D01E1
:10FAD000D4F880309B68984700216F4800F062FDA1
:10FAE000802160716C4800F05DFD20716A48FEF76E
:10FAF00009F8D4F88030DB689847D5F8CC20D4F8E2
:10FB000080301068C0F3414084F821000422227044
:10FB100000F003009B6998470025A07994F82130F4
:10FB200094F820202179019000955B4800F054FD65
:10FB3000A079019094F8213094F820206179009503
:10FB4000554800F049FD14B0BDE8F081A378092BB9
:10FB50003FF670AFDFE813F0F500E700AF00A60056
:10FB6000770063004F003B008B003400E36F4B4C89
:10FB70009B684948214698478DF80F009DF80F3043
:10FB80004BB90623237055E7E36F4449DB684248CD
:10FB900098478DF80F009DF80F0003F025FB14B077
:10FBA000BDE8F08103F0F0FAD4F880305B68984744
:10FBB000E36F3B495B683848984714B0BDE8F08173
:10FBC000D4F880305B6B98470823237032E794F8B1
:10FBD0003200324C002800F0178204A903F01CFB0D
:10FBE00000287FF427AFD4F8803004A81B6B984717
:10FBF0000823A3701EE794F83100284C002800F079
:10FC0000F38104A903F008FB00287FF413AFD4F8B4
:10FC1000803004A8DB6A98470723A3700AE794F8AA
:10FC200030001E4C002800F0E78104A903F0F4FA2C
:10FC300000287FF4FFAED4F8803004A89B6A984770
:10FC40000623A370F6E6E08E144C03F01DFB00289B
:10FC50007FF4F0AED4F8803004F150025B6A04F116
:10FC60003E0104F1340098470523A370E2E60B4EF1
:10FC700094F83930E3820025092707482575314675
:10FC80002B462A4625836583677503F0B1F8002863
:10FC90007FF4D0AEB770CDE6E4BD0120A8C301204B
:10FCA000C8C30120092003F0EFFA00287FF4C2AE98
:10FCB0000423A370BEE6C64EC64F00252B462A4637
:10FCC0004FF0050E2575258365833146012538469D
:10FCD00084F815E0E58203F08BF800287FF4AAAEE3
:10FCE0000220FDF7F7FED6F8803086F820501B6A18
:10FCF000984796F8203031790322B2701BB107EB98
:10FD0000411787F8AC33B34D2846FDF73DFE94F814
:10FD1000203061791BB105EB411585F8AC33AD4856
:10FD2000FDF732FE86E6122003F0CCFB00287FF4BC
:10FD300081AED4F88030A848DB6998470223A370CD
:10FD400078E6082003F0BEFB00287FF473AE94F839
:10FD50002930A048A371FDF7D5FE6179A37905EBA1
:10FD600041120126B2F8B203A670984202D00BB13C
:10FD7000A2F8B2339748FDF707FE2179A37905EB86
:10FD80004115B5F8B2239A42C9D0002BC7D0A5F8C7
:10FD9000B233C4E7A37B8E4A0133DBB2022BA373D9
:10FDA00040F23F81082153789174137042E66379E1
:10FDB000874A1D4495F89B33DBB2012B00F02C8160
:10FDC000022B00F04C81032B7FF434AE0B232377FE
:10FDD00030E661797F4801F1150205EB42120223FA
:10FDE00005EB411682F814310023C2F818316F1860
:10FDF000012286F8AE33C6F8BC33C6F8C03386F8A5
:10FE0000C52387F89B33FDF719FD0A23237711E6F5
:10FE100023796F496F4A1D4495F89B33DBB2012B60
:10FE200000F0FA80032BD1D052696C4892680D8A99
:10FE3000008892B2521B8242C8D8042B7FF4FAADDC
:10FE40004A788B740A70F5E56179654F614801F174
:10FE5000150305EB431305EB4112032683F81461E8
:10FE60000D44C3F818710826002382F8AE33C2F897
:10FE7000C033C2F8BC6385F89B33FDF7DFFC022377
:10FE80002377D7E52179A268A789524801F11503A4
:10FE900005EB4313022683F8146105EB4116C3F802
:10FEA00018210D4400230122C6F8C03386F8AE2382
:10FEB000C6F8BC7385F89B33FDF7C0FC0423237799
:10FEC000B8E56379474A2B44116893F89B33DBB25A
:10FED0008B4218BF1360012B00F0A680032B7FF428
:10FEE000A9AD0B2205232277A374A3E52179394814
:10FEF00001F1150205EB42126F18022605EB4115C0
:10FF0000002382F814610126C2F81831C5F8BC3309
:10FF1000C5F8C03385F8AE6387F89B33FDF78EFCD8
:10FF20000823237786E56179A789A6684B0105EB4D
:10FF3000030E01F115024FF0000801F11E008EF8CA
:10FF4000AE8305EB42182B4405EB401005EB421243
:10FF50004FF0010CCEF8BC73C8F818610D440026B0
:10FF6000022780F805C0C3F8C0631A4882F81471EC
:10FF700085F89B63FDF762FC062323775AE5237916
:10FF8000134A2B4493F89B33DBB2012B5ED0042B36
:10FF90005FD0032B3FF41AAF6B69104A9B68218A2C
:10FFA00012889BB25B1A93423FF610AF42E5637929
:10FFB000074A1D4495F89B33DBB2012B4CD0042B30
:10FFC00050D0022B7FF4FFAE0523137732E500BF3C
:10FFD000A8C30120E4BD0120CAC3012034B7012019
:10FFE000BCC301209C000020D4F880302648DB6A86
:10FFF00098470723A3701DE5D4F8803022489B6AF8
:020000040801F1
:1000000098470623A37015E5D4F880301E481B6B73
:1000100098470823A3700DE5637823700D23237799
:1000200008E50123137705E5237D618B174A23F04B
:100030007F03DBB2D9B1164941F288300880EBB9B1
:10004000052313776B699B682382F3E409231377F5
:10005000A2E753781370EDE407231377EAE409234A
:100060001377E7E4537813700C231377E2E408491D
:10007000322008802BB907231377E3E70323137794
:10008000E0E709231377DDE778730108A8C30120AF
:1000900034B7012030B5824283B0044617D04FF602
:1000A000E0724FF6FF75012B08BF15460B46094A53
:1000B0000948152105F072FC21010022009240310F
:1000C0002B4650220448FEF78DFE03B030BD4FF49E
:1000D0007845EBE77C730108F4B6012070B5134D49
:1000E000134C82B050220026114628464FF6FF736B
:1000F0000096FEF777FE284605F0C0FC4FF47843E3
:10010000C50005F150022046009350214FF6FF73C1
:10011000FEF768FE009605F1580220464FF6FF7381
:100120005021FEF75FFE02B070BD00BF24B7012072
:100130008473010882B000230193019B0133332BA8
:100140000193FAD902B0704700B583B00023154877
:100150000193154AFFF7EEFFC3681969019106E0A4
:10016000FFF7E8FFC368013A1969019115D00199B9
:100170000029F5DA01990C4A41F001010191019938
:1001800019611969019103E019690191013A02D0DD
:100190000199C907F8D4FFF7CDFF002003B05DF83F
:1001A00004FB00BFE4BD0120400D030008B5114A67
:1001B00092F8C83092F8C910003318BF0123022901
:1001C00014D003290FD001290AD0002182F8C910C8
:1001D000094A1360FFF72CFB084B00221A6008BD88
:1001E00043F00403F4E743F00603F1E743F00203AE
:1001F000EEE700BF38B70120EC3600201CB7012025
:100200000C4A0D4B70B4136003F5804603F50045AE
:1002100003F54043D360B0F5804F084B084C56605F
:100220004FF00001956006BF01221A60196021603D
:1002300070BC70470CB701200000001020B70120EF
:10024000F0B601200209130700F00F000AD410B421
:10025000094901238C5C03FA00F0204388545DF8BF
:10026000044B7047054901220B7802FA00F023EA9B
:1002700000000870704700BF9400002036B70120CE
:1002800003091A0700F00F000BD410B4094C012128
:10029000E25C01FA00F022EA0000E0545DF8044B51
:1002A0007047054901220B7802FA00F018430870E4
:1002B000704700BF9400002036B70120FE2907D008
:1002C0001F2900F08D807F2900F08480FF20704777
:1002D000F0B54A4BD3F8C420C0435207C3B262D52D
:1002E00013F0010E1CBF464A107803F0020208BF4B
:1002F000FF2002F0FF0712B1414A5278104003F08C
:10030000040202F0FF0612B13D4A9278104003F059
:10031000080202F0FF0512B1394AD278104003F00A
:10032000100202F0FF0412B1354A1279104003F0B6
:10033000200202F0FF0112B1314A5279104003F05D
:10034000400C0CF0FF02BCF1000F05D0DFF8B0C08C
:100350009CF806C000EA0C005BB2002B47DBBEF144
:10036000000F05D0DFF89CE09EF800E000EA0E00E8
:1003700017B1244F7F78384016B1224EB6783040FE
:1003800015B1204DED78284014B11E4C2479204041
:1003900011B11C494979084012B11A4A92791040AA
:1003A000002B20DBF0BD03F0020703F0040603F08E
:1003B000080503F0100403F0200103F0400203F0ED
:1003C000010EFFB2F6B2EDB2E4B2C9B2D2B25BB284
:1003D000FF20C4E7FF287FF479AF0B4B18787047F4
:1003E0000A4B18787047074BDB791840F0BDDFF8EF
:1003F00010C09CF807C000EA0C00B0E738B7012035
:10040000E436002094000020A000002036B7012030
:10041000002070470023C0F810331846704700BF13
:100420000123C0F810330020704700BFF8B53E4DDF
:1004300095F845300446042B23D8DFE803F03C242C
:100440003C1303000023012221270B26CA820F75CB
:100450004E750B834B831A4602F0CAFC88B985F8A7
:100460004500F8BD00230A2221264A750E75CB826D
:100470000B834B831A4602F0BBFC00284FD00328A5
:100480004DD00120F8BD294B4FF4085000221B89A4
:10049000C882812706260A834B830F754E7504F5A3
:1004A0008872204602F0A4FC0028EAD1032385F8D4
:1004B00045300120F8BD4FF4045000228127062664
:1004C0000923C8820A830F754E754B8304F5887221
:1004D000204602F08DFC0028D3D194F8130194F843
:1004E0001211124B94F8186194F8172194F81071B6
:1004F0001F7001EB002194F8110194F814715980D8
:1005000002EB062294F8161194F815615870012038
:100510001F715E7199711A8185F84500F8BD042339
:1005200085F845300120F8BD88BC012008B80120BD
:1005300070B51A4C94F840100546E9B994F841108A
:10054000164E19B9164B00221A7070BD2846FDF7D9
:1005500055F996F84130072B07D805EB4305B5F858
:100560008C35C3F30E03A5F88C35002384F8413095
:100570000B4B00221A7070BDFDF740F994F8403023
:10058000072B07D805EB4303B3F88C25C2F30E0203
:10059000A3F88C25002384F84030CFE788BC0120E5
:1005A000C3BD012030B400F28A52002332F9024F59
:1005B000002CDDB205DA0133082BF7D1FF2030BC67
:1005C000704700EB43006FEA41416FEA5141A0F8E8
:1005D0008C15284630BC7047F8B500EB410500EBA0
:1005E0004114B5F88C559DF8187084F8AC2305F0CB
:1005F0007F06C5F3C01584F8AD6384F8AE53BDF82B
:100600001C6084F8AF33002584F8B173A4F8B2639A
:1006100084F8C45384F8C55313B9012384F8B03364
:10062000FDF7B2F90020F8BD2DE9F04391F8443010
:10063000364D0622012B83B00C4685F8422007D0A8
:10064000D1F880301B6C9847012003B0BDE8F083DF
:1006500091F84530012B074654D0022B04BF2C4B98
:100660002B6594F8561094F85230B4F8540085F87D
:100670004830002285F8422085F845200929234A80
:10068000A5F8460098BF0A21A2F84A1094F84260E3
:10069000022E28BF02267EB3013EF6B21A0604EBF4
:1006A000C606A0464FF00309194638461CD485F803
:1006B0004330FFF777FF014685F84100B5F8460063
:1006C00094F8213094F820200190CDF8009038461D
:1006D000FFF782FFB0450FD098F85A301A0608F19C
:1006E000080819463846E2D585F84430FFF75AFF26
:1006F000014685F84000E1E7064B0020187003B082
:10070000BDE8F083044B2B65ABE700BF88BC01203C
:10071000B8000020C3BD0120A400002080B485B033
:1007200000AF78607B68D3F890301B68BB60FB7AC1
:1007300043F08003FB72FB7A43F04003FB727B685B
:10074000D3F89030BA681A600023FB60BB7B43F09B
:100750002003BB737B68DB68FA685A610123184683
:100760001437BD465DF8047B704700BF80B588B084
:1007700000AF78600023FB7200237B613B7D43F078
:1007800010033B757B68DB687A68D26891697A6987
:10079000D2430A409A617B68DB681B6ABB613B7E7F
:1007A000C3F30303DBB2FB72FB7ADBB27A6822335A
:1007B0009B0013449B681B68FB60BB7EC3F3430331
:1007C000DBB2022B40F08D803B8BC3F30A139BB24C
:1007D000002B40F38580FB7ADBB27A6815335B012E
:1007E000134403F58C731B68002B79D0FB7ADBB2C2
:1007F0007A6815335B01134403F58C7319683B8BDE
:10080000C3F30A139BB21A467868FDF73BF93B7EA7
:10081000C3F30303DBB218463B7EC3F30303DBB22F
:100820007A6815335B01134403F58C731B683A8BAC
:10083000C2F30A1292B21A44796800F115035B01FF
:100840000B4403F58C731A603B7EC3F30303DBB2E6
:1008500018463B7EC3F30303DBB27A685B011344A3
:1008600003F570731B683A8BC2F30A1292B21A44F2
:10087000796843010B4403F570731A60FB7ADBB2AD
:100880007A685B01134403F570731B68FB61FB7AA4
:10089000DBB21A467B68D432F96943F82210FB7A3E
:1008A000DBB27A6822339B0013449B681B693B616F
:1008B0007B8AC3F3C9039BB2002B11DDFB7B43F0A2
:1008C0008003FB73FB7B6FF38613FB73FB7ADBB256
:1008D0007A6822339B0013449B68FA681A6000E030
:1008E00000BF3B7D43F010033B757B68DB687A6893
:1008F000D26891697A690A439A61012318462037C0
:10090000BD4680BD80B59CB000AF786039607A6824
:100910003B6822339B0013449B68FB66FB6E9B681D
:10092000BB66FB6EDB687B66BA6E7B6E1340BB6694
:100930007A683B6822339B0013449B681B683B66C4
:1009400000237B6697F8683003F00403DBB2002BCA
:100950001DD00023FB603B7B43F004033B73FA682C
:10096000FB6E9A607A683B6822339B0013449B6855
:10097000DB683B613B7C43F002033B747A683B6875
:1009800022339B0013449B683A69DA6093E097F83E
:10099000683003F02003DBB2002B09D000237B6119
:1009A0003B7D43F020033B757A69FB6E9A6082E0E1
:1009B00097F8683003F00803DBB2002B3BD07A686D
:1009C0003B6822339B0013449B68DB68BB613B7E22
:1009D00043F002033B767A683B6822339B00134462
:1009E0009B68BA69DA607A683B68134403F56373FD
:1009F00005221A700023FB613B7F43F010033B7715
:100A0000FA69FB6E9A6000233B6297F8203043F04E
:100A1000080387F820303A6AFB6E9A6097F86830CE
:100A20006FF3041387F868303B68DBB219467868C7
:100A3000FCF7E4FE3FE097F8693003F00403DBB213
:100A4000002B38D07A683B6822339B0013449B68A4
:100A5000DB687B6297F8243043F0020387F8243088
:100A60007A683B6822339B0013449B687A6ADA6099
:100A70003B68DBB219467868FCF7C0FE0023BB6216
:100A800097F8283043F0100387F82830BA6AFB6ED5
:100A90009A607A683B68134403F5637308221A70FE
:100AA0000023FB6297F82D3043F0040387F82D30C4
:100AB000FA6AFB6E9A6097F8693003F00203DBB2C2
:100AC000002B27D07A683B6822339B0013449B6835
:100AD000DB683B6397F8303043F0020387F830302F
:100AE0007A683B6822339B0013449B683A6BDA6058
:100AF0003B68DBB219467868FCF780FE00237B6315
:100B000097F8353043F0020387F835307A6BFB6E87
:100B10009A60CBE197F8683003F00103DBB2002B59
:100B200000F09B807B68DB78012B17D17A683B68EB
:100B300022339B0013449B681B69FB657A683B6802
:100B40005B01134403F56F731B68FA6DC2F3120265
:100B5000991A7B683A68D43243F822107A683B6865
:100B6000134403F5637301221A707A683B68C43337
:100B70009B00134400225A600023BB6397F838306F
:100B800043F0010387F83830BA6BFB6E9A6097F830
:100B9000623003F00C03DBB2002B06D097F8623012
:100BA00003F00C03DBB2082B39D17A683B6822339F
:100BB0009B0013449B68DB68FB6397F83C3043F071
:100BC000020387F83C307A683B6822339B00134469
:100BD0009B68FA6BDA603B68DBB219467868FCF711
:100BE0000DFE00233B6497F8403043F0100387F874
:100BF00040303A6CFB6E9A607A683B681E335B014A
:100C0000134404331B7883F00103D9B27A683B683C
:100C10001E335B01134404330A461A7045E197F80A
:100C2000623003F00C03DBB20C2B40F03E8197F8EE
:100C3000633043F0200387F863307A683B682233DF
:100C40009B0013449B683A6E1A607A683B681344B1
:100C500003F29B3301221A7028E197F8683003F001
:100C60000203DBB2002B7DD07A683B6822339B0005
:100C700013449B68DB687B6497F844306FF341034F
:100C800087F844307A683B6822339B0013449B68A2
:100C90007A6CDA607A683B68134403F563731B78F7
:100CA000DBB2012B07D17A683B68134403F29B3314
:100CB00001221A704AE07A683B68134403F56373B3
:100CC0001B78DBB2052B07D17A683B68134403F22B
:100CD0009B3304221A7039E07A683B68134403F5A9
:100CE00063731B78DBB2062B08D07A683B68134429
:100CF00003F563731B78DBB2082B0ED17A683B686F
:100D0000C4339B00134400225A607A683B68134442
:100D100003F29B3303221A7018E097F8623003F055
:100D20000C03DBB20C2B11D17A683B681E335B01DC
:100D3000134404331B7883F00103D9B27A683B680B
:100D40001E335B01134404330A461A700023BB644C
:100D500097F8483043F0020387F84830BA6CFB6ECE
:100D60009A60A3E097F8683023F07F03DBB2002B92
:100D70003BD07A683B6822339B0013449B68DB6856
:100D8000FB6497F84C3043F0020387F84C307A68E4
:100D90003B6822339B0013449B68FA6CDA607A68E4
:100DA0003B68C4339B0013445B685A1C79683B68FA
:100DB000C4339B000B445A607A683B68134403F5C4
:100DC000637306221A703B68DBB219467868FCF739
:100DD00015FD00233B6597F8503043F0800387F8FA
:100DE00050303A6DFB6E9A6060E097F8683003F01F
:100DF0001003DBB2002B59D097F8623003F00C03DC
:100E0000DBB20C2B1CD17A683B6822339B00134465
:100E10009B68DB687B6597F8543043F0020387F8E2
:100E200054307A683B6822339B0013449B687A6D88
:100E3000DA603B68DBB219467868FCF7DFFC21E03A
:100E400097F8623003F00C03DBB2002B06D097F862
:100E5000623003F00C03DBB2082B13D197F8633038
:100E600043F0800387F8633097F863306FF386139D
:100E700087F863307A683B6822339B0013449B6891
:100E80003A6E1A607A683B68134403F56373032271
:100E90001A700023BB6597F8583043F0100387F8A9
:100EA0005830BA6DFB6E9A6000E000BF012318460F
:100EB0007037BD4680BD00BF80B59AB000AF786086
:100EC00039607A683B6822339B0013449B687B66D9
:100ED0007B6E9B683B667B6EDB68FB653A6EFB6DE9
:100EE00013403B667A683B6822339B0013449B683F
:100EF0001B68BB6597F8603003F00403DBB2002B7E
:100F00001DD00023BB603B7A43F004033B72BA68F8
:100F10007B6E9A607A683B6822339B0013449B681F
:100F2000DB68FB603B7B43F002033B737A683B6802
:100F300022339B0013449B68FA68DA6060E297F8FA
:100F4000603003F02003DBB2002B09D000233B61AB
:100F50003B7C43F020033B743A697B6E9A604FE21E
:100F600097F8613003F00203DBB2002B23D07A68DC
:100F70003B6822339B0013449B68DB687B613B7DAD
:100F800043F002033B757A683B6822339B001344AD
:100F90009B687A69DA603B68DBB219467868FCF7CF
:100FA0002DFC0023BB617B7E43F002037B76BA6994
:100FB0007B6E9A6024E297F8603003F00103DBB2A5
:100FC000002B33D07A683B68C4339B001344002263
:100FD0005A607A683B6822339B0013449B68DB6845
:100FE000FB613B7F43F002033B777A683B68223327
:100FF0009B0013449B68FA69DA603B68DBB21946D0
:101000007868FCF7FBFB00233B6297F8203043F045
:10101000010387F820303A6A7B6E9A607A683B68F1
:10102000134403F5637301221A70E9E197F8603005
:1010300003F00803DBB2002B2ED000237B6297F86D
:10104000243043F0080387F824307A6A7B6E9A6074
:101050007A683B6822339B0013449B68DB68BB6261
:1010600097F8283043F0020387F828307A683B6805
:1010700022339B0013449B68BA6ADA603B68DBB298
:1010800019467868FCF7BAFB7A683B68134403F5A5
:10109000637305221A70B3E197F8603003F0100310
:1010A000DBB2002B35D07A683B68C4339B00134415
:1010B00000225A607A683B6822339B0013449B6885
:1010C000DB68FB6297F82C3043F0020387F82C3082
:1010D0007A683B6822339B0013449B68FA6ADA60A3
:1010E0003B68DBB219467868FCF788FB00233B635A
:1010F00097F8303043F0100387F830303A6B7B6E4E
:101100009A607A683B68134403F5637303221A708C
:1011100076E197F8603023F07F03DBB2002B3BD001
:101120007A683B6822339B0013449B68DB687B63CF
:1011300097F8343043F0020387F834307A683B681C
:1011400022339B0013449B687A6BDA603B68DBB206
:1011500019467868FCF752FB7A683B68C4339B00F9
:1011600013445B685A1C79683B68C4339B000B448A
:101170005A607A683B68134403F5637306221A7059
:101180000023BB6397F8383043F0800387F838308A
:10119000BA6B7B6E9A6033E197F8603003F04003DE
:1011A000DBB2002B35D07A683B68C4339B00134414
:1011B00000225A607A683B6822339B0013449B6884
:1011C000DB68FB6397F83C3043F0020387F83C3060
:1011D0007A683B6822339B0013449B68FA6BDA60A1
:1011E0003B68DBB219467868FCF708FB00233B64D8
:1011F00097F8403043F0400387F840303A6C7B6EFC
:101200009A607A683B68134403F5637304221A708A
:10121000F6E097F8613003F00403DBB2002B39D01D
:101220007A683B6822339B0013449B68DB687B64CD
:1012300097F8443043F0020387F844307A683B68FB
:1012400022339B0013449B687A6CDA603B68DBB204
:1012500019467868FCF7D2FA0023BB6497F8483047
:1012600043F0100387F84830BA6C7B6E9A607A6856
:101270003B68134403F5637308221A700023FB6470
:1012800097F84D3043F0040387F84D30FA6C7B6ECD
:101290009A60B5E097F8603003F00203DBB2002BF0
:1012A00000F0AE807A683B6822339B0013449B6851
:1012B000DB683B6597F850306FF3410387F8503097
:1012C0007A683B6822339B0013449B683A6DDA606E
:1012D0007A683B68134403F563731B78DBB2012B18
:1012E00020D17A683B68134403F29B3301221A70C1
:1012F00097F85A3003F00C03DBB2082B74D17A68EC
:101300003B681E335B01134405331B7883F00103F4
:10131000D9B27A683B681E335B01134405330A4631
:101320001A7062E07A683B68134403F563731B78B4
:10133000DBB2032B07D17A683B68134403F29B337B
:1013400002221A7051E07A683B68134403F5637314
:101350001B78DBB2042B16D17A683B685B0113441F
:1013600003F56C731B78012B05D13B68DBB2194682
:101370007868FCF72FFA7A683B68134403F29B33D2
:1013800002221A7031E07A683B68134403F56373F4
:101390001B78DBB2052B07D17A683B68134403F254
:1013A0009B3304221A7020E07A683B68134403F5EB
:1013B00063731B78DBB2062B17D17A683B68C433A2
:1013C0009B0013445B68032B0FD17A683B6813447E
:1013D00003F29B3303221A707A683B68C4339B0084
:1013E000134400225A6000E000BF00237B6597F899
:1013F000543043F0020387F854307A6D7B6E9A6064
:10140000012318466837BD4680BD00BF80B588B04F
:1014100000AF78600023FB610023BB610023FB6009
:1014200000237B6100233B617B68D3F8CC301B68D1
:101430007B617B68D3F8CC301B683B613B7C6FF3EE
:1014400082033B743B7C6FF341033B743B7C6FF343
:10145000C3033B743B7C6FF345133B743B7D03F04C
:101460000203DBB2002B0CD03B7C43F002033B7445
:101470003F4B1B685B6878689847BB6943F0010382
:10148000BB613B7D03F00803DBB2002B52D03B7CF9
:1014900043F008033B743B7D03F00403DBB2002BF5
:1014A00048D0334B1B685B6878689847BB7D03F076
:1014B0000603DBB2042B05D0BB7D03F00603DBB2D1
:1014C000022B31D17B685B691B68FB60BB7D03F03D
:1014D0000603DBB2042B15D17B685B6941F27072A5
:1014E0005A603B7B03F00303DBB2022B1FD07B6807
:1014F0001B7A022B03D102217868FCF7BDFA012385
:10150000FB6116E07B685B694BF680325A603B7B7F
:1015100003F00303DBB2012B0BD001217868FCF749
:10152000ABFA0123FB6104E00123FB6102E000BF91
:1015300000E000BF3B7D03F02003DBB2002B07D0AF
:101540003B7C43F020033B74BB6943F00103BB6168
:10155000FB69002B02D07868FCF7D4FA7B68D3F8DB
:10156000CC303A691A60BB6918462037BD4680BD49
:10157000A873010880B586B000AF78607B685B69AE
:101580001B69BB603B7BC3F3C303DBB27A685B01BF
:10159000134403F56F731B6803339B08FB8296E0CB
:1015A0003B899B00BB82BA8A3B7BC3F3C303DBB29C
:1015B00079685B010B4403F56F731B689A4219D974
:1015C0003B7BC3F3C303DBB27A685B01134403F5CF
:1015D0006F731B68BB8200233B61FB7C43F00403F9
:1015E000FB747B68DB687A68D26891693A69D24398
:1015F0000A409A613B7BC3F3C303DBB27A685B01A9
:10160000134403F56F731B6803339B08FB823B7B1A
:10161000C3F3C303DBB27A6815335B01134403F5EC
:101620008C7319683B7BC3F3C303DBB21A46BB8AD6
:101630007868FCF73BFA3B7BC3F3C303DBB2184685
:101640003B7BC3F3C303DBB27A6815335B011344FE
:1016500003F58C731A68BB8A1A44796800F1150384
:101660005B010B4403F58C731A603B7BC3F3C3032C
:10167000DBB218463B7BC3F3C303DBB27A685B0182
:10168000134403F56F731A68BB8AD21A7968430151
:101690000B4403F56F731A603B7BC3F3C303DBB2E8
:1016A00018463B7BC3F3C303DBB27A685B01134488
:1016B00003F570731A68BB8A1A44796843010B44B6
:1016C00003F570731A607B685B691B69BB603B89BB
:1016D000FA8A9A420CD23B7BC3F3C303DBB27A682B
:1016E0005B01134403F56F731B68002B7FF458AF45
:1016F000012318461837BD4680BD00BF80B588B0AD
:1017000000AF78607B68DB68DB6AFB603B7CC3F31F
:10171000C303DBB27A685B01134403F56F731B6884
:1017200003339B08FB8396E0BB899B00BB83BA8B8A
:101730003B7CC3F3C303DBB279685B010B4403F565
:101740006F731B689A4219D93B7CC3F3C303DBB2A6
:101750007A685B01134403F56F731B68BB83002336
:10176000BB613B7E43F020033B767B68DB687A6895
:10177000D2689169BA69D2430A409A613B7CC3F34B
:10178000C303DBB27A685B01134403F56F731B6814
:1017900003339B08FB833B7CC3F3C303DBB27A6850
:1017A00015335B01134403F58C7319683B7CC3F359
:1017B000C303DBB21A46BB8B7868FCF777F93B7C36
:1017C000C3F3C303DBB218463B7CC3F3C303DBB2F2
:1017D0007A6815335B01134403F58C731A68BB8B6D
:1017E0001A44796800F115035B010B4403F58C730F
:1017F0001A603B7CC3F3C303DBB218463B7CC3F3E4
:10180000C303DBB27A685B01134403F56F731A6894
:10181000BB8BD21A796843010B4403F56F731A60CE
:101820003B7CC3F3C303DBB218463B7CC3F3C30367
:10183000DBB27A685B01134403F570731A68BB8BE3
:101840001A44796843010B4403F570731A607B688E
:10185000DB68DB6AFB60BB89FA8B9A420CD23B7C6B
:10186000C3F3C303DBB27A685B01134403F56F7300
:101870001B68002B7FF458AF012318462037BD4664
:1018800080BD00BF80B584B000AF78600023FB60EE
:10189000084B1B689B6878689847FB7B43F02003E4
:1018A000FB737B68DB68FA685A61012318461037BE
:1018B000BD4680BDA873010880B584B000AF7860D4
:1018C0000023FB60084B1B681B68786898473B7BCC
:1018D00043F008033B737B68DB68FA685A610123B5
:1018E00018461037BD4680BDA87301082DE9F041A8
:1018F000DFF84080D8F80030984216D20C4E0546EA
:101900000F1A06EB001600240023314620463A4603
:10191000FEF7C0FBD8F800300135AB4204F10104FA
:1019200006F1100601D9072CEED1BDE8F08100BF09
:101930005CB801201CB8012004F08EB838B52A4BE1
:1019400019685A69140601D5080600D438BD8021EB
:10195000264A596113691906F8D413695B060ED437
:10196000234A1378591E072903D8224801784908C9
:1019700001700133DBB20A2B0DD8137038BD1C4A3D
:101980001378591E0729F4D81A480178490861F0DC
:101990007F010170EDE7174C20780023F0281370C9
:1019A00013D0E02817D0144D144A2B8811881843FF
:1019B000814205D0124B10801B6893B1114B186007
:1019C00000232B600023237038BD0B4A136843F4B7
:1019D00000731360F6E7084A136843F480731360DA
:1019E000F0E7FDF7D7FBEBE7003C014000040240C5
:1019F00038B8012012B8012018B801205CBC0120C1
:101A000034B801204025002038B5104C104D03E0BB
:101A10000020FDF785FC48B92368002BF8D1FDF7BD
:101A200025FC0020FDF77CFC0028F5D02B68022B5C
:101A300006D0FDF769FE0028EED1064B186038BDD0
:101A4000FDF786FE0028E7D1F7E700BF2CB801209C
:101A500030B8012014B801202DE9F0411F4B204E71
:101A60001F780023044602460D46184656F82710F4
:101A7000FEF710FB224600231A490120FEF70AFB5D
:101A80002246002318490220FEF704FB22460023C9
:101A900016490320FEF7FEFAC5B92B462246144923
:101AA0000420FEF7F7FA2246002312490520FEF72C
:101AB000F1FA114A114B92F880100620224653F891
:101AC0002110BDE8F0410023FEF7E4BA01232246CD
:101AD0000B490420FEF7DEFAE5E700BFC000002056
:101AE000C074010804740108F86101081462010857
:101AF000187401082074010838B70120FC7301082C
:101B00000C7401082DE9F843644BD3F8C4305A072C
:101B100011D4634B1C6800221A604CB9614B1B68DE
:101B200033B1614B1B68012B00F08480002B59D02E
:101B30002046BDE8F8835D4CDFF888915C4E0027B5
:101B40004FF0FF054FF0010808FA07F3DB43DBB263
:101B5000A9F81A500F20A9F81830FAF78DFE33694A
:101B6000DB4303F01F034744042004F8013FFAF766
:101B700075FE082FE6D14F480778FB0711D54E4D6B
:101B800002792B795340DF0635D512F0100F444B04
:101B900040F2723418BF4FF4B97403C885E80300EB
:101BA000B9E7C37903F0020303F0FF017BBB424DA9
:101BB000DFF814C10A46864677B1AE5C00237E404A
:101BC00008FA03F4344212D002EB82010B443CF8D1
:101BD000131009B127424BD00132082A25D01EF834
:101BE000017FE9E7FDF742FB2046BDE8F8830133BA
:101BF000052BE5D1F0E71E0730D4DC073BD512F00A
